:020000040800F2
:1000000000500020C1980008A9980008AB9800088B
:10001000AD980008AF980008B198000800000000F3
:10002000000000000000000000000000B39800087D
:10003000B598000800000000B7980008B9980008BB
:100040000999000809990008099900080999000808
:1000500009990008099900080999000809990008F8
:1000600009990008099900080999000809990008E8
:1000700009990008099900080999000809990008D8
:1000800009990008099900080999000809990008C8
:1000900009990008099900080999000809990008B8
:1000A00009990008099900080999000809990008A8
:1000B000352A0008099900080999000809990008DB
:1000C0000999000809990008099900080999000888
:1000D00009990008BD230008099900087942000821
:1000E000D17D000809990008099900080000000066
:1000F0000000000000000000000000000000000000
:0C01000000000000000000005FF808F1A3
:1001100010B5054C237833B9044B13B10448AFF341
:1001200000800123237010BD280000200000000083
:10013000DCB3000808B5034B1BB103490348AFF318
:10014000008008BD000000002C000020DCB3000887
:1001500010F8012B11F8013B012A28BF9A42F7D071
:10016000D01A7047034613F8012B002AFBD1181A46
:100170000138704780F0004002E000BF81F000418C
:1001800042001FBF5FEA410392EA030F7FEA226C3D
:100190007FEA236C6AD04FEA1262D2EB1363C1BFCD
:1001A000D218414048404140B8BF5B42192B88BF3C
:1001B000704710F0004F40F4000020F07F4018BF5F
:1001C000404211F0004F41F4000121F07F4118BF7F
:1001D000494292EA030F3FD0A2F1010241FA03FC27
:1001E00010EB0C00C3F1200301FA03F100F000430F
:1001F00002D5494260EB4000B0F5000F13D3B0F1D7
:10020000807F06D340084FEA310102F10102FE2A45
:1002100051D2B1F1004F40EBC25008BF20F00100B5
:1002200040EA03007047490040EB0000013A28BF54
:10023000B0F5000FEDD2B0FA80FCACF1080CB2EBD7
:100240000C0200FA0CF0AABF00EBC2505242184355
:10025000BCBFD0401843704792F0000F81F40001FA
:1002600006BF80F400000132013BB5E74FEA4103CD
:100270007FEA226C18BF7FEA236C21D092EA030F39
:1002800004D092F0000F08BF0846704790EA010FB3
:100290001CBF0020704712F07F4F04D1400028BFE0
:1002A00040F00040704712F100723CBF00F50000C2
:1002B000704700F0004343F0FE4040F400007047F8
:1002C0007FEA226216BF08467FEA236301464202A4
:1002D00006BF5FEA412390EA010F40F480007047B7
:1002E0004FF0000304E000BF10F0004348BF40425D
:1002F0005FEA000C08BF704743F0964301464FF099
:1003000000001CE050EA010208BF70474FF00003F4
:100310000AE000BF50EA010208BF704711F0004335
:1003200002D5404261EB41015FEA010C02BF844605
:100330000146002043F0B64308BFA3F18053A3F564
:100340000003BCFA8CF2083AA3EBC25310DB01FAAB
:1003500002FC634400FA02FCC2F12002BCF1004F2F
:1003600020FA02F243EB020008BF20F001007047C0
:1003700002F1200201FA02FCC2F1200250EA4C0014
:1003800021FA02F243EB020008BF20EADC7070475A
:100390004FF0FF0C1CEAD0521EBF1CEAD15392EA68
:1003A0000C0F93EA0C0F6FD01A4480EA010C400244
:1003B00018BF5FEA41211ED04FF0006343EA50109E
:1003C00043EA5111A0FB01310CF00040B1F5000FE0
:1003D0003EBF490041EAD3715B0040EA010062F18F
:1003E0007F02FD2A1DD8B3F1004F40EBC25008BF79
:1003F00020F00100704790F0000F0CF0004C08BF97
:1004000049024CEA502040EA51207F3AC2BFD2F163
:10041000FF0340EAC250704740F400004FF0000371
:10042000013A5DDC12F1190FDCBF00F000407047AB
:10043000C2F10002410021FA02F1C2F1200200FAE9
:1004400002FC5FEA310040F1000053EA4C0308BFB0
:1004500020EADC70704792F0000F00F0004C02BF01
:10046000400010F4000F013AF9D040EA0C0093F07C
:10047000000F01F0004C02BF490011F4000F013BD6
:10048000F9D041EA0C018FE70CEAD15392EA0C0F44
:1004900018BF93EA0C0F0AD030F0004C18BF31F0AF
:1004A000004CD8D180EA010000F00040704790F085
:1004B000000F17BF90F0004F084691F0000F91F029
:1004C000004F14D092EA0C0F01D142020FD193EAEF
:1004D0000C0F03D14B0218BF084608D180EA010077
:1004E00000F0004040F0FE4040F40000704740F053
:1004F000FE4040F4400070474FF0FF0C1CEAD05221
:100500001EBF1CEAD15392EA0C0F93EA0C0F69D07C
:10051000A2EB030280EA010C49024FEA402037D0E7
:100520004FF0805343EA111143EA10130CF00040DE
:100530008B4238BF5B0042F17D024FF4000C8B42CE
:1005400024BF5B1A40EA0C00B3EB510F24BFA3EBAE
:10055000510340EA5C00B3EB910F24BFA3EB91037E
:1005600040EA9C00B3EBD10F24BFA3EBD10340EAD8
:10057000DC001B0118BF5FEA1C1CE0D1FD2A3FF61E
:1005800050AF8B4240EBC25008BF20F001007047D3
:100590000CF0004C4CEA50207F32C2BFD2F1FF0376
:1005A00040EAC250704740F400004FF00003013AA7
:1005B00037E792F0000F00F0004C02BF400010F44B
:1005C000000F013AF9D040EA0C0093F0000F01F05F
:1005D000004C02BF490011F4000F013BF9D041EA81
:1005E0000C0195E70CEAD15392EA0C0F08D14202B4
:1005F0007FF47DAF93EA0C0F7FF470AF084676E787
:1006000093EA0C0F04D14B023FF44CAF08466EE75F
:1006100030F0004C18BF31F0004CCAD130F000422D
:100620007FF45CAF31F000437FF43CAF5FE700BF85
:100630004FF0FF3C06E000BF4FF0010C02E000BFAE
:100640004FF0010C4DF804CD4FEA40024FEA410350
:100650007FEA226C18BF7FEA236C11D001B052EA06
:10066000530C18BF90EA010F58BFB2EB030088BFCC
:10067000C81738BF6FEAE17018BF40F0010070473B
:100680007FEA226C02D15FEA402C05D17FEA236C1D
:10069000E4D15FEA412CE1D05DF8040B704700BF64
:1006A000844608466146FFE70FB5FFF7C9FF0028FB
:1006B00048BF10F1000F0FBD4DF808EDFFF7F4FF34
:1006C0000CBF012000205DF808FB00BF4DF808EDCD
:1006D000FFF7EAFF34BF012000205DF808FB00BFF0
:1006E0004DF808EDFFF7E0FF94BF012000205DF812
:1006F00008FB00BF4DF808EDFFF7D2FF94BF0120C3
:1007000000205DF808FB00BF4DF808EDFFF7C8FFBB
:1007100034BF012000205DF808FB00BF4FEA400213
:10072000B2F1FE4F0FD34FF09E03B3EB12620DD91F
:100730004FEA002343F0004310F0004F23FA02F089
:1007400018BF404270474FF00000704712F1610F30
:1007500001D1420205D110F0004008BF6FF0004007
:1007600070474FF00000704742000ED2B2F1FE4FCA
:100770000BD34FF09E03B3EB126209D44FEA002370
:1007800043F0004323FA02F070474FF00000704737
:1007900012F1610F01D1420202D14FF0FF307047D8
:1007A0004FF00000704700BF0022427082700122AB
:1007B000C2700222B1FA81F102710322490901706B
:1007C0004271704743788B421FD0012941700AD093
:1007D000022910D0C1B90123C370022381700371B3
:1007E000032343717047037843B1012383700223CD
:1007F000C3700023F3E70378002BF6D00223837045
:100800000023C3700123EAE7FEE770470B8882B03C
:10081000ADF800304B880239ADF80230CB88ADF826
:1008200004300B89ADF80630431C053013F8012F56
:100830000DF1080C0CEB420232F8082C834221F82F
:10084000022FF3D102B0704708448078704738B562
:100850004FF07F337F22C0F8A03000254FF6FF73A2
:100860000446A0F8A43080F8A62080F8A950A0F88B
:10087000AA30AC3000F0B2FC84F8B85038BD70B586
:10088000154604461E46114600F04FFC294604F169
:10089000140000F04AFC294604F1280000F045FC51
:1008A000294604F13C0000F040FC294604F15000C8
:1008B00000F03BFC294604F1640000F036FC2946B8
:1008C00004F1780000F031FC294604F18C0000F0BE
:1008D0002CFC04F1AC0032464FF4FA734FF4FA6189
:1008E00000F062FC2046BDE87040FFF7B0BF7047E3
:1008F00000F022BC143000F01FBC283000F01CBCFB
:1009000090F8A43013B990F9A000704790F9A100B5
:10091000704790F8A43013B990F9A200704790F98D
:10092000A300704710B5044607F078FC38B104F115
:10093000140000F005FC012838BF0120C0B210BD32
:1009400010B5044607F06AFC38B104F1500000F01D
:10095000F7FB012838BF0120C0B210BD4FF47A71F7
:10096000AC3000F042BC0021AC3000F03EBC08B519
:10097000AC3000F04BFCB0F57A7FA8BF4FF47A7032
:1009800020EAE07008BD10B5044600F0AFFB04F1AA
:10099000140000F0ABFB04F1280000F0A7FB04F109
:1009A0003C0000F0A3FB04F1500000F09FFB04F1B9
:1009B000640000F0A7FB04F17800BDE8104000F0EF
:1009C000A1BB7F2807D0002807DA10F1800F06D0DE
:1009D0004042C0B2704700207047012070477F201E
:1009E000704710B1404240B270477F2070477F2867
:1009F0000FD010F1310F0EDA10F1780F0DDBFE235E
:100A0000783040B2584346232330B0FBF3F0C0B2F5
:100A10007047FF207047FE207047002070477F28F6
:100A200005D031B1002806DA4042C0B27047FF203D
:100A30007047FE207047002070477F2811D010F1CA
:100A4000310F10DA10F1780F10DB40F2A963783023
:100A500040B2584346232330B0FBF3F0AC3080B2B1
:100A600070470020704740F255707047AC207047C7
:100A700063289FBF40F2A9635843642332309DBF6F
:100A8000B0FBF3F0AC3080B240F2557070474FF4D9
:100A9000F063A0F58060584340F2FF7390FBF3F0E1
:100AA00000F5787080B27047FFF7F1BF4FF496639E
:100AB000A0F58060584340F2FF7390FBF3F000F222
:100AC000DC5080B27047A0F58060D0EB001048BFCA
:100AD000033040F38F007047032812DD0C2812DD2D
:100AE0000F2812DD122812DD162812DD192812DD5A
:100AF0001C2812DD1F2812DD2128CCBFFF20062074
:100B0000704700207047012070470220704708207E
:100B10007047032070470720704704207047052066
:100B20007047000005289ABF014B185CFF207047F2
:100B300053B400087F281ABF4042C0B2002070475B
:100B40007F2811D010F1320F10DA884210DD6423B3
:100B5000401A5843C1F1FF2101F57F01CE313130F8
:100B600090FBF1F0C0B27047FF20704764207047DF
:100B700000207047014B4840185C70475CB4000887
:100B800052B110B4054C0A4411F8013B58408A4256
:100B9000205CF9D110BC7047704700BF5CB40008FE
:100BA000002805DB212805DC044B33F810007047D2
:100BB000002070474FF4FA60704700BF86B5000808
:100BC000392808D822280ED9094B2338C0B2C3408F
:100BD00003F0010070475F2807D0613819288CBFE7
:100BE000002001207047002070470120704700BF9F
:100BF00001EC7F00F8B5024600245F27451E461D24
:100C000015F8010FFF2804BF0134E4B2FFF7D8FF45
:100C100000B92F70AE42F3D1062C04D119B10B6884
:100C200013608B88938000239371F8BD2DE9F843FE
:100C3000012500264FF02808DFF82C90471E441DA0
:100C400017F8011F08480AF070FB034610B1A0EB2B
:100C50000903DBB2A3FB05329E19A742A5FB08538B
:100C6000EED13046BDE8F8835CB5000810B5417997
:100C7000A1F13000C3B2092B07D80523B0FBF3F371
:100C800003EB8303C01AC0B210BD044C20460AF027
:100C90004CFB0028F1D0001BC0B2EEE75CB50008A9
:100CA00070B50446FFF75EFA002582B2501EABB263
:100CB000834204EB030103DAE65C0135302EF6D003
:100CC000D21A2046BDE8704001320AF0FDBA000099
:100CD0002DE9F04F0D4699B0164600211A461F46E1
:100CE00080460AF00BFB00212A2201A800910AF09D
:100CF00005FBDFF8CC90DFF8CCA0DFF8CCB005EB3B
:100D00004606AE4211D16846FFF72CFA30B100F129
:100D100060030DEB0300002300F8613C6946404688
:100D20000AF046FB19B0BDE8F08F47F6FF7335F9BE
:100D3000020B9842E7D0002812DC59460CA80AF0B2
:100D400037FB6846FFF70EFA04460CA8FFF70AFACD
:100D50000444A742D5D368460CA90AF0D7FAD0E7D5
:100D6000B0F57A7F0BDA0CA980B20AF01DF80CA856
:100D7000FFF796FF51460CA80AF0C8FAE1E7642392
:100D80003230B0FBF3F00CA980B20AF00DF80CA8D9
:100D9000FFF786FF0CA8FFF7E5F900F15F036B444E
:100DA00013F8302C00F160010DEB010000F8302C3D
:100DB0002E2203F8302C0023494600F82F3CDAE7B6
:100DC00010B400080BB4000806B40008F0B589B0F0
:100DD0006D4600242F468E1CE1B28A4204D8394663
:100DE000FFF776FF09B0F0BD36F82410013425F87E
:100DF000021BF1E742F21073B0FBF3F2642103FB34
:100E00001200B0FBF1F301FB130000EB023000EB2A
:100E1000831080B2704770B50E4600210546144617
:100E20000AF06CFA00239AB2944200D870BDF25CCA
:100E3000002AFBD0EA540133F5E70000052911D858
:100E4000DFE801F00306080A0C0E0749FFF7E3BFCD
:100E50000649FBE70649F9E70649F7E70649F5E7DA
:100E60000649F3E70649F1E714B4000819B400088D
:100E70001EB4000823B4000828B400082DB40008EC
:100E800032B40008052911D8DFE801F00306080A8A
:100E90000C0E0749FFF7BFBF0649FBE70649F9E714
:100EA0000649F7E70649F5E70649F3E70649F1E79A
:100EB00034B4000839B400083EB4000843B4000854
:100EC00048B400084CB4000832B4000870B50E46AF
:100ED00014460021013205460AF010FA00239AB2A6
:100EE000944200D870BDF25C002AFBD0EA54013372
:100EF000F5E77D23438043F23903C360002309B241
:100F000001808180C3800372704700000268044939
:100F1000044B01FB023323F000430360180C7047BD
:100F2000FD430300C39E2600F0B5002597B0016085
:100F3000858004465622294668460AF0DFF90126D4
:100F4000E27DAA4209D80023802104F1B800A375EC
:100F500017B0BDE8F0400AF0D1B92046FFF7D6FF40
:100F6000E77900217B1B90FBF3F2EC4602FB1300B8
:100F70000A46C0B2CBB29F4222D8002300221146BB
:100F8000277BD0B2874226D80029D9D1A27961190E
:100F9000033A012A05D925B191F9172012BB012B7B
:100FA000CED90B76A26852F82310583305F10E0201
:100FB0006B44013544F8221003F8586CEDB2BFE7DA
:100FC0001CF801EBBEF1000F03D18242D6D00132F2
:100FD000D2B20131CEE72069805C0132984208BF6D
:100FE0000121CEE7501E8342DBDB01329342D8DC85
:100FF000A6E72DE9F047154696B0013D0160027164
:1010000004464371EDB25622002168460AF076F993
:10101000022D98BF4FF003094FF0000794F80780A6
:101020008ABF4FF00109B8FBF9F800253E464FF0A2
:10103000010AE27DB24209D80023802104F1B80000
:10104000A37516B0BDE8F0470AF058B92046FFF77F
:101050005DFFA8EB060390FBF3F2002102FB1300F7
:10106000EC460A46C0B2CBB2434506D21CF801EBAF
:10107000BEF1000F29D1824225D10020434528BF6F
:101080004346844609FB035194F80CE0C9B2C2B24E
:1010900096451CD8BCF1000FCBD116B1FFB9012B7E
:1010A000C7D9A2191176A2681F4652F8211006F17D
:1010B0000E0244F8221003F158026A44013602F885
:1010C00058ACF6B2B5E70132D2B20131CBE72269B2
:1010D000125C01308A4208BF4FF0010CD7E77A1E3C
:1010E0009342DEDB7A1C9342DBDCA2E76421D0E989
:1010F0000123D31AC3604B43418A8260B3FBF1F3EF
:1011000003747047D0E90123D31AC0E90223704762
:1011100043682BB16421C2684A43B2FBF3F2D3B2F5
:1011200003740023C3604360704700234182C0E919
:101130000233436003747047436801334360704770
:10114000007C704743680B44436070470023C0E94C
:101150000133C36003747047F0B5047C0360012C55
:1011600011D94FF47A7744688568141B7C43C668AC
:101170004D1B05FB16442B4494FBF3F33344C3602F
:10118000C0E90121F0BD1CB90123C4600374F7E775
:101190004FF47A744368D31A634384680C1B93FB3F
:1011A000F4F3C3600223F1E72DE9F0410446104651
:1011B0001D4616468846FFF793F8074606EB0800DB
:1011C000FFF78EF801463846FFF796F96560206014
:1011D0002846FFF789F8A060BDE8F08110B5044605
:1011E0004068FFF781F8A06010BD38B504468568F7
:1011F0000846FFF779F82946FEF7C0FF2168FFF798
:10120000C7F82946FEF7BCFFA06038BD08B54FF00F
:101210007C518068FEF7B4FFFFF780FA08BD704785
:1012200070477047002070477047002070470020CB
:10123000704770470020704700207047054B82B010
:10124000DA690243DA61DB6903400193019B02B072
:10125000704700BF00100240054B82B09A690243FC
:101260009A619B6903400193019B02B0704700BFE4
:101270000010024000F10C0353E8003F23F080030C
:1012800000F10C0141E80032002AF3D17047000060
:101290000B4B0C4A1B6830B4A2FB03239B0C00FBD6
:1012A00003F2094D02F5FA72A5FB025207499209B1
:1012B0004C684B681B1B9342FBD330BC704700BF8C
:1012C0001C00002083DE1B43D34D6210001000E0A1
:1012D000044B1888044B80B21B889BB2C01A18BFFD
:1012E0000120704798280020962800200288044B8F
:1012F0005140C9B233F8113083EA1223038070479A
:10130000BCCD00089AB110B4B0F800C0084C0A4433
:1013100011F8013B83EA0C03DBB234F8133091423D
:1013200083EA1C2CA0F800C0F2D110BC70477047B3
:10133000BCCD00084FF6FF7337B50446ADF8063054
:101340004518AC4203D1BDF8060003B030BD14F817
:10135000011B0DF10600FFF7C9FFF2E708B51E20DB
:10136000FFF796FF4FF48052034B28205A61BDE8E7
:101370000840FFF78DBF00BF000C014008B5642096
:10138000FFF786FF4FF48052024B1A61BDE8084018
:10139000FFF77EBF000C014008B5FFF799FF00384A
:1013A00018BF012008BD01207047002070470020B1
:1013B000704700000278024B51405B5C037070473D
:1013C0003CBA0008FF230370704700BF704770B538
:1013D0000B78054603704B780C4643700B78FD2B59
:1013E00038D10A268B788370CB78C3700B79037160
:1013F0004B7943718B7983718B68C3718B68C3F3AD
:101400000F2303728B7A4372627804F10C01A819DE
:1014100009F0D6FF6378B4F80C213344EA54B4F8E9
:101420000C115A1C92B2090AA954A278981CD2072E
:1014300080B20ED504F58872054404F58E7452F816
:10144000041BA24245F8041BF9D112780F332A700D
:1014500098B270BD00238B700B79062683704B7990
:10146000C3708B7903718B684371CDE7242208B573
:101470000021034809F042FF0022024B1A7008BD08
:1014800050050020F80200202DE9F04113780446B1
:10149000037092F80180FD2B0F46154680F80180FD
:1014A00054D10A2693788370D378C370137903716B
:1014B00053794371937983716B7A127A1B0403EB2E
:1014C0000223EA79134423F07F43A268A91963F346
:1014D0001702A26004F10C00424609F071FF7A7B0A
:1014E000904507D208F10C000021A2EB080220442D
:1014F00009F004FF63781E44AB195A78AB5D03EB27
:101500000223A4F80C31A378DB070ED50236B6B25D
:10151000354404F5887305F10C0255F8041B954217
:1015200043F8041BF9D12A781A70BB7A84F8213168
:10153000FB7A84F822313B7B84F823317B7B84F86F
:1015400024313B7884F82031BDE8F08100234380CA
:10155000937806260371D378437113798371537995
:10156000B3E7000070B50D4C0D4E0546062204F1A0
:101570000A0106F58970FFF7A9FC237CC3F3031366
:1015800086F81A31637CC3F3030386F81B31637A50
:10159000DB0744BF02232B7370BD00BF811E0020F8
:1015A000A400002070B504462420E270207022467A
:1015B0005820BDF8145023711B0A63712B0AA170C7
:1015C0006070A57102F8073F049B59198B420CD13A
:1015D0006A1D92B2E11C0020FFF7D2FA05F108065D
:1015E000A05505F1090080B270BD13F8010B02F897
:1015F000010FEBE710B502780A4BD243D2B2447820
:101600009A5C90F802E062409A5C90F803C082EA2B
:101610000E029A5C017982EA0C029A5C4A40985C5C
:1016200010BD00BF3CBA0008F8B53C290446BDF81F
:101630001C5036D0A1F12106714271414900D007FA
:1016400048BF41F0080192074FF0240222704FF08A
:101650006F02E3704FEA132348BF41F0100123717A
:10166000A61C2B0A6270A170A37130466571FFF74A
:10167000C1FF2246069B02F8070F59198B4212D16F
:10168000A91D304689B2FFF755FE05F1080705F19F
:101690000903E0559BB2000AE05405F10A0080B24C
:1016A000F8BD0121CBE713F8010B02F8010FE5E7C4
:1016B0006FF02002084B1A605B68084A02F60C03C0
:1016C00053E8003F43F0200302F60C0040E80031ED
:1016D0000029F3D1704700BF0038014000300140BD
:1016E00050294FEA10122CD018D830292CD00DD800
:1016F00010292CD041F6786343F6F040202908BF2A
:10170000034617489040B0FBF3F0704741F678630A
:1017100047F61220402908BF0346F2E7802919D076
:1017200008D8602918D041F678630E48702908BFA0
:101730000346E6E741F678630B48902908BF034665
:10174000DFE74AF2E423DCE745F24013D9E742F64B
:10175000A003D6E7054BD4E74FF22443D1E700BFFF
:1017600040420F0048E8010020A1070090D003008C
:101770002DE9F04F0C4651880546B1F58C7F85B0B8
:1017800011D300211170D91CC9B2012995BF0121C3
:101790000023518053809CBF2370117000232B7055
:1017A00005B0BDE8F08F10780E2800F28B8001A6FE
:1017B00056F820F087170008F117000819180008DC
:1017C00033180008C5180008C5180008C518000817
:1017D000C5180008C5180008C5180008C518000875
:1017E000C5180008C5180008C518000845180008E5
:1017F000481C5080635421789BB2FD2906D10C33DC
:101800000A21D380022391801370C7E70621083391
:10181000D38091800E23F7E7481C5080D80763548B
:1018200042BFD1880D31D180012B8CBF002303230F
:10183000EAE7002B01F101005080635414BF00233C
:101840000E23E1E7481C508063545388D1888B42B3
:1018500032D3002353801370022369802B702378C6
:10186000FD2B35D163792B72A3796B72637A227A5F
:101870001B0403EB0223E27913446B60637803F1EA
:101880000C026A80A278D10701D519336B8000263B
:101890004FF4BC720C206968DFF8E8806E81B318E1
:1018A00001335B0800FB03F758F80770B94218D200
:1018B0005A1EB242F3D816E092889A423FF66EAFB3
:1018C00001236CE70023137053809380D38066E775
:1018D000E3782B7223796B7263796B6063780833DA
:1018E000D4E71E46E5D80C27774358F807309942CD
:1018F00027D123782046FD2B0CBF4FF00A094FF06B
:10190000060910F801BF474409EB0B03591E89B2C1
:101910000193FFF70FFD97F804A0ADF80E005146B4
:101920000DF10E00FFF7E2FC019BE2185278E35C38
:1019300003EB0223BDF80E209BB29A4203D005238D
:101940002DE703232BE7BB79DA0706D5FA79934510
:1019500082BF04EB09018A5CAA729B0709D50C239C
:1019600003FB068362781B7A9A4282BF4C44E35C95
:10197000EB720C2303FB06835B7985F80CA06B7379
:101980000EE700BF3CBB0008F0B5FD23054604464A
:1019900085B005F80C3B8DF8043090F8243103F144
:1019A0000C020244012B42D80026637066808DF839
:1019B00005308B7A0DF1050023718DF808308B7A94
:1019C000ADF8066001338B72637909218DF8093017
:1019D000A3798DF80A30A368C3F317031A128DF8A0
:1019E0000B301B148DF80D308DF80C20FFF7A2FC86
:1019F000677829463A46ADF802000DF10200FFF77C
:101A000081FC94F82311FFF771FC94F82421BDF8B0
:101A100002309742A4F80C3110D2314607F10C0085
:101A2000D21B204405B0BDE8F04009F067BC12F8B5
:101A3000010D0028B8D1013BDBB2B3E705B0F0BD22
:101A40000023044A1380044A1380044A1380044A82
:101A50001380704796280020982800209A2C002098
:101A60009C2C002007B503688DF8071001221B6924
:101A70000DF10701984703B05DF804FB70B504460B
:101A800008460D46FEF76EFB2368294682B21B69A5
:101A90002046BDE8704018470120FFF7DDBB00007D
:101AA0000D4B984202D10420FFF7D6BB0B4B984256
:101AB00005D003F58063984203D11020F4E7082095
:101AC000F2E7074B984201D12020EDE7054B984201
:101AD00000D070474020E7E700080140000C0140BB
:101AE00000140140001801400B4B984203D14FF401
:101AF0000060FFF7B1BBB0F1804F04D0074B9842B4
:101B000004D1022000E00120FFF798BB044B98426B
:101B100001D10420F8E77047002C01400004004088
:101B2000000800402DE9F0410C46154686B00746F6
:101B30001022002102A81E469DF8348009F0DEFB29
:101B400001940B2D07D8DFE805F00E0E070A1414D8
:101B5000141616161B1DFEE70823029303E0082344
:101B6000029301230593032E0ED8DFE806F01E2012
:101B70000E1E0123F1E70123029304230493F2E7ED
:101B80000923EAE70923F7E7FEE701230393B8F106
:101B9000000F02D03846FFF783FF053D042D0BD818
:101BA000DFE805F007110A0711000323EEE702231F
:101BB000ECE7C4F30F247C61384601A908F000FE6D
:101BC00006B0BDE8F081C4F30F243C61F4E713B51F
:101BD0004FF0010C0024CDE9004CFFF7A3FF02B049
:101BE00010BD000030B50023154687B00446ADF89F
:101BF0000630FFF779FF042D04D8DFE805F02A2E20
:101C000004323B00FEE71C4B1C4A1B68B3FBF2F39B
:101C10009BB20022013BCDE90221204601A9ADF88B
:101C200004300492059208F00BFF236823F0800330
:101C30002360A36823F4804323F00703A360636851
:101C400023F070036360A36823F08003A36007B0F0
:101C500030BD094B0A4A1B68D8E7074B094A1B6885
:101C6000D4E7054B064A1B68B3FBF2F303EB83038F
:101C70005B00CDE70123CCE71C00002080A8120107
:101C800040420F0000127A0010B50446FFF7AAFF89
:101C9000236843F00103236010BD00224FF0FF31A1
:101CA000FFF7F2BF1A4B10B55B681A4C236007F0C0
:101CB0002DFE194808F034FD184808F031FD184889
:101CC00008F02EFD174808F0BBFF174808F0B8FFD2
:101CD00008F0FAFD4FF0E022002313615361936195
:101CE00072B64FF0FF319A0002F16042013302F503
:101CF0006142082BC2F88010C2F88011F3D162B69D
:101D0000034B1B6883F3088823689847FEE700BFEE
:101D100000F0FF1FF402002000080140000C014009
:101D20000010014000380140004400400749084AC3
:101D3000881AEFF30883521A1A44013A013B984279
:101D400088BF0022AA2109F0D9BA00BF00500020A4
:101D50000004000010B50E4C032306220D490E4866
:101D6000FFF735FF2046032302220C49FFF72FFF20
:101D70000323052240F608010948FFF728FF204603
:101D8000BDE810400323052244F24001FFF71FBFC6
:101D90000008014040004004001001408000800421
:101DA000000C01400822034B5A614022A3F58063D6
:101DB0001A617047000C01404022034B5A6108220F
:101DC000C3F81024704700BF00080140104A4FF4C8
:101DD0007041536923F4704391FAA1F153610D4BA3
:101DE0005A6822F400425A601A6822F400421A60CB
:101DF000DA6822F40042DA609A6842F400429A609B
:101E0000D022054B83F828234FF480725A60704724
:101E1000000001400004014000E100E04FF40042F6
:101E2000034B5A611A6842F400421A60704700BFBF
:101E30000004014010B5054C0023062242F22001A7
:101E40002046FFF7C4FE2023236110BD0008014097
:101E50000023032201490248FFF7B9BE0100010433
:101E600000080140024B9868C043C0F3002070474F
:101E70000008014010B50A4C0023052220460949FC
:101E8000FFF7A5FE0023052220460749FFF79FFE26
:101E90004FF4805363614FF40063636110BD00BF72
:101EA0000008014010001004080008040549CB6830
:101EB0001A04DB4302F0805203F4805313430B6196
:101EC000704700BF000801400549CB681A04DB4396
:101ED00002F0006203F4006313430B61704700BF1C
:101EE0000008014010B5054C002305222046044996
:101EF000FFF76DFE4FF40073636110BD000C0140ED
:101F0000020002044FF40072024B1628CCBF1A6183
:101F10005A617047000C014073B504461C2C0E46F4
:101F2000184628DC192C2ADC162C2CDC122C2EDC72
:101F30000F2C30DC0C2C32DC062CB5BF03250A2517
:101F400064244FF4347440F6E443C4EB0424B4FB3B
:101F5000F3F41570C4F30B138DF8043003682401F7
:101F60008DF805400C215C6801AA0223A0470023DC
:101F7000337002B070BD1E2540F6CA04E3E71B258E
:101F800040F2C264DFE7182540F2C354DBE71425B2
:101F900040F2AB44D7E711254FF47A74D3E70E250E
:101FA00040F26B34CFE70000084611461A46014B59
:101FB000FFF7B2BF300300200C4BD3F8FC2022F017
:101FC0008072C3F8FC20D3F8FC2042F08072C3F882
:101FD000FC20A3F55D431A6822F001021A601A681A
:101FE00042F001021A6000225A60704700ED00E0E2
:101FF000064B074A1B680749B3FBF2F3434310B58E
:102000004C684A68121B9A42FBD310BD1C0000208A
:1020100040420F00001000E02DE9F84381464CF2E9
:1020200050300E4617461D4607F056FD88BBB9F1E5
:10203000010F06D0B9F1020F0CBF4FF002094FF0AB
:1020400004094FF00008144A136943F001031361B7
:102050004FEA0814C4F12002A4F1200305FA02F2A9
:1020600027FA04F4144325FA03F31C43A4B24CF2F8
:10207000503026F8184007F02FFD28B908F1010864
:102080005FFA88F39945E3D8034A136923F0010303
:102090001361BDE8F88300BF002002407FB5012333
:1020A0000022CDE9040301A902A8CDE9022307F02B
:1020B0004FFD00280CBF0420052007B05DF804FB8D
:1020C0000A4608B5014600230220FFF7A5FF0028B5
:1020D0000CBF0420052008BD08B5FFF7DFFF031F74
:1020E0005842584108BD08B5FFF7EAFF031F5842A0
:1020F000584108BD2DE9F047264B274D01280FBF59
:102100007D267C26AA461D460F4614462349244AAE
:1021100006BF89469A46914607F0C2FC31462846DA
:10212000FFF7DAFF28B9002407F0CCFC2046BDE811
:10213000F087002F08BF4FF478744FF00008033485
:10214000C4F38F0405F11006AAEB050A1FFA88F301
:102150009C4209D84FF011312846FFF7C4FF041EF6
:1021600018BF0124A400DFE73FB95AF806104B1C42
:1021700006D108F101080436E8E757F82810F6E719
:102180004E4505D23046FFF7AEFF0028F1D1CAE731
:102190000324C9E700F0010800F40108FFF7010873
:1021A000FFF3010810B507F07BFC7C210848FFF71E
:1021B00093FF044638B17D210648FFF78DFF041ECA
:1021C00018BF0124A40007F07DFC204610BD00BF0D
:1021D00000F0010800F4010830B5002340F2EF34AC
:1021E000064D9AB2914201D8042030BDA34203D0DB
:1021F0005A5DC2540133F4E70320F6E710F00108FA
:1022000038B504460D4672B60A4601460020FFF76F
:1022100071FF62B6042806D172B601202A46214613
:10222000FFF768FF62B638BD38B5124B1C68D3F8AB
:102230000054B4F1113F09D1B5F1113F17D000227C
:1022400001201146BDE83840FFF754BFB5F1113FFA
:1022500003D1002211461046F4E7FFF7A3FF04283C
:1022600004D12C4001340CBF0220012038BD0420D1
:10227000FCE700BF00F00108034B18739A68D2070F
:10228000FCD5187B704700BF0038004038B5441EAD
:102290008D18A94200D138BD14F8010FFFF7ECFFEB
:1022A00001F8010BF5E7084611461A46FFF7EEBFA5
:1022B00038B50446054D0144A14200D138BD287807
:1022C000FFF7DAFF04F8010BF6E700BF1400002067
:1022D00008461146FFF7ECBF10B5044601448C4296
:1022E00000D110BD14F8010BFFF7C6FFF7E7084651
:1022F0001146FFF7F1BF000070B58CB0294C2822C1
:10230000002102A808F0FAFFFFF7C6FB4FF4804057
:10231000FEF794FF2449204603230622FFF757FCCB
:10232000062501264FF48053204623610A22032309
:102330001E49CDE90056FFF7F5FB204603230A228C
:102340001B49CDE90056FFF7EDFB032320461A4653
:102350001849CDE90056FFF7E5FB08220023089253
:102360004FF48272CDE90533CDE90933029303922C
:1023700004934FF400720723A4F55444204602A9A5
:102380000B93079208F02FFB236843F04003236070
:10239000A3689B07FCD5FF22237B074B1A700CB068
:1023A00070BD00BF000C014010001004200020048C
:1023B0008000800440004004140000201C4B10B436
:1023C0001A68940611D5D96888060ED5194C1A4892
:1023D0005968238800880133C3F30A0380B2984206
:1023E0001FBF1648C9B2C1542380110744BF104B08
:1023F0005B68120616D50E48C3681B0612D5104B33
:10240000104A1988138889B29BB299420CD013885C
:102410000133C3F30903138013880B4A9BB2D35CC7
:10242000DBB2436010BC704710BCFEF723BF00BF97
:10243000003801409828002096280020962000208F
:102440009C2C00209A2C00209A2800200E490F4A2C
:102450000B8812880133C3F3090392B29A4211D058
:102460000B4AD0540B4A0B8002F60C0353E8003F92
:1024700043F0800302F60C0040E800310029F3D15C
:1024800001207047002070479C2C00209A2C0020CF
:102490009A2800200030014038B504464518AC4267
:1024A00000D138BD14F8010BFFF7D0FFF7E708465D
:1024B0001146FFF7F1BF0000054B064A1B88128842
:1024C0009B1A98B21B0444BF00F5006080B27047AD
:1024D0009828002096280020FFF7EEBF0848094AF8
:1024E0000188138889B29BB29942F9D013880133CD
:1024F000C3F30A0313801388034A9BB2D05C70476E
:10250000982800209628002096200020FFF7E6BF9C
:10251000002300B589B0CDE90633CB1A18BF0123DB
:102520001B03CDE902320C2301900491034801A959
:10253000059308F0B7FB09B05DF804FB00380140D3
:1025400010B5064CE36823F40053E360FFF7E0FFA7
:10255000E36843F40053E36010BD00BF003801405E
:10256000002208461146FFF7EBBF000073B53A4C56
:102570000825E368012623F40053E360FFF78CFA93
:102580004FF48040FEF768FE00F1804003230A22EA
:10259000CDE90056314900F54840FFF7C3FA03235F
:1025A000CDE900561A462E492E48FFF7BBFA002205
:1025B0004FF461401146FFF7ABFFB022236923F4CB
:1025C00090432361636923F02A036361264B83F8F8
:1025D000252320225A602046FEF74CFE234A02F6AD
:1025E0000C0353E8003F23F0400302F60C0040E8E0
:1025F00000310029F3D16FF0400323601C4B198098
:102600001C4B198002F60C0353E8003F23F0200313
:1026100002F60C0040E800310029F3D16FF02002EF
:102620000D4B1A60144A1180144A11801A6922F461
:1026300000621A615A6922F008025A611A6922F48A
:1026400080421A615A6922F022025A61DA6842F421
:102650000052DA6002B070BD00380140020002048E
:10266000040004040008014000E100E000300140E3
:102670009A2C00209C2C00209628002098280020CE
:1026800008B5FFF773FFBDE80840FFF711B8FFF783
:10269000F7BF00007FB500250126044644F2400143
:1026A000FFF7FAF902230B220F48CDE90056FFF796
:1026B00039FA02230B2248F28001CDE900560A487C
:1026C000FFF730FA2268094B9A420AD103F5DE334C
:1026D000DA6942F40012DA61DB6903F40013039350
:1026E000039B04B070BD00BF000C014000540040CB
:1026F0000848094B4FF4804203600023C0E90332CD
:10270000064AC0E90533C0E90733C0E9012307F0F1
:1027100063BB00BF7805002000540040801A06000B
:1027200013B50B46054902460C784FF0FF310448BB
:102730000091610007F0F8FB02B010BDCC0500204D
:1027400078050020007920B50D46194638B1044BB4
:1027500010461D70FFF7E4FFB0FA80F0400920BD7D
:10276000CC050020044B0A22197804484FF0FF33AF
:10277000490007F0B1BC00BFCC050020780500205F
:1027800008B5FFF7B5FF0022014B1A7008BD00BF66
:10279000CC05002010B50446FFF7F2FF0C22044BD5
:1027A0001A70FFF7DFFFB0FA80F35B09237110BDE9
:1027B000CC050020024B1A68024B1A60704700BF1C
:1027C000A02C00203C030020054A064B1968136822
:1027D00099421DBF0133012013600020704700BFE4
:1027E0003C030020A02C0020034A044B11681B78F6
:1027F0000B441360704700BFA02C00202000002075
:102800000148FFF74ABA00BF00040040014B586A74
:1028100080B270470004004008B5FFF7F1FFBDE843
:102820000840FFF7C7BF2DE9F04116460546884628
:10283000002707F035F9B6B2BBB29E4201D8042496
:102840000DE058F827102B688B4202D10435013770
:10285000F2E72846FFF747FC04460028F6D107F0C8
:1028600031F92046BDE8F081037807B56BB1084B1C
:102870001B68B3F5FA6F08D3002302220370694680
:102880004068CDE90033FFF7CEFF03B05DF804FBED
:10289000A02C002000000000012337B52C4A038043
:1028A00004462C4B2C48D3E90051914208BF854285
:1028B0004FF0000202D1227003B030BD22A1D1E955
:1028C0000001C3E90001254825496260D0E90032D2
:1028D0005D1C03D0B3F1AA3F00D023B9551C0CD026
:1028E000B2F1AA3F09D008308842EFD172B67E21FA
:1028F0001A48FFF7F1FB62B6184860600368426847
:10290000591C009304D1551C1BD14FF0AA3311E080
:10291000B3F1AA3F06D1511C0BD0B2F1AA3F10D19E
:10292000002307E06BB9B2F1AA3F0AD14FF48072DD
:1029300022801A46CDE9003269460222FFF773FF72
:10294000BAE700232370F4E712345678FEDCBA901D
:10295000FEDCBA90000000201234567800F801081E
:1029600000FC01080A490B8803B9FEE772B64FF074
:10297000804309885A6A114464325963DA636FF0FC
:1029800002021A616FF008021A6162B6704700BF56
:102990004400002000B5032289B04FF0FF314FF012
:1029A0008040FFF771F920220021684608F0A6FC5C
:1029B00064236A4601214FF08040039308F078F8C1
:1029C000C8236A464FF480714FF08040039308F0AB
:1029D0006FF8A022044B83F81C234FF080521A603A
:1029E00009B05DF804FB00BF00E100E04FF0804358
:1029F000DA6842F00202DA60DA6842F00802DA606D
:102A00007047000010B50022044601EB8101074B1E
:102A100001EB810189001980054B1A70FFF7BAFF9D
:102A20002046BDE81040FFF7E1BF00BF4400002092
:102A3000390300204FF080431A6991070AD56FF0DF
:102A400002021A615A6B6432DA63084A596B1288BF
:102A50000A445A634FF080431A69120705D56FF094
:102A600008021A610122024B1A70704744000020CC
:102A7000390300202DE9F0411B4C90220021201D3C
:102A800008F03CFC2023062663800F23DFF85C80DF
:102A900032464146A380A0192C232680FEF796F9E2
:102AA0004FF480330025124F32464146C4E90D737E
:102AB00004F13E002C23A587FEF788F901230D4978
:102AC00004F17C00A4F87030C4E91D55E76684F871
:102AD000725008F06DFC7F2384F89130052384F850
:102AE0009230BDE8F08100BF60020020F8B9000814
:102AF000020001003AB6000870B5094E05460C46C2
:102B0000415C304608F011FC034628B1831B0133B9
:102B1000DBB2282B28BF0023F35C2B5570BD00BF10
:102B200010BA000870B50C461146064608F040FC85
:102B300044B10025052130460135FFF7DDFFEBB23A
:102B40009C42F7D870BD000073B5054605F111062B
:102B5000214C0146214A68463601FFF7E3FFB01CCD
:102B60006946204408F024FC0223264473720023A3
:102B700004EB0512A2F81A311422042102FB0540CD
:102B800001224FF4807580F8501040F20111A0F836
:102B90004A20C264A0F8522080F85520A0F8565070
:102BA000A0F8581040F2032084F83430E284A56283
:102BB000A08584F82E2084F8303084F83330C4F8AF
:102BC0003A30C4F83E30C4F84230A4F84610A4F8B5
:102BD000481002B070BD00BFA4000020F0B500088E
:102BE000F7B5054605F111060146AE4AAE4C6846FA
:102BF0003701FFF797FFB81C694627442044FDF7CB
:102C0000F9FF7B7AA94A052B88BF022304EB061043
:102C100088BF7B721188437A41FA03F3DF070FD430
:102C20000223437261B14807C1F3800308D441FA1B
:102C300003F7FF07D8B240F1D08104EB06135872B6
:102C400004EB051191F81A012B01052802D9002087
:102C500081F81A01E718508897F81A1140FA01F123
:102C6000C90711D4052187F81A1168B18706C0F386
:102C7000401109D440FA01FC1CF0010FCFB200F062
:102C8000B181E11881F81A71E11891F81B0103284C
:102C900002D9002081F81B0104EB0616717A012984
:102CA00003D9042901D000219180E618908896F874
:102CB0001B1140FA01F111F001010ED186F81B1130
:102CC00058B110F0010108D140FA01F7FF07CEB268
:102CD00040F18D81234483F81B61142303FB0541DC
:102CE00091F84A00052802D9012081F84A0003FB27
:102CF000054393F84B10042902D9002183F84B10A7
:102D0000142303FB0543918E93F84B0041FA00F026
:102D1000C00712D4012083F84B0071B18807C1F3BA
:102D200040030AD441FA03F6F707D8B240F16481B0
:102D3000142303FB054383F84B00142303FB0543D3
:102D400093F84C10032902D9012183F84C10142068
:102D500000FB0540D18E90F84C3041FA03F313F09C
:102D6000010310D180F84C3069B111F001030AD190
:102D700041FA03F6F607D8B240F14381142303FB6E
:102D8000054383F84C00142303FB054393F84E10CE
:102D9000012902D9002183F84E10142000FB0540C0
:102DA000118F90F84E3041FA03F313F0010310D164
:102DB00080F84E3069B111F001030AD141FA03F6EF
:102DC000F707D8B240F12281142303FB054383F8AF
:102DD0004E00142303FB054393F84F10022902D938
:102DE000002183F84F10142000FB0540518F90F80C
:102DF0004F3041FA03F313F0010310D180F84F3044
:102E000069B111F001030AD141FA03F6F607D8B20D
:102E100040F10181142303FB054383F84F00142381
:102E200003FB054191F84D00022802D9002081F8EA
:102E30004D0003FB054393F85010052902D90421E6
:102E400083F85010142303FB054191F85200012828
:102E500002D9012081F8520003FB054393F8551075
:102E6000012902D9012183F85510142303FB0543DE
:102E700093F85310022902D9002183F8531014202B
:102E800000FB0540918F90F8533041FA03F313F0A3
:102E9000010318D180F85330A9B111F0010312D108
:102EA00006E000BFF0B50008A4000020600200208A
:102EB00041FA03F6F707D8B240F1B280142303FBBE
:102EC000054383F85300142303FB054191F8560092
:102ED0000C2802D9002081F8560003FB054393F823
:102EE0004C10012906D193F84F10022904BF00218C
:102EF00083F84F101423012140F2011003FB054316
:102F000083F85710A3F8580094F82630052B01D900
:102F100084F8261094F82730042B02D9002384F873
:102F20002730B2F86C0094F8273040FA03F313F01E
:102F3000010F814B0ED1012184F8271050B1860773
:102F4000C0F3400106D440FA01F7FF07CEB26CD5BA
:102F500083F8276094F82810022902D9002184F808
:102F6000281094F82910022902D9012184F8291087
:102F7000B2F86E1094F8292041FA02F212F0010220
:102F80000CD184F8292049B111F0010206D141FA8F
:102F900002F6F607D0B24CD583F8290094F82A201F
:102FA0000C2A02D9002284F82A2093F832200C2A15
:102FB00002D9002283F8322093F82B20042A02D968
:102FC000002283F82B20002210465C4911F9014FA2
:102FD00014F1780F31DA087031E00133102B7FF4EF
:102FE00026AE2DE6013110297FF444AE4CE60131C6
:102FF00010297FF469AE70E60133102B7FF492AE96
:103000009BE60133102B7FF4B3AEBCE60133102BEB
:103010007FF4D4AEDDE60133102B7FF4F5AEFEE68F
:103020000133102B7FF444AF4DE7013110298AD1D1
:1030300090E70132102AAAD1B0E7782CCBDC01321C
:10304000D2B20C2AC2D1002201203D4911F8014F11
:103050000132022CD2B288BF0870042AF6D193F84C
:103060003420012A02D9002283F83420354AB2F8EC
:10307000701093F8342041FA02F212F001020CD1E0
:1030800083F8342049B111F0010206D141FA02F46B
:10309000E407D0B211D583F8340093F82C20052A28
:1030A00002D9032283F82C2093F82D20032A08D874
:1030B0000AD1002283F8342006E00132102AE5D13B
:1030C000EBE7022283F82D2093F82E20022A02D962
:1030D000012283F82E2093F83020022A02D9002200
:1030E00083F8302093F833200C2A02D9002283F889
:1030F00033201421FF2201FB05314FF6FF7081F8C8
:10310000512081F8542083F82F2083F831204FF08C
:10311000FF3203EB0515C5F81C21A5F820011A6242
:103120009A84A1F85A20A1F85C2083F83500DA8649
:103130001A8703B0F0BD00BFA4000020DD0000200E
:10314000E90000206002002010B5052804D8DFE85F
:1031500000F01E04221A1E22FEE720241F210F2247
:103160000F4B987003380128A3F84A104FF0000164
:1031700094BF0020012019711A771974A3F84840F0
:103180009873987610BD09246F210722E8E714246C
:1031900032210A22E4E7352413211922E0E700BF97
:1031A000480000202DE9F74300F111067A4F36015F
:1031B00006F10209B94405464846FDF737FD0421EA
:1031C0008046764C01900DEB0100FEF7B3F8C4F891
:1031D0000880C4F814804FF001083E44737A2E0131
:1031E00007EB0515E08395F81A01637084F85180A8
:1031F000A4F85280A4F85480FFF7A6FF97F8262081
:10320000674B13F92230237323766378052B09D893
:10321000DFE803F0030656585A5C0023637301E0AD
:1032200084F80D805F4B617B1B88617603F001029F
:10323000980748BF42F00202A2855D0748BFA28DF1
:1032400084F8281044BF42F00402A285180742BF48
:10325000A28D42F01002A285DA0642BFA28D42F092
:103260002002A2859B0642BFA38D43F00803A385DD
:10327000002384F82A3021B94846FDF7F7FC84F88A
:103280002A003E4496F81B2184F829206AB1E18B7C
:1032900002EB021303EB03230B444FF01131E383E2
:1032A000A36801FB0233A3606361E38B94F82850A9
:1032B0006362052D0CD8DFE805F00C4D4F15434532
:1032C0000223ABE70423A9E70523A7E70323A5E728
:1032D000FEE7A378032B03D8DFE803F003424003A3
:1032E000FEE71825304E84F8205016E90F0086E8D6
:1032F0000F0040F2E2432846A4F84C30FCF7F4FFFC
:103300004FF07F51FDF744F8FDF72EFA4FF47A7332
:10331000B4F848206D08B3FBF2F3052D38BF05253E
:10332000A4F8403097F82C30C0B2A4F84E0084F8CE
:103330005050052B24D8DFE803F0152C2023262934
:103340000225CFE7A378022B08D0052B06D0012B4E
:1033500006D0FEE71925C5E70625C3E70C25C1E71A
:103360001225BFE74FF4165363640023A4F85630C8
:1033700084F8583003B0BDE8F0834FF41643F3E708
:103380004FF46143F0E74FF4E133EDE74FF461337D
:10339000EAE74FF49643E7E7A40000204800002046
:1033A000F8B9000860020020780000204FF4DE72B7
:1033B000FF21014807F0A2BFA40000204FF4DE71F6
:1033C0000148FEF71DBF00BFA40000204FF4DE71CE
:1033D0000148FEF701BF00BFA400002008B5FFF7B9
:1033E000F5FF034B1878BDE80840FFF7F9BB00BFB5
:1033F0004800002038B5FFF7D9FFFEF715FF042875
:103400000CD0FFF7D3FFFEF70FFF042803D1FFF71F
:10341000DDFF042806D0FFF7C9FF03E0FFF7D6FF62
:103420000428EED110222649264807F08BFF254CB0
:1034300038B110222046244907F084FF08B1FFF775
:10344000B5FFA38AB3F5215F28D008D30025E8B2E1
:103450000135FFF779FB0A2DF9D10023E3774FF40B
:1034600021530125A38242F64203226914499A425C
:1034700014484FF010021CBF0125236107F062FFC2
:1034800070B110220E490F48FDF7C5FC08220F4904
:103490000F48FDF7C0FCFFF791FF03E00025E2E7CE
:1034A000002DF8D10023E3770A4C2370FFF7E2FAEE
:1034B0002078FFF795FB2078BDE83840FFF772BE13
:1034C000F7B50008A400002008B6000819B60008E7
:1034D000560200204800002037B50C4605468B7880
:1034E0004A78097807F0B9FDE37928460193A37972
:1034F0002279E1780093637907F0DFFD6178207825
:10350000FEF7EEF8A86103B030BDC36837B50446D6
:10351000A3B1024652F8143B5D6900F11503A847B8
:1035200032233F220B21204607F0F1FC09237022B1
:10353000009380212046237D07F01DFE03B030BD9F
:1035400073B5C160044607F013FD80238DF8073082
:1035500001230DF107021946204607F08DFC204695
:1035600007F00CFDE3681C4E1B78204606EB0313A6
:103570005D78294607F01FFD2946204607F02CFDFF
:1035800003222021204607F010FD04230C222621CF
:10359000204607F0BCFCE368204693F90810FFF7CB
:1035A000B4FFE3681D7805B1FEE731462046266189
:1035B000FFF792FF2A462946204607F041FD2046A4
:1035C0002B46C022C82107F0A4FDFF21204602B0EF
:1035D000BDE8704007F0BABDBCCF000810B5044686
:1035E00007F0CCFC2046BDE81040FF2107F0AEBD3F
:1035F00038B504460368C1685D6991F9081000F1A7
:10360000150300F11402A847E3681B7803B1FEE735
:10361000034B902160202361FEF762F8A06138BD62
:10362000BCCF0008C36810B504463BB103690BB9B1
:10363000FFF7DEFF2369B3F90C0010BD1846FCE765
:10364000C36810B5044633B103690BB9FFF7D0FF67
:1036500094F9150010BD1846FCE7000090F8D8302A
:103660005BB190F8D930074A180102EB03139B684D
:103670001978135853F821007047837D0E3350F8A2
:103680002300704798B9000813B5194B0288DB8BEB
:1036900004469A4227D1837813F0D00F25D183793D
:1036A000812B22D84FF6FF730D2201460DF1060043
:1036B000ADF80630FDF726FEB4F80D20BDF8063053
:1036C0009A420ED14C2204F10D01FDF71BFEB4F815
:1036D0005900BDF80630C01A18BF0120800002B0A2
:1036E00010BD0320FBE70120F9E70220F7E700BF48
:1036F000480000200A7ACB7902F0070243EA02234D
:1037000003804B7A0A7A03F03F035B0143EAD2035A
:1037100043808B7A4A7A9B0043EA9213CA7A02F07A
:10372000010243EA822383800B7BCA7A03F00F03F2
:10373000DB0143EA5203C3800B7BC3F30112012A6E
:1037400011D813F0300F14BF012300239B02038311
:103750000B7B7F2B0AD813F0C00F14BF012300236B
:103760009B024383704740F2FF73F0E740F2FF7320
:10377000F7E70A7ACB7902F0070243EA02230380D3
:103780004B7A0A7A03F03F035B0143EAD20343809A
:103790008B7A4A7A9B0043EA9213CA7A02F00102BA
:1037A00043EA822383800B7BCA7A03F00F03DB0199
:1037B00043EA5203C3800A7CCB7B02F0070243EA50
:1037C000022303814B7C0A7C03F03F035B0143EA45
:1037D000D20343818B7C4A7C9B0043EA9213CA7CD0
:1037E00002F0010243EA822383810B7DCA7C03F04D
:1037F0000F03DB0143EA5203C3814B7DDB000382ED
:103800008B7DDB004382CB7DDB0083820B7EDB0084
:10381000C3820B7BC3F30112012A2BD813F0300FA4
:1038200014BF012300239B0203830B7B7F2B24D82F
:1038300013F0C00F14BF012300239B0243830B7DB1
:10384000C3F30112012A1BD813F0300F14BF012358
:1038500000239B0283830B7D7F2B14D813F0C00FB2
:1038600014BF012300239B02C3834FF480630384AE
:103870004384704740F2FF73D6E740F2FF73DDE701
:1038800040F2FF73E6E740F2FF73EDE737B5214BF7
:103890000446DB8B0D4603804A78837862F3C303CA
:1038A00083704A79C37862F30003C3708A794379DD
:1038B00062F38613437191F90200FDF782F8E37811
:1038C000214660F34703E370EA7823790DF106009F
:1038D00062F3060323712A79DBB202F0010203F0DE
:1038E0007F0343EAC21323712A796379C2F3450245
:1038F00023F03F03134363714FF6FF735922ADF872
:103900000630FDF7FFFCBDF80630A4F8593003B0CF
:1039100030BD00BF480000202DE9F34104461546A4
:1039200088469DF820605B22522E4FF000011F4612
:1039300028BF522607F0E2FC2D4BDB8B23802A7830
:10394000A37862F30203A3706978DBB2C90001F0C7
:10395000080103F0070341EA08111943A1706A79CD
:10396000E37862F30003E370AA79637962F3861364
:10397000637195F90200FDF724F8E37860F34703DB
:10398000E370EA78237962F3060323712A79DBB2C4
:1039900002F0010203F07F0343EAC21323712A7984
:1039A0006379C2F3450223F03F0313432246637158
:1039B000A37966F3470302F8063F3B463E44B34211
:1039C00010D14FF6FF73592221460DF10600ADF8D4
:1039D0000630FDF797FCBDF80630A4F8593002B068
:1039E000BDE8F08113F8011B02F8011FE7E700BFF3
:1039F0004800002007B5009313460A460121FFF74F
:103A00008BFF03B05DF804FB30B5374B027893F8B9
:103A1000261000F1160461F30302027093F82710D8
:103A200061F30712027093F82810427861F30302E1
:103A3000427093F8291061F30712427093F82A102C
:103A4000827861F30302827093F83210827961F315
:103A50000302827193F82B10827861F3071282704F
:103A600093F83410C27961F30302C27193F82C10F9
:103A7000C27861F30302C27093F82D1061F307124C
:103A8000C27093F82E10027961F303020271427939
:103A900093F8301061F30302427193F83310827986
:103AA00061F30712827103F1390100F10A0211F981
:103AB000015F02F8015FA242F9D193F84610C27D7E
:103AC00061F30102C27593F8471061F38302C27576
:103AD00093F8481061F30512C27593F8493063F307
:103AE0008712C27530BD00BFA40000200278314BA0
:103AF000C2F3030230B583F82620027803F13901BE
:103B0000C2F3031283F82720427800F11604C2F3AF
:103B1000030283F828204278C2F3031283F8292095
:103B20008278C2F3030283F82A208279C2F3030267
:103B300083F832208278C2F3031283F82B20C279F3
:103B4000C2F3030283F83420C278C2F3030283F87D
:103B50002C20C278C2F3031283F82D200279C2F31D
:103B6000030283F82E204279C2F3030283F8302047
:103B70008279C2F3031283F8332000F10A0212F9AA
:103B8000015FA24201F8015FF9D1C27DC2F30102D7
:103B900083F84620C27DC2F3810283F84720C27DAC
:103BA000C2F3011283F84820C27DC2F3811283F868
:103BB000492030BDA400002070B5522698B032468E
:103BC00004460D4603A8002107F098FB212342F686
:103BD00042008DF80C30FDF70DF9ADF80E004FF4F2
:103BE0002150FDF707F914221A49ADF810000DF124
:103BF0001200FDF710F91848FFF722FD174B8DF85A
:103C0000260093F851300AA88DF82730FFF7FCFE04
:103C1000134A144B0221CDE91223134B204614936F
:103C200047F6FF73ADF85430104BADF84610B3F8BB
:103C30006C208DF85620B3F86E20B3F870308DF8F4
:103C400057208DF858302A46009603ABFFF764FEE4
:103C500018B070BD1FB60008481E002048000020A4
:103C60000A006400FA00F401E803FF7F600200200C
:103C700038B504460F4D00F11B01062205F5897089
:103C8000FDF724F994F8213004F12500C3F3030370
:103C900085F8193194F82130C3F3031385F81A31EC
:103CA00094F82230C3F3030385F81B31BDE8384094
:103CB000FFF71CBFA400002000230A4A838012687B
:103CC00083718260084A83810384136803615368A7
:103CD000064A4361136883615368C3614EF66023EB
:103CE00003607047A02C002029B6000832B60008F7
:103CF00010B50D4C0220FFF727FA2046FFF76EFCA7
:103D000003212046FFF701FCE36803B9FEE71B78B7
:103D100003B1FEE7054920462161FFF7DDFB2046A0
:103D2000FFF75CFC10BD00BF481E0020BCCF0008A0
:103D300008B590F8203002468BB9FEF793F810B919
:103D400082F8210008BD92F8213001335BB2312B9B
:103D500082F82130F6DD012382F82030F2E7FEF709
:103D600081F818B1322382F82130EBE792F8213044
:103D7000013B5BB2002B82F82130D8BF82F82000D3
:103D8000E0E700000A4B90F820201B6872B18268BF
:103D90009B1AB3F57A6F01D901234371037923B9D3
:103DA000437913B101230371037370478360F5E70F
:103DB000A02C00200346007B821E012A4FF0000247
:103DC00002D893F8201009B91A737047104670474B
:103DD0000A4A38B51388044601339BB2502B0D466E
:103DE00001D8138038BD002305491380FDF746FE36
:103DF00029462046FDF742FEF4E700BF40030020BD
:103E00003BB600082DE9F74F1646054688466D4932
:103E1000FDF734FE31462846FDF730FE00226A4B9E
:103E2000B8F1010F694C1A8011D14FF480534FF44F
:103E30000067636146F2A8102761FEF7D9F8676151
:103E4000FEF7D6F831462846FFF7C2FFF2E7A8F1A1
:103E500002034FF400620C2B00F2A780DFE803F0AE
:103E60003141531C07A5A5A56363636363004FF449
:103E700000684FF4805746F2A810C4F810806761BC
:103E8000FEF7B6F8C4F814802761FEF7B1F83146A2
:103E90002846FFF79DFFEEE74FF400684FF4805788
:103EA00046F2A810C4F810802761FEF7A1F8C4F804
:103EB00014806761FEF79CF831462846FFF788FFBB
:103EC000EEE74FF48057626146F2A8102761FEF7D3
:103ED0008FF86761FEF78CF831462846FFF778FFC8
:103EE000F2E74FF480534FF40067236146F2A810C5
:103EF0002761FEF77DF86761FEF77AF831462846BC
:103F0000FFF766FFF2E74FF48057226146F2A810F0
:103F10002761FEF76DF86761FEF76AF831462846BB
:103F2000FFF756FFF2E700274FF4805B4FF400697C
:103F3000A8F1090A5FFA8AFA0423574538BFC4F882
:103F400010B0019346F2A810C4F81090FEF750F894
:103F5000C4F81490FEF74CF831462846FFF738FFB6
:103F6000019B013B13F0FF03EBD10423C4F814B011
:103F7000019346F2A810C4F81090FEF739F8C4F87F
:103F80001490FEF735F831462846FFF721FF019BD4
:103F9000013B13F0FF03EBD10137A8F10803FFB297
:103FA000DBB2BB4238BF0027C6E74FF48053226123
:103FB00023614CF25030FEF71BF831462846FFF7DC
:103FC00007FFF6E73BB60008400300200008014069
:103FD00010B5044694F9013008468B4201D123788C
:103FE00023B901232370FDF78DFF607010BD000021
:103FF00037B50C461D4668B907480DF106020DF1AC
:10400000070107F0F1F82B4622469DF806100248FA
:1040100006F09EFF03B030BD481E002038B50C46A8
:104020001546014690B9FDF7BDFE0A482B462246CB
:1040300006F07EFFFF21074807F088F8054807F0E3
:10404000ADF8BDE838407D20FDF7D2BF0148FFF74D
:10405000C5FA38BD481E00202DE9F0415B27054612
:10406000174C0E463A460021204607F047F9AB6947
:1040700004F10E002360EB6912496360124B1B7858
:104080009A1E53425341627A63F3000262724222E3
:10409000A27228220023E272142223736373FCF7B6
:1040A000BAFE59212046FDF745F9084BA4F85900FE
:1040B0003A4621463046BDE8F0411B7FFFF7AEBFD0
:1040C000D31C00201FB600082B030020480000204E
:1040D00013B50C4638B91148C36833B9812281F849
:1040E000A23081F8A02002B010BD01F1A2020DF1B2
:1040F000060107F05FF8BDF90630002B08DB4FF62C
:10410000FF73ADF80630BDF8063084F8A030EAE75A
:104110007F33F8DA4FF68173F3E700BF481E0020C3
:104120000A4608B501460148FFF76CFE0C00002066
:104130000023FF22037043708370C27003717047C5
:10414000C178034629B98278017101328270012059
:104150007047007801281ED0022805D0C8B99A7887
:10416000187101329A70F2E798785A784240D20773
:1041700004D40022013098701A71E8E7FF2902D1B7
:104180000020187170471A790132D2B291421A7127
:10419000EFD300207047FF29F2D01A790132D2B252
:1041A00091421A71F5D29A7801329A7000221A71EE
:1041B0007047000008B5437802789A4213D0052B67
:1041C0008ABF052303700370027888BF4370064BD3
:1041D000064813F92210064B19731976C36813B1F8
:1041E0001972FFF792F908BDF8B90008481E0020BF
:1041F0004800002010B50AB9437010BD541E0B2CA6
:10420000FBD80332D2B231F8122040F27E618A42EA
:1042100003D95AB222EAE2721AE0B2F5C17F02D2A1
:104220009A1E52B2F6E740F2A9518A4204D95AB214
:10423000052A1CDCDA1EF4E740F256218A4218D91E
:1042400040F2D4418A4208D95AB2042AF2DD02224D
:104250009A42C8BF5AB24270CFE7B2F54B7F04D240
:104260005AB2032AE6DD0122F2E75A1ED9E70322F9
:10427000EEE70022ECE700000E4803681A0617D5A7
:10428000C3681B0614D50C4B0C4A1988138889B2D5
:104290009BB299420AD013880133DBB21380138892
:1042A000074A9BB2D35CDBB243607047FCF7E2BFC6
:1042B000704700BF0048004094200020922000205A
:1042C000921F00200E490F4A0B8812880133DBB27F
:1042D00092B29A4212D00C4AD0544FF040220B8036
:1042E00002F60C0353E8003F43F0800302F60C0093
:1042F00040E800310029F3D10120704700207047C9
:104300009420002092200020921F002038B50446FF
:104310004518AC4200D138BD14F8010BFFF7D2FFAD
:10432000F7E708461146FFF7F1BF0000002300B58C
:1043300089B0CDE90633CB1A18BF01231B03CDE9A1
:1043400002320C2301900491034801A9059306F061
:10435000A9FC09B05DF804FB0048004010B5064C0C
:10436000E36823F40053E360FFF7E0FFE36843F4FE
:104370000053E36010BD00BF0048004008B531B1F4
:104380004FF400524FF480610248FFF7E7FF01202D
:1043900008BD00BFA086010013B52B4C2B49E36874
:1043A00023F40053E360FDF777FB4FF48020FCF724
:1043B00045FF082301222648CDE9003203230A22C3
:1043C000FDF7B0FB002223481146FFF7AFFFC022E4
:1043D000236923F490432361636923F02A03636113
:1043E0001D4B83F8272380225A602046FCF742FFAA
:1043F0004FF0402101F60C0353E8003F23F0400347
:1044000001F60C0040E80032002AF3D16FF04003BF
:104410002360124B1A80124B1A80236923F4006325
:104420002361636923F008036361236923F48043F4
:104430002361636923F022036361E36843F400535B
:10444000E36002B010BD00BF004800400400040457
:10445000000C0140A086010000E100E09220002055
:104460009420002030B51C4C85B00E22002105465A
:10447000684606F043FFB4F8A0302046ADF800309F
:10448000FCF750FA8DF802002046FCF742FAB4F827
:10449000A4308DF803001148ADF80430FFF7D0F8D0
:1044A00094F8A6308DF806008DF8073094F8A930FE
:1044B00069468DF80830B4F8AA302846ADF80A30BD
:1044C000074B9B788DF80C3001238DF80D3004F0EC
:1044D0004CFD05B030BD00BF8C1D0020481E0020E3
:1044E000480000200148FEF73DBA00BF891D0020AA
:1044F000F8B50E460746144D5B2329463046144650
:104500002A46FFF775FDD7E9041328686A689A42BE
:1045100008BF884209D0002430460C49FFF7D8FD77
:10452000002C0CBF01200320F8BD59212846FCF7C0
:1045300001FFB5F859308342EDD114B1FFF7D2FF36
:10454000EAE70124E8E700BF811E00208C1D00205F
:1045500013B5012104460844FCF7ECFEA178ADF840
:1045600006000DF10600FCF7C1FEE178FCF7BEFE87
:104570002179FCF7BBFE6179FCF7B8FEA179FCF765
:10458000B5FE04F108010322FCF7BCFE627804F1D9
:104590000C01FCF7B7FE94F82311FCF7A7FEBDF859
:1045A0000630A4F80C3102B010BD0000003818BF6E
:1045B0000120014B18707047F80200202DE9F041EE
:1045C000002A4AD1042B00F2A1809EB2002B42D0D7
:1045D0004FF0800EFF254C4C0F8894F81EC0C35D31
:1045E000013223EA0C03C355A37F1FFA82FC5B0848
:1045F000A3773BB90B8801330B8084F81EE00B884E
:10460000C554A37FB1F8008010F8087027EA0303AF
:1046100000F80830A37F5B08A3773BB90B88013310
:104620000B8084F81EE00B88C554A37FB1F800808E
:1046300010F8087027EA030300F80830A37F5B082E
:10464000A37733B90B8801330B8084F81EE00B8805
:10465000C5546645C0D8BDE8F081FF2AFBD1032BC5
:1046600000F249819EB2002BF5D000258027264C10
:10467000B1F800C094F81EE010F80C30013523EAC0
:104680000E0300F80C30A37F5B08A37733B90B88C7
:1046900001330B80A7770B88C254A37FB1F8008049
:1046A0001FFA85FC10F808E02EEA030300F8083032
:1046B000A37F5B08A37733B90B8801330B80A777FF
:1046C0000B88C254A37F5B08A37733B90B880133EF
:1046D0000B80A7770B88C254A37FB1F8008010F835
:1046E00008E02EEA030300F80830A37F5B08A377F5
:1046F0002BB90B8801330B80A7770B88C254664512
:10470000B6D8BDE8F08100BF500500200D889A4C56
:10471000425DA67F03F5C06322EA06024255A27FEE
:104720005208A2773AB90A88FF2501320A8080220E
:10473000A2770A8885540D88A67F425D22EA060288
:104740004255A27F5208A2773AB90A88FF25013262
:104750000A808022A2770A888554A27F5208A27715
:104760003AB90A88FF2501320A808022A2770A8896
:104770008554A27F5208A2773AB90A88FF250132F0
:104780000A808022A2770A8885540D88A67F425D20
:1047900022EA06024255A27F5208A2773AB90A8855
:1047A000FF2501320A808022A2770A8885541E06DE
:1047B00005D40D88A67F425D22EA06024255A27FFB
:1047C0005208A2773AB90A88FF2501320A8080226E
:1047D000A2770A8885545D0605D40D88A67F425DC0
:1047E00022EA06024255A27F5208A2773AB90A8805
:1047F000FF2501320A808022A2770A8885549A0612
:1048000005D40D88A67F425D22EA06024255A27FAA
:104810005208A2773AB90A88FF2501320A8080221D
:10482000A2770A888554DF0605D40D88A67F425DED
:1048300022EA06024255A27F5208A2773AB90A88B4
:10484000FF2501320A808022A2770A8885541E073C
:1048500005D40D88A67F425D22EA06024255A27F5A
:104860005208A2773AB90A88FF2501320A808022CD
:10487000A2770A8885545D0705D40D88A67F425D1E
:1048800022EA06024255A27F5208A2773AB90A8864
:10489000FF2501320A808022A2770A8885549A0770
:1048A00005D40D88A67F425D22EA06024255A27F0A
:1048B0005208A2773AB90A88FF2501320A8080227D
:1048C000A2770A888554DB0705D40A88A57F835C14
:1048D00023EA05038354A37F5B08A377002B7FF4AF
:1048E000BAAE8025FF220B8801330B80A5770B8899
:1048F000C254BDE8F0810E881F4C855DA77F03F58B
:10490000E06325EA07058555A57F6D08A57735B9CC
:1049100080260D8801350D80A6770D8842550D88BB
:10492000A67F425D22EA06024255A27F5208A27784
:104930003AB90A88FF2501320A808022A2770A88C4
:104940008554A27F5208A2773AB90A88FF2501321E
:104950000A808022A2770A888554A27F5208A27713
:10496000002A7FF418AF0A88FF2501320A808022CE
:10497000A2770A8885540EE7500500202DE9F047FC
:1049800000278026FF25A64C0F809846A677057045
:10499000002B00F0438103F1FF391FFA89F9BA4671
:1049A0003B469144561E0BE0554540F0CE80013702
:1049B000BFB20A88424580F0C1804E4500F01D819B
:1049C00016F8015F002BEFD16B1EDBB2FD2B00F25E
:1049D000B8803F2B40F2F38005F14103DBB23F2B5F
:1049E00000F2BA80A37F01355B08EDB2A377002BFC
:1049F00000F0F8805B08A37753B94FF0800CFF22DA
:104A00000B8801330B8084F81EC00B88C254A37F2F
:104A1000AA0608D4B1F800C010F80C2022EA03035B
:104A200000F80C30A37F5B08A37753B94FF0800CDC
:104A3000FF220B8801330B8084F81EC00B88C25400
:104A4000A37FEA0608D4B1F800C010F80C2022EACF
:104A5000030300F80C30A37F5B08A37753B94FF032
:104A6000800CFF220B8801330B8084F81EC00B885A
:104A7000C254A37F2A0708D4B1F800C010F80C2054
:104A800022EA030300F80C30A37F5B08A37753B935
:104A90004FF0800CFF220B8801330B8084F81EC07E
:104AA0000B88C254A37F6A0708D4B1F800C010F87D
:104AB0000C2022EA030300F80C30A37F5B08A377E5
:104AC00053B94FF0800CFF220B8801330B8084F820
:104AD0001EC00B88C254A37FAA0708D4B1F800C037
:104AE00010F80C2022EA030300F80C30A37F5B08C7
:104AF000A37753B94FF0800CFF220B8801330B8052
:104B000084F81EC00B88C254A37FEA0705D40D8821
:104B1000425D22EA03034355A37F5B08A377CBB929
:104B20004FF0800CFF250A8801320A8084F81EC0ED
:104B30000A8885540A884245FFF43FAF0020BDE84B
:104B4000F0870127AA463B4633E75246FBB2FFF700
:104B500035FD39E700232CE70A8894F81EC0835CF2
:104B60003F3523EA0C038354A37FEDB25B08A377A0
:104B700053B94FF0800CFF220B8801330B8084F86F
:104B80001EC00B88C254A37F5B08A37753B94FF0B4
:104B9000800CFF220B8801330B8084F81EC00B8829
:104BA000C254A37F6A063FF525AFB1F800C010F8E4
:104BB0000C2022EA030300F80C30A37F1AE7A37F3E
:104BC0007F355B08EDB2A377002BEED14FF0800C60
:104BD000FF220B8801330B8084F81EC00B88C2545F
:104BE000A37FE2E74FF0800CFF220B8801330B809C
:104BF00084F81EC00B88C254DFE75BB9A37F802B0B
:104C00001EBF013292B20A80904594BF002001205D
:104C1000BDE8F0875246FBB2FFF7D0FC0A88EDE70B
:104C20005005002047F26F7300222DE9F04F82708B
:104C300003800B780D46A3F1FE03B3FA83F35B09FF
:104C400083708A78044612F001011CBF43F0800390
:104C50008370D5F8202185B022F07F4222F0FF0238
:104C600012B143F008038370AA68C2F31702FF2A47
:104C700019D9B2F5803F13D34FF0020863F07F03D8
:104C8000A37041EA0801E17009260B220A210823DA
:104C900007204FF0060C4FF0050E4FF0040912E00C
:104CA00043F00203A3701E0600F1EC8008260A22DE
:104CB00009214FF00008072306204FF0050C4FF0A4
:104CC000040E4FF0030995F801A0374604F809A037
:104CD00095F804A09B4604F80EA095F805E0019114
:104CE00004F80CE095F806C0A14404F800C0A078D0
:104CF000000709D595F821018B46E0540B4695F83D
:104D000022111646E1551746AA68E254A37899077E
:104D100008D5AB680BF10202C3F30F23E35597B23A
:104D2000B3463E46B8F1000F05D0AB7AB346E35523
:104D3000771CBFB23E46A378DA0606D595F8233134
:104D4000B346E355771CBFB23E46504B01361B7845
:104D50001FFA86F8A04405F10C0A43B152464046BA
:104D60006B780DF10E01FFF709FE00286ED16A780D
:104D7000514693B24046019306F022FB2178444B02
:104D8000C943C9B2627894F80780595C94F802A0CC
:104D900051404246595C94F803908AEA010A13F89C
:104DA0000A1094F804E089EA010913F8091094F84C
:104DB00005C08EEA010E13F80E10A0798CEA010CE2
:104DC00013F80C10BBF1070F80EA0100195C82EAAE
:104DD00001029A5C25D0217ABBF1080F82EA010218
:104DE0009A5C1ED0617ABBF1090F82EA01029A5CDB
:104DF00017D0A17ABBF10A0F82EA01029A5C10D0A7
:104E0000E17ABBF10B0F82EA01029A5C09D0217BA7
:104E1000BBF10C0F82EA01029A5C1EBF617B4A4023
:104E20009A5CE255019AB5F80C311644B6B2A35516
:104E3000B5F80C21731C9BB2120AE254AB78B01C7B
:104E4000DB0780B20CD405B0BDE8F08FA37843F047
:104E50004003A370BDF80E30019389F800308DE750
:104E6000D5F81821D5F81071D5F81411231827504A
:104E700059609A6095F81C210F36B0B21A7305B0CC
:104E8000BDE8F08F4FF00008FDE600BFF8020020FB
:104E90003CBA00082DE9F04F0746944D0C462846D1
:104EA000394683B0164606F08BFA00238021904ADB
:104EB0002380138482F82210002E00F0CD804FF062
:104EC000400B4FF0FF089E4695F800C082F822B0D4
:104ED0004FEADC1C92F8229015F803A04FEA4C0C24
:104EE0001AEA090F4FEA590018BF4CF0010C82F87A
:104EF0002200002800F0B380BCF1020F00F04484CF
:104F0000BCF1030F00F0DF83BCF1010F40F0BA8069
:104F10009E4240F2A18015F8039019EA000F14BFD9
:104F20004FF0010C4FF0000C5FEA500A40F0B683DE
:104F300001339BB29E42138482F8221040F28C808F
:104F4000E8564FEA4C0C002801DA4CF0010C4020E6
:104F500082F822B000909E427ED9009815F8039006
:104F60004FEA4C0C19EA000F00985FFA8CFC18BF4E
:104F70004CF0010C5FEA500A40F0258401339BB2EB
:104F80009E42138482F8221066D94FEA4C0015F92C
:104F900003C015F80390BCF1000FC0B201DA40F075
:104FA00001004FEA400C19F0400F18BF20205FFAB3
:104FB0008CFC00F09D854CF0010C002840F0998598
:104FC00001339BB29E42138482F8221044D915F912
:104FD00003904FEA4C0CB9F1000F5FFA8CF015F812
:104FE00003C001DA40F0010040001CF0400F18BF80
:104FF0004FF0200AC0B200F0B78540F0010082F8FF
:1050000022A0BAF1000F03D10133138482F82210D9
:105010007D2821D84130238803F1010CA4F800C079
:10502000F854138C9E4217D992F8220015F803C049
:1050300010EA0C0F4FEA500014BF4FF0010C4FF074
:10504000000C82F8220020B901339BB2138482F84D
:1050500022109E423FF63EAF03B0BDE8F08F013311
:105060009BB2BCF1020F138482F8221000F0AD81D4
:10507000BCF1030F00F03482BCF1010F4FF080004F
:105080003FF446AF9E42E7D915F803C010EA0C0F73
:105090001ED05FEA50092DD101339BB29E4213848A
:1050A00082F82210D8D9E8560028C0F2E8804FF0E4
:1050B00080094FEA590082F8220018B9013313849D
:1050C00082F822102388581C208007F80380A8E764
:1050D000400882F8220018B90133138482F82210A4
:1050E0002388581C208007F803E09AE72404002056
:1050F0005005002019EA0C0FDBD0800840F0C0807A
:1051000001339BB29E42138482F82210A4D9E85640
:105110000028C0F2668280205FEA500C40F0418295
:1051200001339BB29E42138482F8221094D9E85C2A
:105130004FEAD01C40064FEA4C0C40F1BB842020C3
:105140004CF0010C82F8220028B9802001339BB278
:10515000138482F822109E427FF67EAF15F80390EA
:105160004FEA4C0C10EA090F5FFA8CFC18BF4CF0A8
:10517000010C400840F06D8301339BB29E421384C2
:1051800082F822107FF668AFE8564FEA4C0C0028F0
:105190005FFA8CFC80F22F8480205FEA50094CF08B
:1051A000010C40F0648301339BB29E42138482F869
:1051B00022107FF651AF4FEA4C0015F903C0C0B280
:1051C000BCF1000F80F223844FF080095FEA590997
:1051D00040F0010040F0588301339BB29E4213849B
:1051E00082F822107FF638AF15F903C04000BCF1F9
:1051F000000FC0B280F224844FF080095FEA5909A1
:1052000040F0010040F04C8301339BB29E42138476
:1052100082F822107FF620AF15F903C04000BCF1E0
:10522000000FC0B2C0F20F844FF0400915F803C060
:10523000400019EA0C0FC0B200F051834FEA59093F
:1052400040F0010082F82290B9F1000F40F0028492
:1052500001339BB2138482F822101FFA80FC0028CD
:105260003FF4E0AE00232088013300F10109A4F8E7
:10527000009007F800E098B26045F4D3D1E64020F2
:1052800015F803C010EA0C0F3FF446AF400840F099
:10529000A98101339BB29E42138482F822107FF6CB
:1052A000DBAE15F803904FEAD91C19F0400F4FEA16
:1052B0004C0C00F0F38320204CF0010C002840F04F
:1052C000EE8301339BB29E42138482F822107FF654
:1052D000C3AE4FEA4C0C5FFA8CF015F903C015F819
:1052E0000390BCF1000F01DA40F00100400019F01A
:1052F000400F18BF4FF0200CC0B200F02A8440F0DD
:105300000100BCF1000F40F0268401339BB29E42A5
:10531000138482F822107FF69FAE15F903C0400077
:10532000BCF1000FC0B201DA40F001004FF0400ABA
:1053300082F822B09E427FF68FAE15F803C040007F
:105340001AEA0C0FC0B218BF40F001005FEA5A0C15
:1053500040F0D48201339BB29E42138482F8221023
:105360007FF67AAE15F903C04000BCF1000FC0B261
:10537000C0F273834FF0400C15F8039040001CEA14
:10538000090FC0B200F0D9824FEA5C0C40F0010076
:1053900082F822C0BCF1000F40F0668301339BB25B
:1053A000138482F822101FFA80FC00283FF43AAEE2
:1053B00000232088013300F10109A4F8009007F8C8
:1053C000008098B28445F4D82BE69E427FF644AE26
:1053D0004FF04009E85CC009B2F820C0430015F85E
:1053E0000C004FEA590A19EA000F01D043F00103FB
:1053F000BAF1000F40F0B0820CF1010C1FFA8CFCE6
:105400006645A2F820C082F822107FF625AE15F975
:105410000C905800B9F1000FC0B280F2DA8240233C
:1054200040F00100002B40F0A4820CF1010C1FFAA7
:105430008CFC6645A2F820C082F822107FF60CAEE4
:1054400015F90C304FEA4009002B5FFA89F980F218
:10545000C982402049F00109002840F099820CF1EE
:10546000010C1FFA8CFC6645A2F820C082F82210BD
:105470007FF6F2AD15F90C004FEA49030028DBB2C4
:1054800080F2BC824FF0400943F00103B9F1000FF4
:1054900040F08D820CF1010C1FFA8CFC6645A2F8DD
:1054A00020C082F822107FF6D7AD15F90C005B0002
:1054B0000028DBB280F2C182402043F0010382F871
:1054C000220028B90CF1010CA2F820C082F82210A9
:1054D0002088013300F1010CA4F800C03B54A0E582
:1054E0009E427FF6B9AD4FF0400915F803C04FEA70
:1054F000DC101CEA090F4FEA40004FEA590A01D0BC
:1055000040F00100BAF1000F40F0348301339BB248
:105510009E42138482F822107FF69EAD15F9039007
:105520004000B9F1000F15F803C0C0B201DA40F035
:10553000010040001CF0400F18BF4FF0200AC0B21D
:1055400000F0EF8240F00100BAF1000F40F0EB8272
:1055500001339BB29E42138482F822107FF67CAD09
:1055600015F903904000B9F1000F15F803C0C0B25F
:1055700001DA40F0010040001CF0400F18BF4FF06E
:10558000200AC0B200F0D88240F0010082F822A0C8
:10559000BAF1000F03D10133138482F8221041388D
:1055A00039E515F8039019EA0C0F14BF4FF0010C00
:1055B0004FF0000C5FEA900A40F0358201339BB255
:1055C0009E42138482F822107FF646ADE8564FEAD9
:1055D0004C0C002801DA4CF0010C402082F822B07B
:1055E000B9E5402015F8039019EA000F14BF4FF0F9
:1055F000010C4FF0000C5FEA500A40F00B820133BF
:105600009BB29E42138482F822107FF625ADE856A5
:1056100015F8039000284FEA4C0C01DA4CF0010C0D
:105620004FEA4C0C19F0400F18BF4FF0200A5FFAF8
:105630008CFC00F046824CF0010CBAF1000F40F0F7
:10564000428201339BB29E42138482F822107FF67D
:1056500003AD15F903904FEA4C00B9F1000F15F8AE
:1056600003C0C0B201DA40F0010040001CF0400F5E
:1056700018BF4FF0200AC0B200F0638240F0010072
:1056800082F822A0BAF1000F7FF454AE01339BB22E
:105690004FF0800A138482F822104BE6800819EA42
:1056A0000A0F00904FEA4C0C01D04CF0010C82F82C
:1056B000220000287FF44FAC01339BB2802013847A
:1056C00082F8221046E415F803C01CEA000F14BF4C
:1056D000012000205FEA99097FF40BAF01339BB2F0
:1056E0009E42138482F822107FF6B6AC15F903901F
:1056F00015F803C0B9F1000F4FEA400001DA40F09D
:1057000001001CF0400F18BF4FF020094FEA400085
:1057100000F0B98140F00100B9F1000F40F0B5810F
:1057200001339BB29E42138482F822107FF694AC20
:1057300015F903904000B9F1000F15F803C0C0B28D
:1057400001DA40F0010040001CF0400F18BF4FF09C
:105750002009C0B200F0C18140F00100B9F1000F92
:1057600040F0BD8101339BB29E42138482F8221027
:105770007FF672ACEB564000002BC0B201DA40F06D
:10578000010082F822B00AE792F8229019EA0A0F83
:1057900014BF012000205FEA59097FF41DAE0133D8
:1057A0001FFA83FC6645A2F820C082F822107FF61B
:1057B00053AC15F90C904300B9F1000F80F202814F
:1057C0004FF0400A12E64FEA4C0C800819EA0A0F23
:1057D0005FFA8CFC019001D04CF0010C002840F0E5
:1057E000D28101339BB29E42138482F822107FF64D
:1057F00033AC4FEA4C0015F903C015F80390BCF127
:10580000000FC0B201DA40F00100400019F0400F73
:1058100018BF4FF0200C5FFA80FA00F075814AF053
:10582000010ABCF1000F40F0718101339BB29E422E
:10583000138482F822107FF60FACEB564FEA4A0031
:10584000002BC0B201DA40F0010082F822B0FFF76D
:10585000DFBB15F803904FEA4C0C10EA090F5FFA12
:105860008CFC7FF49AAC5FEA50093FF49CAC4FEAA1
:105870004C0015F803C0C0B219EA0C0F7FF4A6ACB7
:105880005FEA59093FF4A8AC15F803C0400019EAD3
:105890000C0FC0B27FF4B2AC5FEA59093FF4B4AC6C
:1058A00015F803C0400019EA0C0FC0B201D040F057
:1058B00001005FEA59097FF4B9AC01339BB29E4203
:1058C000138482F822107FF6C7AB15F903C040009D
:1058D000BCF1000FC0B2C0F2B9804FF080094FEAAE
:1058E000590982F82290B9F1000F3FF4B1AC1FFAC8
:1058F00080FC00287FF4B6ACFFF796BB15F8039048
:1059000040001CEA090FC0B201D040F001005FEA7C
:105910005C0C7FF431AD01339BB29E42138482F85C
:1059200022107FF699AB15F903C04000BCF1000FBF
:10593000C0B2C0F295804FF0800C4FEA5C0C82F848
:1059400022C0BCF1000F3FF429AD1FFA80FC0028F3
:105950007FF42EADFFF768BB15F80C9058001AEADB
:10596000090FC0B24FEA5A037FF45AAD002B3FF43F
:105970005CAD15F80CA04FEA400913EA0A0F5FFA74
:1059800089F94FEA53007FF465AD00283FF467AD15
:1059900015F80CA04FEA490310EA0A0FDBB24FEAF0
:1059A00050097FF471ADB9F1000F3FF473AD15F8F4
:1059B0000CA05B0019EA0A0FDBB24FEA59003FF472
:1059C0007EAD7AE515F80C3080005B064FD52023BC
:1059D00026E59B005FFA83F915F80C30580648D588
:1059E000202037E58000C3B215F80C00400642D5F0
:1059F0004FF0200948E54FF0400938E715F80C0052
:105A00004FEA89034006DBB238D5202055E54FF038
:105A1000400939E719EA0A0F4FEA90004FEA4C0CA7
:105A20003FF44CAC48E419EA0A0F4FEAD0004FEAC1
:105A30004C0C3FF487ABFFF783BB82F822B047E5FD
:105A40004FF040092CE74FF0800930E740F00100AB
:105A500082F822B01FFA80FC04E44FF0800C54E777
:105A600040F0010082F822B01FFA80FCA0E420235D
:105A70007FE720208CE74FF0200998E74FF02000C7
:105A800082F8220024E54FF02009400019EA0C0FAB
:105A9000C0B24FEA590A3FF457AD53E520204FEA10
:105AA0004C0C19EA000F5FFA8CFC4FEA500A3FF4E5
:105AB000C4ADC0E54FF0200082F822002020FFF79F
:105AC0004ABB4FF0200A4FEA4C0019EA0A0FC0B255
:105AD0004FEA5A0C3FF415AC11E44FF02009400096
:105AE00019EA0C0FC0B24FEA590A3FF44FAD4BE52B
:105AF00020204FEA4C0C10EA090F5FFA8CFA4FEAAB
:105B0000500C3FF48EAE8AE64FF0200C4FEA4A006C
:105B100019EA0C0FC0B24FEA5C0A3FF470AAFFF713
:105B20006CBA4FF0200A40001AEA0C0FC0B24FEADC
:105B30005A093FF413AE0FE64FF0200382F82230EB
:105B40002DE54FF0200C4FF0200A82F822C0FFF71D
:105B5000F1BB4FF0200C400019EA0C0FC0B24FEA25
:105B60005C0A3FF48DAD89E54FF0200382F82230C6
:105B7000FFF74EBA40001AEA0C0F4FEA9909C0B27B
:105B80003FF4CAADC6E5824600984FEA4C0C19EACC
:105B90000A0F4FEAD0005FFA8CFC3FF40EAAFFF721
:105BA0000ABA00BF2DE9F04F0D4651881446B1F5F1
:105BB0008F7F06468BB00BD90022227000226F2BFC
:105BC000628000F06281002333700BB0BDE8F08F7B
:105BD00012780E2A24D80E2A00F2108101A050F863
:105BE00022F000BFBD5B0008095E0008FD5D0008F3
:105BF000FD5D0008095E0008095E0008095E0008F6
:105C0000095E0008095E0008095E0008555E00088C
:105C1000FD5D0008FD5D0008FD5D0008795E00087F
:105C2000692A40F2E9806A2A40F0E8809B4FFA8AAC
:105C300002F1FF3C1FFA8CFC002A00F07982FF225F
:105C40000CF1030CDFF858E2BC44B91C11F8010B4D
:105C5000424061451EF80220F8D1934200F0D18104
:105C600000222270C4F80220E280FA8A022AAAD90D
:105C700039796F2900F02E83032AA4D079796F290E
:105C800000F03883042A9ED0B9796F2900F035835B
:105C9000052A98D0F9796F2900F03B83062A92D023
:105CA000397A6F2900F04682072A8CD0797A6F29D9
:105CB00000F03283082A86D0B97A6F2900F02F834A
:105CC000092A80D0F97A6F2900F02C830A2A3FF440
:105CD0007AAF397B6F2900F028830B2A3FF473AF2A
:105CE000797B6F2900F024830C2A3FF46CAFB97BD9
:105CF0006F2900F020830D2A3FF465AFF97B6F29EF
:105D000000F01C830E2A3FF45EAF397C6F2900F04F
:105D10001B830F2A3FF457AF797C6F2900F0118362
:105D2000102A3FF450AFB97C6F2900F01083112A7C
:105D30003FF449AFF97C6F2900F00C83122A3FF43D
:105D400042AF397D6F2908BF4FF012087FF43BAF97
:105D500002F101091FFA89F93A44A7F816905FFA8F
:105D600089F993704F494A4602A805F029FB6F2331
:105D70004FF0010CBB704FF0000E6423A7F800E059
:105D8000A7F816C0237008EB0C0399451FFA89F297
:105D90007FF619AF901EA0EB080002A95A1E80B230
:105DA0000B444FF06A084FF007094FF0660A0A44A7
:105DB000184405E0002B40F0C08190423FF403AF4F
:105DC000FB8A12F8011F03F1010B3B44A7F816B040
:105DD00099702378092BEDD9A3F1640BBBF1050F62
:105DE000EBD8653B042B00F2B882DFE813F0210109
:105DF0001901140110011D01632A05D80023237025
:105E0000C4F80230E380DFE6244FFA8A511C3A449A
:105E1000F98293702278092A00F2A680002A3FF4C2
:105E2000D2AE013A082A3FF6CEAE01A151F822F0D7
:105E30000D610008C75B0008C75B000859600008D7
:105E400059600008F7600008AD600008E1600008D4
:105E5000CB6000084A1C114E62806B54A088727F90
:105E6000618883189942FFF6B0AE33785F0600F17F
:105E7000E8810E232370A8E64A1C62806B54E288F6
:105E80006388934210D201239EE604490A808B70F6
:105E900001226423CA822370002395E65005002066
:105EA0003CBA0008520500200023022163802370C1
:105EB000317072802B78FD2B00F08A80EB78337282
:105EC0002B7973726B7973606A78083272804FF441
:105ED000BC700022F6210446DFF8D0C27281013482
:105EE00099424FEA540431D84CD38B4240F08D8014
:105EF0002B78FD2B00F082804FF0060B284610F81F
:105F000001AF62000BEB0A0909F1FF3189B201927E
:105F1000FBF710FADFF8948204EB440708EB8707DD
:105F20003979ADF8080002A80191FBF7DFF905EB1C
:105F30000902527815F80930019903EB0223BDF8E4
:105F400008209BB29A421FD005233DE6601E14181C
:105F5000824204F1010780F06D8127F0010101EB1D
:105F600057015CF82110BAE7A2F1640105293FF658
:105F70002AAE653A042A00F2F981DFE802F0819343
:105F800079757D002246E2E7BB79DA0706D5FA7912
:105F9000924582BF521912F80B20B2729B070BD5A3
:105FA0006300234408EB83031B7A6A789A4282BF1A
:105FB0005B1913F80B30F3724FEA4409A14408EB64
:105FC000890898F80530317373730BB0BDE8F08F12
:105FD0006B793372AB7973726B7A297AEA791B0425
:105FE00003EB0123134473606A7802F10C017180A2
:105FF000A978C9077FF56BAF193267E74FF00A0B35
:106000007CE70A2201232270DEE50323DCE5F97632
:1060100084F80090D1E64FF06803B9762370CCE69F
:10602000797084F800C0C8E6397784F80080C4E647
:10603000397001F001036188033B01F1010B87F81E
:1060400001E0A4F802B06B5497F90030002BACBF0C
:10605000634653462370B0E66288511C6180AB549E
:1060600023780133237017E70722FB762270AAE515
:106070006822BB762270A6E56A223B772270A2E5F1
:1060800000227A7062883B7003F00103033B511CCD
:106090006180AB5497F90030002BB4BF6623012315
:1060A0002370F9E601227B7022708CE56288511C16
:1060B0006180AB543B787A78134313F0020340F0CD
:1060C000D8806288511C6180AB546288511C618009
:1060D000AB543B78D8064CBF69236A232370DBE6B8
:1060E0006288511C6180AB547B7813F00203ECD0C2
:1060F00009232370D0E66288511C6180AB543B7841
:106100001D074CBF672307232370C5E66288511C17
:106110003A836180AB543A787B7712F0010200F049
:10612000C48006220833E380A28004232370B3E6F0
:10613000FF2292E54FF006080AE6013B082B3FF6E6
:106140003CAE0FF2080B5BF823F000BF856100083E
:10615000BB5D0008BB5D000871610008716100084B
:10616000FF610008CD61000819620008B1610008F4
:10617000638803F1010BA4F802B0E95423780133DA
:1061800023701AE6638803F1010B3B83A4F802B085
:10619000E9543B78797713F001036DD00623083179
:1061A000E180A3800423237007E600BF3CBB000806
:1061B000638803F1010BA4F802B0E9543B78DB06D5
:1061C0007FF533AF4FF069032370F6E5638803F181
:1061D000010BA4F802B0E9543B7879780B4313F033
:1061E000020343D1618801F1010BA4F802B06B54A2
:1061F000618801F1010BA4F802B06B54DEE76388FB
:1062000003F1010BA4F802B0E9543B7819077FF5BC
:10621000FFAE67232370D0E5638803F1010BA4F878
:1062200002B0E9547B7813F00203E1D04FF0090388
:106230002370C2E5554902EB4200144651F8201084
:1062400053E602A92844FEF725FE737FBDF8081027
:106250006288CB1A9BB21A446280727F1A447277AA
:10626000E2881344E380338BE95402E60823237069
:10627000A3E5082323700FE60C31E1800A21A180F9
:10628000797811F0010128D0618801F1010BA4F89F
:1062900002B005F801C0618801F1010BA4F802B059
:1062A0006B54E3880D33E3807CE70C33E3800A23EF
:1062B0007978A38011F0010122D001216388581858
:1062C0006080E954638859186180EA54E3880D338B
:1062D000E3802AE74FF002083AE5638803F1010BF7
:1062E000A4F802B0E954638803F1010BA4F802B0EA
:1062F000E95457E74FF003082AE54FF0040827E573
:1063000063885A1C6280E95463885A1C6280E9548D
:106310000BE74FF005081BE54FF0070818E54FF0B5
:10632000080815E54FF0090812E54FF00A080FE5D7
:106330004FF00B080CE54FF00C0809E54FF00D0885
:1063400006E54FF00F0803E54FF00E0800E54FF0AB
:106350001008FDE44FF01108FAE477290ED084F814
:1063600000E0C4F802E0A4F806E026E5772B09D0A7
:1063700000232370C4F80230E38024E44FF0650367
:1063800023701AE56523237086E500BF3CBB000837
:106390002DE9F8431F46184B164693F83020044663
:1063A0003AB393F82B301FB11BB31F1F18BF01273F
:1063B000A1F1020804F5E36901F11E0538F8020FA6
:1063C000FAF774FB29F8020FB8F80000FAF77BFB24
:1063D000A845A9F82000F1D1084B86F001061B68FA
:1063E00084F85A77C4F85C37012384F8606784F82E
:1063F0001937BDE8F88300BFA4000020A02C0020BE
:1064000010B500F27C7400F5B0712046FAF7DFFF9A
:1064100001462046BDE81040FCF73EB8B0F8E8342D
:10642000B0F8EA249B1A98B21B0444BF00F5007030
:1064300080B2003818BF012070470346D0F8F82614
:10644000B0F8E8140132C0F8F826D0F8002701327D
:10645000C0F80027B0F8EA2491421FBF811891F8D4
:10646000EE04B3F8EC1401321ABF0A40A3F8EA2490
:10647000002070470F4B93F82D305A1E012A02D886
:106480000D48FFF7DABF032B10D10C4AB2F81E36C5
:10649000B2F81C1699420BD0D11891F82206B2F826
:1064A000201601330B40A2F81E367047FCF716B8D1
:1064B00000207047A4000020E0050020880E002086
:1064C0000023064AA0F8EA341380054AA0F8E8340D
:1064D0001380044A1380044A1380704796280020D2
:1064E000982800209A2C00209C2C002008B50848F1
:1064F000FFF7E6FF0023074AC2F81C36064A13805E
:10650000064A1380064A1380064A138008BD00BF5E
:10651000E0050020880E0020962800209828002002
:106520009A2C00209C2C0020B0F8EA24B0F8E83423
:1065300010B59B1A9CB21B0448BF04F500740146B9
:1065400048BFA4B2FBF7B8FF0319D1F8F00618440E
:1065500080B210BDF8B5D0F8F4360446CB1AB3F5C6
:106560007A7F0E4690F8187726D2632B01D8002048
:106570007DE0012F0AD0022F19D0002FF7D1FFF7AD
:10658000D3FFB0F5806FF2D9012305E0FFF7CCFF10
:10659000B0F5806F03D9022384F818370CE0204649
:1065A000FFF7C2FFB0F5C07FE1D20023F4E7FFF7A9
:1065B000BBFFB0F5806FE7D33448C4F8F466FAF750
:1065C000D6F9334D334A2B681168C3F1000C411AD8
:1065D000614501DB99424BDD0A2310602B60136893
:1065E0005221B3F5FA7FBCBF4FF4FA7313601268FF
:1065F00064254A432849D4F8F836B1F848106B436B
:1066000092FBF1F2B3FBF2F35F2B35D8552B35D863
:106610003B2B03D94B2B34BF5B25322594F818371D
:10662000022B2DD0012B2DD013B9002F18BF3325ED
:106630004FF47A733146D4F8002704F20470FAF765
:106640008BFD94F81837FBB9642D0BD10322D4F8D5
:10665000F436A3F29A23C4F8F436D4F8F8365B0083
:10666000B3FBF2F30120C4F8F83684F8FC56F8BD09
:10667000002BB4DD013BB1E70025CFE71E25CDE7B8
:106680000025D5E73225D3E70023EBE78C1D00205A
:1066900008000020FC0200204800002070B5D0F85F
:1066A000F4360446CB1AB3F57A7F0E4690F81827D5
:1066B00014D2032A08D8DFE802F002092730FFF7D6
:1066C00033FFB0F5487F26D8002029E0FFF72CFFE4
:1066D000B0F5AF6F11D9022384F81837304B94F816
:1066E0001857B3F84800C4F8F466D4F8F836032D08
:1066F0004ED8DFE805F03716494B2046FFF714FF68
:10670000A328E1D80323E7E7632BDDD9FFF70CFFCC
:10671000B0F5AF6FE2D20123DEE7002084F818075E
:1067200070BD21254FF47A733146D4F8002704F266
:106730000470FAF711FD94F818377BBB642D0BD168
:106740000522D4F8F436A3F54873C4F8F436D4F827
:10675000F8369B00B3FBF2F30120C4F8F83684F856
:10676000FC56DDE764210F4A4B43B2FBF0F2B3FB6A
:10677000F2F35F2BD6D8552B0CD83B2B0CD94B2BD7
:1067800034BF5B253225CDE70025CBE75D25C9E782
:106790006425C7E71E25C5E70D46C3E70023DBE7F1
:1067A0004800002050400100F8B5234F0446384609
:1067B000FAF7A6F8FAF71BF9064697F9A600FAF7D2
:1067C00016F905463846FAF7A4F894F8FC366D2217
:1067D00084F87231FF2384F87431332384F86531EF
:1067E000442384F86631D4F86831C0F10A0062F3BA
:1067F0001703C4F868310023C4F86C3184F881327F
:106800004FF43943A4F88232092300B280F3070021
:1068100084F8730184F8706104F5B07084F87151E4
:1068200084F8843204F5AA71FBF7AEF82046BDE87F
:10683000F840FFF7E5BD00BF8C1D00202DE9F04FAB
:106840000446B0F828670378B0F822E7B0F824C708
:10685000B0F81CA7B0F81E97B0F82087B0F82677DC
:10686000B0F82A57B0F82C07A4F87A610026B4F8DB
:106870002E2785B00092B4F83027B4F8361701926D
:10688000B4F83227B4F834B70292B4F83827A4F831
:1068900074E10392B4F81A27A4F876C1A4F86C2125
:1068A00084F87C31A4F86EA1A4F87091A4F87281E8
:1068B000A4F8787184F87D61A4F87E51009A84F878
:1068C0008132A4F88221019A4FF4F843A4F884217C
:1068D000029AA4F88A11A4F88621039A4621A4F802
:1068E0008C21FF2284F865214422A4F882322623D9
:1068F00084F86621D4F86821A4F8800161F31702B6
:1069000004F5B070A4F888B184F88E6184F88F61C2
:1069100084F8906184F89161C4F8682184F8843225
:1069200004F5AA71FBF730F8204605B0BDE8F04F3A
:10693000FFF766BDF0B591B004466D4600F23A73BC
:1069400000F25A762A4618685968083303C2B342DF
:106950001546F7D1202200210DEB020004F0CEFCF9
:1069600094F8602794F85A370AB943F00203A4F860
:106970007031002384F87331102384F874316B462E
:106980002678D4F85C2784F87261C4F86C2104F28C
:10699000751510AF1A4603CABA42286069601346DB
:1069A00005F10805F6D1332384F8653144234FF40B
:1069B000D27284F86631D4F8683104F5B07062F3AD
:1069C0001703C4F868314FF4A053A4F88232492366
:1069D00084F8816284F8843204F5AA71FAF7D4FF4E
:1069E000204611B0BDE8F040FFF70ABD5D4B2DE930
:1069F000F04F1A68D0F864370446D31A122BA3B0AC
:106A000040F2AC80DFF86081584E98F80010C0F872
:106A100064278A1E5142514196F9A000F9F7FFFF01
:106A200096F8A43096F8A520012B0CBF0323012370
:106A3000012A96F8AA200CBF43F0080343F0040390
:106A4000012A96F8AB2008BF43F010030746012A3D
:106A500047480CBF43F0200543F04005FCF7FEFD1E
:106A6000F9F73EFC4349F9F793FC04F009FC42496D
:106A7000F9F78EFC82463D4896F9A290F9F752FF4D
:106A800083463A48F9F75CFF98F8001001908B1E96
:106A900002290CBF96F8A9804FF0000859425941CD
:106AA00096F9A600F9F7BBFF80220646002102A84E
:106AB00004F024FC019B6FF02F028DF80D304FF68F
:106AC0007F73ADF81230ADF814307F238DF8163097
:106AD000002384F86D3184F86F311723ADF8085026
:106AE000257884F86C2184F8703102A9802284F81A
:106AF0006E5104F271108DF80CB08DF80E708DF897
:106B00000F908DF810808DF81160CDF817A0CDF89A
:106B10001BA004F055FC332384F86531442340F274
:106B2000811284F86631D4F8683104F5B07062F3EC
:106B30001703C4F868314FF41343A4F88232852355
:106B400084F8815284F8843204F5AA71FAF71CFFA4
:106B5000204623B0BDE8F04FFFF752BC23B0BDE89C
:106B6000F08F00BFA02C00202B0300208C1D0020E4
:106B70004403002000007A3D00007A442DE9F043F0
:106B800004464B4B4B48A9B01D68FCF759FD40F635
:106B9000C312D4F86837EB1A934204D894F96C37CF
:106BA000834200F08180444EC4F86857B1784FF0BA
:106BB000060805298CBF0025404B4FF000079BBFFE
:106BC00033F811903E4BA94633F811507F238DF8CE
:106BD0001030B6F84A30424684F86C078DF8110040
:106BE0000DF11200ADF80430ADF806308DF80F103D
:106BF000ADF80C708DF80E80FAF744F971784246C2
:106C000006A8FAF71BF92B48ADF80A50ADF8089022
:106C1000FCF708FD40428DF81E002648FCF702FDF7
:106C20004042642239468DF81F0008AD0FA801AE1E
:106C300004F064FB0FCE0FC596E807006FF02E033B
:106C400084F86C311C2385E807002578802284F8BD
:106C5000703108A984F86D7184F86E5184F86F71F1
:106C600004F2711004F0ACFB332384F86531442343
:106C700040F2811284F86631D4F8683104F5B070BE
:106C800062F31703C4F868314FF41343A4F8823257
:106C9000852384F8815284F8843204F5AA71FAF7C6
:106CA00073FE2046FFF7ACFB29B0BDE8F08300BFC0
:106CB000A02C0020481E0020480000207EB90008BB
:106CC0008AB9000810B5044690F87407B4F8701734
:106CD00084F86F016FF06E00A4F86C11002184F845
:106CE00070016FF02A0084F86E1184F8731133215B
:106CF00094F8733784F87101122084F8753184F8A0
:106D000082328F2384F86511442184F872014D206A
:106D100084F883320A2384F86611D4F8681194F851
:106D2000722760F31701C4F8681104F5B07084F895
:106D3000742184F8812284F8843204F5AA71FAF768
:106D400023FE2046BDE81040FFF75ABB4FF07E53AC
:106D5000082110B5C0F86C31002380F88811022199
:106D6000C0F87031C0F87431C0F87831C0F87C31A7
:106D7000C0F88031C0F8843180F88C31332380F83A
:106D80008911012180F86531442380F88B114C2151
:106D900080F86631D0F86831044661F31703C0F813
:106DA000683149F60103A0F882322123027880F885
:106DB000843280F88A2180F8812200F5AA7100F5DA
:106DC000B070FAF7E1FD2046BDE81040FFF718BBB0
:106DD000F0B54E780D46202E04468BB001F10C0123
:106DE00032D8324601A804F0EBFA01AB0021C6F11B
:106DF0002102981904F082FA9DF82230332B57D1E2
:106E00009DF82330442B53D1BDF82030F62B02D00F
:106E1000B3F5FA7F4CD1B4F87027A4F870379A42D2
:106E20001CBF002284F87427012284F86D276A7938
:106E3000F62B84F87227AA7984F8732713D0B3F558
:106E4000FA7F1CD0002324E00B4601AA05F12C0791
:106E5000164618685968083303C6BB423246F7D154
:106E60001B783370C8E713490398F9F725FC00280D
:106E7000E8D011490498F9F71FFC0028E2D00F4927
:106E80000798F9F719FC0028DCD09DF82430012B75
:106E900002D184F874370BE0022BD3D194F8742715
:106EA000002ACFD084F87437054B1B68C4F87837B4
:106EB0000BB0F0BD000040400000884288AC96490D
:106EC000A02C00204FF47F4303800023C0E901334E
:106ED000C0E90333436103767047000038B50023EF
:106EE000C0E90733C0E955334362C0F85C3104465A
:106EF000FAF7BCFA254B9878022845D0431F584230
:106F00005841FDF753FB40F2FF130025A4F8EC3481
:106F10001F4B04F204701B68C4E9A25503F57A7391
:106F2000C4F8F436C4F89052A4F8EA54A4F8E8542B
:106F3000C4F8F05684F8FC5684F81857C4F8F8568C
:106F4000C4F80057FAF702F9294684F8195704F2F1
:106F50001A70402204F0D2F97D23204684F85A5753
:106F6000C4F85C5784F86057C4F86457C4F868578D
:106F7000A4F86C37A4F8725784F87457C4F878579B
:106F8000BDE83840FFF79EBF0120BAE74800002067
:106F9000A02C002030B40E4A92F82E40012C14D1BF
:106FA0000C4A0178126881B140F6C4150169511A82
:106FB000A94202D930BCFFF785BF416829B94169B0
:106FC000511AFA2984BF4261047630BC704700BF71
:106FD000A4000020A02C00204378032B06D1C06819
:106FE000B0F5834F34BF0020012070470020704768
:106FF0007FB50B46324900F1280691F82D10044662
:10700000022900F11C02314668461BD1FEF7CAFD79
:107010009DF80030022B50D104F5B0753246694618
:107020002846FAF731FAD4F8683123F07F436E2B03
:107030002FD1244B9A78052A3DD8DFE802F030346E
:1070400038063038FAF794FBE2E75A6CB2F5613F44
:1070500094BF002201222046FFF7BEFFC8B9C2B18B
:1070600094F86E31012B14D894F87231042B10D19E
:107070001022154904F27B1004F064F948B9782312
:10708000284684F8883184F8823184F87C31FDF711
:107090005FFA204604B0BDE87040FFF7B1B95A6C02
:1070A000B2F5E13FD4E75A6CB2F5614FD0E75A6CC4
:1070B000B2F5164FCCE70122CDE704B070BD00BF9A
:1070C000A4000020480000203DB60008F0B54E782E
:1070D0000546082E0C4685B001F10C0717D832463C
:1070E000394601A804F06CF901AB0021C6F1090290
:1070F000981904F003F99DF80930032B05D1627942
:107100002A70064A12686B702A6105B0F0BDC86823
:10711000796801AB03C33A7A1A70ECE7A02C00201F
:1071200030B50378044695B013B34A799A421FD11B
:107130004D780C314D2D1DD82A46684604F040F993
:107140000021C5F14E020DEB050004F0D7F842F224
:107150001070049B190EC3F3072200FB0122642167
:107160006360C3F3074301FB0323E360059BA36054
:1071700015B030BD4E22684604F022F9E7E7000062
:107180008A68C2F317024C2A16D0942A0AD0AAB9E8
:107190000B4A92F82E20012A10D18B79012B0DD1A8
:1071A000FFF794BF064A92F82E20012A06D18B7968
:1071B000012B03D1FFF7B4BFFFF70ABE704700BF32
:1071C000A4000020B0F8EA34B0F8E824F0B5D21AF0
:1071D00093B2120444BF03F500739BB2DD2B044647
:1071E00085B006D800F5257600F52275FAF770F817
:1071F00008B905B0F0BDFBF771F9D4F8F0260346E5
:107200000132C4F8F02631462A466846FAF7B0FA49
:107210009DF80030022BE9D104F5707532466946BD
:107220002846FAF731F9184B04F27C7693F82D30A2
:107230002946022B30460FD1FDF7F4FC00239AB209
:1072400090420CD8002329462046C4F8F03605B0F9
:10725000BDE8F040FFF794BFFAF7B9F8EEE7B4F8ED
:10726000E814B4F8EC744A1C3A40B4F8EA74974253
:107270001EBFF75C091981F8EE7403F1010318BF12
:10728000A4F8E824DBE700BFA40000202DE9F041CA
:10729000494BDFF828811E6898F80030484F022BD0
:1072A0001EBF0023A0F8EA34A0F8E83497F82D3088
:1072B0000446013B012B7CD8FFF784FF97F82E5042
:1072C000002D5AD098F80030022B4AD1012D3DD024
:1072D000022D41D000252046FFF75CFE94F81937B7
:1072E00043B1002384F8193797F83030012B4ED082
:1072F000022B4FD015B12046FFF756FA94F86D37A0
:107300002BB10023204684F86D37FFF7DBFC94F89F
:107310007437022B11D1D4F87837F61AB6F57A7F84
:107320000BD9B4F87037F62B3DD0B3F5FA7F3CD0CB
:107330000023A4F8703784F87437237ECBB300237E
:1073400020462376BDE8F041FFF700BD31462046D8
:10735000FFF700F90546BEE731462046FFF79EF9E4
:10736000F8E7D4F8F436F31AB3F57A7F08D200259B
:1073700004F20470F9F7EAFEADE7C4F8F466F7E743
:1073800032230125C4F8F46684F8FC36F0E7FFF7F1
:1073900055FAAFE7FFF7CEFA2046FFF727FB204666
:1073A000FFF7ECFBA6E7FAF77DFC0122054B5A71CB
:1073B000BEE7BDE8F08100BFA02C00202B03002019
:1073C000A40000200003002070B54C880346B4F5EB
:1073D000427F4FF000000AD80D780B2D77D8DFE8F8
:1073E00005F0060F1C2C2F32383B54575B6DA2F171
:1073F00024046242488062410A7083F809033EE037
:107400004D2A01D0582A06D11A7002220A70002093
:1074100083F8090370BD0022F8E702F0FD003C2864
:1074200001D0212AF7D15A701A784D2A0CBF0822B0
:1074300003220A7000229A70E9E79A700422DBE7BF
:107440009A800522D8E7988800EB02229A800622CB
:10745000DCE7DA800722CFE7D88800EB022292B27D
:10746000002ADA800CBF0B220A220A7000224A800E
:10747000012283F80923DB88B3F5407F01D800207F
:10748000C8E7002008704880C4E7DA800922B3E723
:107490009A800A220A70EBE7B4F5407F3CBFE418FB
:1074A00022724A88013292B24A80D88890429CBFA8
:1074B0000B220A70012283F80923E0E783F80823EE
:1074C000022208704880012083F80923A2E708708F
:1074D0004880D4E7CB8870B5B3F5407F31D82423FA
:1074E00003700B7843704B7883700B784D2B14D15D
:1074F000CB88C3708B88037105230022CE88D418F3
:10750000A4B2964200EB040515D891F808232A701E
:10751000CA880132981880B270BD8B78C3708B888E
:1075200003718B881B0A4371CB888371CB881B0A3C
:10753000C3710823E1E78D182D7A0132055592B207
:10754000DCE70020E8E700002DE9F74F16464A88FF
:107550000446B2F5427F0D462ED80B780A2B0FD980
:10756000A3F16402032A03D90020287068802CE06C
:10757000653B8F4F022B32D8DFE803F062A3A600F1
:1075800000210A2BF0D801A050F823F0B9750008AB
:10759000D17500086975000869750008157600083E
:1075A000237600082F7600083576000869750008F4
:1075B00069750008A37600080020A6F124077E4222
:1075C0007E4168802E7084F8090303B0BDE8F08F17
:1075D0006F2E0CBF6423002300202B70F3E716F0FE
:1075E000040F14BF4D2358233E7023703A78D107FF
:1075F0000ED412F0020F14BF21233E236370C2F396
:10760000C003D20648BF43F00203A3700423E3E79C
:107610003C23F3E70523A6802B7084F80913002090
:10762000D3E7A38803EB0623A3800623D4E707232D
:10763000E680F1E7E38803EB0623E3806523CBE7ED
:107640000DF106007E70F9F7BDFE3978F9F7B2FE4C
:10765000A7882179F9F7AEFE390AF9F7ABFEE7887A
:10766000A179F9F7A7FE390AF9F7A4FE9DF80630CB
:10767000B34206D000232B706B80032384F80933B8
:10768000CDE7002F0CBF66230A232B70012384F85B
:10769000093300236B80E288B2F5407FBFD92B709D
:1076A000BDE7B2F5407F3CBF121916726B880133FB
:1076B0009BB26B80E2889A4201D866232B7001232B
:1076C000DCE767237E80F9E74FF6FF73B7F80280A7
:1076D00097F8009008EB06280DF1060049461FFABE
:1076E00088F8ADF80630A7F80280F9F7FFFD267993
:1076F000B4F804A03146F9F7F9FD4FEA1A21F9F779
:10770000F5FD94F806B0B4F806A05946F9F7EEFD79
:107710004FEA1A21F9F7EAFD797804F10807F9F739
:10772000E5FD52463946F9F7EDFDBDF80630434513
:107730003AD119F0040015D0002386EA0B01E21DAE
:1077400098B2824584F8081307D80223012000224A
:107750002A706A8084F8093337E712F8010F013381
:107760004140EDE7A178F9F705FA217984F808039B
:10777000F9F700FAA18884F80803090AF9F7FAF979
:10778000A17984F80803F9F7F5F9E18884F808038A
:10779000090AF9F7EFF93946E28884F80803F9F79E
:1077A000EFF984F80803D0E703230020CFE700BFF8
:1077B000581C0020CB882DE9F041B3F5407F0446EA
:1077C0000D464BD84B783C2B41D0A3F121004342CE
:1077D00043415B002A78A71C4D2AAA7808BF43F0D2
:1077E0000403D10748BF43F0080392074FF0240277
:1077F00022704FF06F0248BF43F010036270A37015
:10780000AB883846E370AB881B0A2371EB88637141
:10781000EB881B0AA371F9F7EDFE0822E071E988F5
:10782000A2F108039BB2561C8B42B6B204EB0208CD
:107830000FD30631384689B2F9F77CFD88F800008D
:10784000000AA055E8880A3080B2BDE8F081012323
:10785000C0E72B441B7AA3543246E0E70020F4E74C
:1078600030B4BDF80C40B4F5407F03D8039430BC6D
:10787000F9F7DABE002030BC704710B5044624206A
:10788000207058206070002023711B0AA170E270E4
:1078900063710522A071E071E11CF9F771F92072A2
:1078A000092010BD2DE9F04F0025D71891468046DC
:1078B0000C462B462A464FF0FF0BDFF8D8A08FB0BE
:1078C0000D80B94502D10FB0BDE8F08F19F8010B5A
:1078D00011463B2809D00132D2B238316944202AFE
:1078E00008BF002201F8300CEBE74FF00001002642
:1078F00038326A4402F8301CF2B25AF8361002A844
:1079000001930092F8F724FCDDE90023A8B9FF2BCE
:1079100018BF23880AEBC6061EBF591C218008F831
:1079200003B02388591C218008F803203379142BD5
:1079300001D8189AD554FF231BE00136372EDBD12E
:10794000FE2B06D023885A1C22806FF0010208F813
:107950000320002602A8F8F705FC721CF6B2B0421C
:1079600023880AD85A1C22804FF03B0208F80320D3
:10797000FE2301350022EDB2A3E7591C218006F158
:1079800038010DEB010616F8301C164608F80310F6
:10799000E0E700BFD0CF000840F2FF3270B4A0F89B
:1079A00020267D22002380F8542A0A2602460360FE
:1079B000C0F80E33A0F81E36A0F81C36A0F8423AE4
:1079C000A0F8443A80F8463AC0F8483AC0F84C3A31
:1079D000C0F8503AC0F8583A00F6672400F66D2512
:1079E00014F8011F09B1B6FBF1F1AC4282F8701A2C
:1079F00082F8713AC2F8743A02F10802F0D170BC10
:107A00001522FF2100F52A6003F078BCF8B5134A6F
:107A1000044692F83000F8B192F82B2003B1DAB1A5
:107A20008E1E04F5226701F11E0536F8020FF9F7E4
:107A30003DF8AE4227F8020FF7D1012384F8423A0D
:107A400094F8453A83F0010384F8433A94F8463AAF
:107A500083F0010384F8443AF8BD00BFA40000207D
:107A600070B5061D04460A4601463046FFF76CFD18
:107A700000B304F6B52531462846FFF72BFD014635
:107A80002846FAF709FD63793C2B13D1218904F6C6
:107A90005A2304F66622A4EB8404A4F5F75406489E
:107AA0001C3C33F8025F8D4204BF056844F8235044
:107AB0009342F6D170BD00BFA02C002070B5124BD0
:107AC0000C4693F82D3011465A1E012A0AD80F4E43
:107AD0006518AC4200D170BD304614F8011BFFF7A9
:107AE00087FAF6E7032B09D1094E6518AC42F2D0AC
:107AF000304614F8011BFFF7B3FFF7E72046BDE857
:107B00007040FAF7C9BC00BFA4000020E0050020C7
:107B1000880E0020B0F81C36B0F81E269B1A98B2CA
:107B20001B0444BF00F5806080B2003818BF0120FC
:107B30007047000008B50C4B93F82D305A1E012AEF
:107B400004D8BDE808400948FEF768BC032B04D1FF
:107B5000BDE808400648FFF7DDBFF9F7B9FB00387C
:107B600018BF012008BD00BFA4000020E0050020D0
:107B7000880E002010B500F6B5240B4620463C21A7
:107B80000222FFF77AFE01462046BDE81040FAF7D0
:107B900083BC00000F4B13B51A68D0F8483AD31ACB
:107BA000122B15D92023C0F8482A00F6B52400F678
:107BB000222001930090C82303223C212046F9F79C
:107BC000F1FC0146204602B0BDE81040FAF764BC63
:107BD00002B010BDA02C00207FB5224B04461A68CD
:107BE000D0F84C3AD31AC72B39D94FF480731E4DB5
:107BF000C0F84C2A2846ADF80830F8F781FE064652
:107C00001A48FBF70FFD01463046F8F799FF8DF84B
:107C10000A002846F8F774FEF8F78CFF95F8A930AB
:107C20008DF80B0028468DF80C30F8F77BFE8DF8A8
:107C30000D002846F8F76DFE072304F6B5240193DE
:107C400002AB3C218DF80E000093032241F20D039C
:107C50002046F9F7A7FC01462046FAF71DFC04B0C0
:107C600070BD00BFA02C00208C1D0020481E0020ED
:107C700030B504461E4B1F4887B01D68FBF7E0FC7B
:107C800040F6C312D4F8503AEB1A934203D894F951
:107C9000543A83422AD00023C4F8505A84F8540A34
:107CA0008DF80830F8F77CFF134D04226978ADF8A1
:107CB0000900ADF80B000DF10D00F9F7BFF8062231
:107CC000A9780DF11100F9F7DDF80F2304F6B524BA
:107CD000019302AB3C210093032241F20E032046A4
:107CE000F9F760FC01462046FAF7D6FB07B030BD35
:107CF000A02C0020481E00204800002070B5FAF794
:107D00005BF9FAF789FDFAF7B5F8FAF7A1F8FAF78F
:107D1000B7FC2449244801F0EDF80024FAF78AF86A
:107D2000FCF73AFBFAF7DEF88022204B204D5A7020
:107D3000C5E903441C70FAF7DFFA1E4B4FF4804686
:107D40001C70FAF707F84FF400421B4B04F1804413
:107D50005A6104F588341948FAF738F8FAF748F9FF
:107D600041F288306661FAF743F94CF250302661EF
:107D7000FAF73EF91248FAF70DFD284603F0FEF82F
:107D80004FF47A70FAF734F9FBF734FB0D48FAF741
:107D900083FDBDE870400C4B0C48B3F84810FAF76F
:107DA00031BE00BFCA0000205C1C0020420300203E
:107DB000481E00201400002000040140E09304004D
:107DC00030030020A41C002048000020891D002052
:107DD0004FF40042174B73B55A61FF21164803F068
:107DE000BBF9164C208023885B0612D5144E3579DA
:107DF0008DB108236A4600210F4803F0A9F8D6E99F
:107E00000402DDE900139A4208BF884201D0002332
:107E1000238002B070BD02236A462946064803F05B
:107E200097F8084BDA8BBDF800309A4218BF2580CE
:107E3000EFE700BF00040140481E0020D0050020ED
:107E400000030020480000200023034A1370034A67
:107E50001370034A13707047D9050020801E00205C
:107E6000380300200023024A1370024A137070473F
:107E7000D9050020801E002008B5437E203B042B3E
:107E80000FD8DFE803F0050E030B0F00FBF7F0FE41
:107E90000123064A1370064A137002E00122054BC3
:107EA0001A7008BDFBF79AFAF2E700BFD905002067
:107EB000801E002038030020034B1B78012B01D1CA
:107EC000FBF77ABE704700BFD90500202DE9F043CB
:107ED000074699B03D48FCF733F90646002860D0C4
:107EE0003B4B1C78002C5CD13A4B1B78022B54D1B5
:107EF0002546DFF8E4900DF10C084846ECB2FFF798
:107F000019FE40B14846FEF7B5FA0135522D08F882
:107F1000010BF2D12C4631482146F9F713F93048CC
:107F2000F9F70AF94FF00109DFF8A0802D4D98F814
:107F3000023028468DF8003095F8A43085F8A570F9
:107F40008DF805308DF806708DF80190F8F7D8FCA3
:107F50008DF802002846F8F7E5FC8DF80300284666
:107F6000F8F7EEFC204F8DF804000EB3184B1B7889
:107F7000CBB9234669461D4803AAFBF73BFD012305
:107F800018483B70F8F7EAFC1648F8F7F0FC0123B4
:107F900088F8033019B0BDE8F0830F48FEF7A6FA61
:107FA000C0E70024BEE769461048FFF785FFE6E713
:107FB0003B7803B9FEE769460C48FBF767FC2846A7
:107FC00087F80090F8F7CFFC2846DEE7641E002013
:107FD000801E00202B03002018000020F01D002030
:107FE000C81D00208C1D0020F90200202E1D00203D
:107FF00070B5CB78284DC3F3000385F8AA304B79D0
:108000000646C3F3801385F8AB30C8780C464008A9
:10801000F8F7E7FC85F8A60023792146C3F30003AF
:1080200085F8A73023791D48C3F3450385F8A830A8
:108030006379227903F03F035B0043EAD21385F8AA
:10804000A9301EB9BDE87040FBF754BBFBF791FBAC
:10805000A37803F0F003202B04D12046BDE8704044
:10806000FFF70ABFFFF7FEFE0D4B1B78022B12D164
:10807000A27904F119010B485208FFF71FFDA179FD
:1080800005F178004908F9F75DF805F15000BDE801
:108090007040F9F751B870BD8C1D0020AC1C002059
:1080A0002B0300201800002070B5054658B9194B65
:1080B00019491C78194803794BB1012C28D0BDE827
:1080C0007040F9F74FBA164B16491C78F2E7012CAD
:1080D000154B164E13D98A78C2F3C0025A70022289
:1080E0001A70E31E58425841FFF782FF3046F8F7F6
:1080F00001FC032C05D13046F8F7FFFB01E001221B
:108100001A7086F8A4500948BDE87040F8F7F0BB33
:1081100070BD00BFD6050020DC1E0020000300203B
:10812000D7050020371F0020641E00208C1D002072
:108130000A4B10B51A7904462AB1BDE81040014631
:108140001846FBF789BFFFF7C1FE054B2046BDE887
:1081500010405B221B7F0349FBF760BF0003002038
:10816000480000202E1D0020244B70B51A790546CA
:108170000E4632B1BDE870400A4601461846FCF78B
:10818000B7B95B231E4A1F49FBF732FF45BB1D48A9
:10819000FBF77AFA044628B31B491C48F9F76EFC32
:1081A00005F130011948C9B2F9F75CFC18491748C4
:1081B000F9F764FC204602F015FE01461348F9F772
:1081C0005DFC0A211148F9F74DFC012C06D0042C66
:1081D00011D0012428460F49FBF77AFF204670BDD5
:1081E0000748D5E72EB10C48FAF7BCFB0CB10224C6
:1081F000F0E70324EEE7002EF9D0F4E700030020B7
:10820000371F0020DC1E00204EB600080C000020A6
:1082100055B600088C1D0020891D0020024B1878DF
:10822000831E5842584170472B030020002370B52D
:108230009CB2A24200D870BD058886886C1C344070
:108240004688A6421EBFCE5C2D18AE7103F1010315
:1082500018BF0480ECE7B0F81E36B0F81C262DE9F4
:10826000F04FD21A93B2110444BF03F580639BB25E
:10827000E62B0446ADF5057D09D8012700F21C6602
:1082800004F2123804F20E35F9F722F818B90DF598
:10829000057DBDE8F08FFAF721F9294602464046F0
:1082A000FFF792F80028EFD094F813333E2B1CD040
:1082B000012394F81323212A09D141F20D01B4F8C6
:1082C00016238A4278D041F20E018A4277D0002BE1
:1082D000D6D004F6B52541462846FFF76BFA294665
:1082E00002463046FFF7A2FFCAE7B4F81633B3F5EB
:1082F000005F35D194F8983A002BD9D199461D46A4
:1083000004A804F2273E04F69F2C03601CF8012FFA
:10831000FF2A0DD0D1081EF8011002F0070241FA21
:1083200002F2D20742BF4FF0010907FA03F21543E8
:108330000133152BEAD1B9F1000F00D005600423F9
:1083400004F6B525CDE9000302223E2142F6FF7373
:108350002846F9F769F9294602463046FFF766FFD5
:10836000B4F816A3BAF1740FA2D14FF000090DF1C1
:10837000100B04F52A635846009304F21A32B4F83D
:1083800018330DF10E01ADF80E90FFF78BFABDF822
:108390000E3004F6B52502223E21CDE900B3284671
:1083A000534684F8989AFFF75BFA2946024630460E
:1083B000FFF73CFF4B467CE784F8457A60E784F89A
:1083C000467A5DE72DE9F047354B04461B78022BD2
:1083D0000CD00023A0F81E36A0F81C3690F86D3A99
:1083E00013B10A22B2FBF3F384F8983A2D4B93F8B9
:1083F0002D30032B51D12046FFF72DFF94F8422A50
:108400003AB10023204684F8423ABDE8F047FFF72E
:10841000C1BB94F8433A33B1204684F8432ABDE8FF
:10842000F047FFF7D9BB94F8448AB8F1000F06D0A3
:10843000204684F8443ABDE8F047FFF719BC1A4BD0
:108440001F68D4F8583AFB1A632B26D9254640F604
:10845000AB5AC4F8587A04F65C2604F1300995F852
:10846000702AAAB195F8713A0133DBB29A420BD85F
:1084700085F8718AD5F8743AFB1A534508D9204615
:108480003188FFF777FB03E085F8713A002BF1D0D4
:1084900008354D4506F10206E1D1BDE8F08700BF81
:1084A0002B030020A4000020A02C00202DE9F04F79
:1084B000DFF8A08287B098F80030012B00F20F811E
:1084C0000BB9F9F733FCA44DFFF718FC696CA3480E
:1084D000FAF746F80022A24B07241A809A704FF44C
:1084E0000062A04B5A614CF25030013CF9F7ECFCB1
:1084F000F9F77EFD14F0FF04F5D19B4802F082FEEF
:10850000122803D001209949FBF70AFE984B99499C
:108510001C80994B94481C80FBF712F87D20F9F7DA
:1085200067FD9648F9F77AFCFBF7C6FB95F820B093
:10853000BBF1200F00D9FEE795F82800AB8D904ED7
:1085400005280393696A95F8297095F82A30B07167
:1085500000D9FEE78B4A4FEA001E02EB001C52F8DE
:108560000E2002B9FEE7DCF808E09CF80C90B2603F
:10857000C6F810E09CF80420A246A446A646029243
:10858000F27186F80C9086F8D900B482039A42FA08
:108590000CF2D20707D5012202FA0CFA4EEA0A0AB7
:1085A0001FFA8AFE92460CF1010CBCF1060FEDD1C8
:1085B000DFF8CCC1BAF1000F01D0ACF814E0BCF880
:1085C00014E0BEF1000F00D1FEE7029AA2EB09020F
:1085D000D2B25A4528BF5A4605288CF8172000F019
:1085E000A680012800F2AA8007F1FF30C0B200F097
:1085F0009480022817D8581EC0B203280CD80C2A21
:1086000002D90C208CF817009CF81700904201D971
:108610008CF817203C4609E0122A84BF12238CF8FC
:1086200017300023F0E7052B28BF002322465448CB
:10863000F8F7DFFC002486F8D840B475FF26524BCB
:108640004F481E705E70FBF709F80146464802F07D
:10865000DEFD4E4B4E481C704E4B1C704E4B1C802A
:108660004E4B1C704E4B1C704E4B1C704E4B1C7076
:108670004E4B1C704E4B1C70FFF7E6FB4D4BB5F894
:108680004A201C704C4B95F840101C704B4B1C70D2
:10869000B5F84830F8F7F3F8B5F848104848F8F757
:1086A00028FC4848FBF744FD474B484893F82910FD
:1086B00000F02DFC4648FEF711FC4648FFF76CF928
:1086C0002948FAF7BDFF01464348FBF781FC434BBD
:1086D0001C80434B1C80FAF76DF888F80060FAF7AD
:1086E00073F8002800F0A0802B4A13880BB1013BDF
:1086F0001380284B1A4A19781388022922D12BB3E8
:10870000013B9BB213809278002A6BD0002B73D16F
:10871000F9F7CCFBF9F7D8FB6EE0022805D80C2A54
:1087200002D90C238CF817303C4600237EE77B1ED1
:10873000022BFAD8082AF7D90823F3E71048F8F7EC
:10874000F3FB77E7002BDBD1C723DBE740F2F31322
:10875000D8E700BFD01C00204800002010000020F7
:10876000D205002000080140481E002057B600082E
:10877000CE0500204C000020D00500200003002082
:108780004403002098B90008D11C0020D80500201F
:108790008C1D00202B0300202E0300202C03002022
:1087A00028030020290300202A030020D7050020E9
:1087B000D60500203B0300203A030020740500206A
:1087C0006C1E0020641E0020A40000205C1C002001
:1087D000E0050020880E0020420300207C1E0020BF
:1087E0007E1E00200229874840F089800BB9F9F7E6
:1087F0005DFB4FF400634361834C2388002B00F042
:108800008580013B9BB281482380FBF791FA804829
:10881000FAF716FF01467F48FBF7DAFB23881BB9FE
:108820007D497E48F9F72AF97D4D7E4C297800294B
:108830006FD0022900F0A08023889BB2FBB12B7877
:10884000032B40F0A78023881E0702D50023238036
:108850002B7023889BB293B12388190648BF2388C5
:1088600023885A0648BF238823886F4A1B0748BFBE
:108870002388002313706D4A23802B7013706C4B78
:108880001A7802F0FF06002A00F014820020187007
:10889000664B1F7807F1FF3CDCF1000848EB0C0841
:1088A000002F00F09080FFF7FFFB0023614A012FAB
:1088B000137205D8604A1377D38313625F4A13702B
:1088C0005F4C2278012A00F2CB80012F15D95D4F31
:1088D00097F8A8303E2B7FD85B4997F8A770887D22
:1088E000002F40F08780834271D0CA7D8B759A42F9
:1088F00098BF0023B04698BF8B750026BAE04FF4AE
:1089000080524261002B7FF477AF03E740F2E733F8
:1089100079E74B4B1B7843B14B4A937DD07D0133B4
:10892000DBB29842937598BF91754748FAF796FE67
:1089300000260146364802F06AFCF9F73DFA0D219F
:1089400001230DF1170232488DF8176002F094FAF6
:10895000FF212F4802F0FAFB2D4802F025FC7D2074
:10896000F9F746FB01232B702F4B1E702F4B1E7007
:10897000364B1E8026805FE73548FBF71BFC2D4BEE
:10898000187AFFF7D5FB03232B7000232F4A13809F
:10899000238051E7012B7FF45CAF238858067FF5D5
:1089A00058AF214B002019782080B1FA81F1490994
:1089B000FFF7DAFB1D4B032818707FF44AAF144809
:1089C00002F02AFC45E70122224B1A706DE722488B
:1089D000017841F0010101702049002A40F08B80AC
:1089E0003F2B4FF001000A7028BF03221A4B207062
:1089F0001A7038E083427FF478AF1748017841F06D
:108A00000201E8E7000801407C1E0020000300206E
:108A1000481E00204203002061B600080C00002020
:108A2000D8050020D0050020D7050020D60500205D
:108A3000390300206C1E0020E0050020880E002075
:108A40002B0300208C1D002044030020CE050020B5
:108A5000D11C0020641E0020280300202C030020CD
:108A6000012F7FF64AAF7B4BB3F84C207A4B1A802C
:108A700002232B702378002B40F0A181B8F1000F66
:108A800000D02B707549734A0B78B2F84E20013331
:108A9000DBB293420B70724A0ADB937DD07D0133C7
:108AA000DBB2984298BF0023937500230B702B70A4
:108AB00092F8D830002B44D0B2F8DC30B2F8DA109B
:108AC00001339BB29942A2F8DC303AD80023062148
:108AD000A2F8DC30908A92F8D9300133DBB2062B51
:108AE00028BF002340FA03F7FF0726D55D48190188
:108AF0004158E9B9FEE70B785B4801330278DBB2F5
:108B00000B706AB9534A92F850209A42ABD8574B2F
:108B10001B78032B06D10223237001230370A2E7E5
:108B20000522F2E7531EDBB29A420B70F3D99AE7A3
:108B300082F8D93000232B7003E0013911F0FF01D6
:108B4000CBD100224A4B1A702278002A00F03181E2
:108B50001EB901221A7002232B704648FAF73EFD17
:108B60002378022B02D00022434B1A70434A138809
:108B700013B9384BB3F84A30013B9BB2138013B999
:108B80003F48F7F700FF3E48F7F7B1FE2378022B86
:108B90000BD03B48F7F75BFE237833B9FFF762F958
:108BA0000123384A1370384A1370384E3046F9F7AB
:108BB0005BFE73783648012B01BF00227270344A85
:108BC0005371FBF7DFF8FBF7F5F80128064607D0ED
:108BD00002282FD005222F4B1A7007B0BDE8F08F66
:108BE0001C4F2B48FBF784F8B7F848302A4A03EBB0
:108BF000830303EB83039B0028481380F9F7B2FE3D
:108C000041F28833B7F84810154AB3FBF1F3A2F8E4
:108C1000DA3000234FF4805182F8D860A2F8DC30BB
:108C20001F4A11614FF4006151611E4A2370967012
:108C30002B70CFE70A4B93F8D930052B08D81A4A86
:108C4000D25C1A4B83F819210122194B1A70C1E723
:108C5000FEE700BF480000202E030020290300206B
:108C60004403002098B900082A03002028030020AC
:108C700074050020481E0020641E00207E1E002077
:108C80008C1D0020D9050020801E0020A41C00207F
:108C9000000300203B03002044000020891D002029
:108CA00000080140D205002078B90008A400002087
:108CB000380300204649474A0B781BB1013BDBB221
:108CC0000B7013B11378002B34D00024424D43486D
:108CD00095F82810147000F045F9414B1B78022BD1
:108CE00046D1404E404896F80090F7F709FE0746F7
:108CF0003D48F7F717FE23464A463C49CDE9007048
:108D0000364800F047FC3548FBF7ACFB2346327889
:108D100037493848FDF73CFB23463278344936481A
:108D2000FEF774FE95F8263095F833202F49334826
:108D3000FBF760FA294800F03DFD2E48FEF7A6FA41
:108D40002D48FFF73FFB2E4B1B78002B3FF445AF20
:108D50002C48FAF743FC4FF400622B4B1A614FF496
:108D600080521A61FAF72AFB012388F8003034E7B1
:108D7000264B1B78C3B16FF07E03009301231B4980
:108D80001A461648019400F005FC144800F001F959
:108D9000012317491A461748FDF7FAFA0123144927
:108DA0001A461548FEF732FE95F82620134B5A70E6
:108DB000C0E72B7813F0FD0F3FF4CFAED3E6144B92
:108DC0001B88002B7FF4BDAE124A23701370B2E6ED
:108DD0003B0300203A030020A40000205C1C00207C
:108DE0002B030020740500208C1D0020AC1C0020EB
:108DF000801C0020E0050020880E0020D11C0020EF
:108E000038030020481E0020000801402A030020EB
:108E10002E0300202903002008B5FFF747FBFCE7DD
:108E200010B51F4B1F4A204C1A60204602F01CF858
:108E30001E4B1F4A23601F4B1F4C1A605A619A62D7
:108E4000DA631A651D4A20465A669A671C4AC3F8B7
:108E50008C2000F043F8002240F2FF11194B2360F0
:108E6000194BC3F8E824C3F8EC14184B40F2FF3157
:108E7000C3F81C26C3F8502A7D2283F8542A144ACA
:108E8000C3F820161068516803F65C2403C4906888
:108E90002060D068128AC3F8680AA3F86C2A10BD53
:108EA000300300206CB60008481E00207CB6000885
:108EB000ECB500088C1D00205C1C0020D4B5000817
:108EC000E0B50008FCB60008E0050020880E002090
:108ED000F4B30008704700207047000010B5044646
:108EE000034B012140F8043BF7F75EFC204610BD20
:108EF00090D1000838B524220D46FF2300210446F6
:108F000003618182104402F0F9F9E56038BD38B59B
:108F10000D46017C0446A94215D0012918D002292A
:108F200012D011B903685B6898470023012D637460
:108F3000257413D0022D0ED02DB923685B68012152
:108F400020469847607438BD0368DB680021EBE772
:108F500003689B68FAE72368DB68F0E72368294623
:108F60009B68EDE70430F7F72DBC037C10B5012BAF
:108F70000ED100F1160301F10C0251F8044B91429D
:108F800043F8044BF9D10A881A8040F20113438256
:108F900010BD037C012B0BD148F281134FF4014229
:108FA000C3820023C0E90632038440F201134382E6
:108FB0007047F0B5054689B008880C4616461F462E
:108FC000F7F765FD9DF806308DF8050023F00703DF
:108FD000C0F30220034360888DF80630F7F757FD91
:108FE0009DF8063000F01F0203F0070343EAC203B6
:108FF0008DF806309DF80730C0F3451023F03F038D
:109000000343A0888DF80730F7F741FD9DF807303E
:1090100000F0030203F03F0343EA82138DF80730A8
:10902000C0F387038DF808309DF80930C0F3802025
:1090300023F001030343E0888DF80930F7F727FD9B
:109040009DF8093000F07F0203F0010343EA420378
:109050008DF809309DF80A30C0F3C31023F00F03D8
:10906000034320898DF80A30F7F711FD9DF80A3087
:1090700000F00F0203F00F0343EA02138DF80A30E9
:109080009DF80B30C0F3061023F07F030343608983
:109090008DF80B30F7F7FBFC9DF80B3000F0010268
:1090A00003F07F0343EAC2138DF80B30C0F347038C
:1090B0008DF80C309DF80D30C0F3412023F00303F0
:1090C0000343A0898DF80D30F7F7E1FC9DF80D30D2
:1090D00000F03F0203F0030343EA82038DF80D30F2
:1090E0009DF80E30C0F3841023F01F030343E08982
:1090F0008DF80E30F7F7CBFC9DF80E3000F007022C
:1091000003F01F03C0F3C70043EA42138DF80F00BA
:10911000208A8DF80E30F7F7BAFC9DF811308DF8E3
:10912000100023F00703C0F302200343608A8DF888
:109130001130F7F7ACFC9DF8113000F01F0203F07E
:10914000070343EAC2038DF811309DF81230C0F3D3
:10915000451023F03F030343A08A8DF81230F7F740
:1091600096FC9DF8123000F0030203F03F0343EA3F
:1091700082138DF81230C0F387038DF813309DF8F9
:109180001430C0F3802023F001030343E08A8DF8FC
:109190001430F7F77CFC9DF8143000F07F0203F0E8
:1091A000010343EA42038DF814309DF81530C0F3F3
:1091B000C31023F00F030343208B8DF81530F7F70E
:1091C00066FC9DF8153000F00F0203F00F0343EA30
:1091D00002138DF815309DF81630C0F3061023F0F9
:1091E0007F030343608B8DF81630F7F750FC9DF832
:1091F000163000F0010203F07F0343EAC2138DF83A
:109200001630C0F347038DF817309DF81830C0F3BF
:10921000412123F003030B43A08B8DF81830F7F79F
:1092200036FC9DF8183000F03F0203F0030343EAD8
:1092300082038DF818309DF81930C0F3841023F0A4
:109240001F030343E08B8DF81930F7F720FC9DF8DE
:10925000193000F0070203F01F0343EA42138DF8B0
:10926000193040F2A953218C628C99428CBF0121A4
:109270000021C0F3C7009A428DF81A0088BF41F060
:1092800002010EB141F004010FB141F008010F23BA
:109290008DF8043000238DF81C302B688DF81B10DE
:1092A000192228461B6801A9984709B0F0BD0000A3
:1092B00030B5054689B008880C46F7F7F5FB9DF8F0
:1092C00008308DF8070023F00703C0F302200343A2
:1092D00060888DF80830F7F7E7FB9DF8083000F05C
:1092E0001F0203F0070343EAC2038DF808309DF81C
:1092F0000930C0F3451023F03F030343A0888DF8E5
:109300000930F7F7D1FB9DF8093000F0030203F0B4
:109310003F0343EA82138DF80930C0F387038DF8C9
:109320000A309DF80B30C0F3802023F00103034383
:10933000E0888DF80B30F7F7B7FB9DF80B3000F0A5
:109340007F0203F0010343EA42038DF80B309DF8DE
:109350000C30C0F3C31023F00F03034320898DF8B2
:109360000C30F7F7A1FB9DF80C3000F00F0203F072
:109370000F0343EA02138DF80C309DF80D30C0F353
:10938000061023F07F03034360898DF80D30F7F753
:109390008BFB9DF80D3000F0010203F07F0343EAE0
:1093A000C2138DF80D30C0F347038DF80E309DF8D1
:1093B0000F30C0F3412023F003030343A0898DF84D
:1093C0000F30F7F771FB9DF80F3000F03F0203F00C
:1093D000030343EA82038DF80F309DF81030C0F389
:1093E000841023F01F030343E0898DF81030F7F752
:1093F0005BFB9DF8103000F0070203F01F03C0F381
:10940000C70043EA42138DF81100208A8DF810300E
:10941000F7F74AFB9DF813308DF8120023F007038D
:10942000C0F302200343608A8DF81330F7F73CFB4A
:109430009DF8133000F01F0203F0070343EAC20354
:109440008DF813309DF81430C0F3451023F03F031E
:109450000343A08A8DF81430F7F726FB9DF81430EB
:1094600000F0030203F03F0343EA82139DF8162045
:109470008DF81430C0F387038DF8153022F0010207
:10948000C0F380231343E08A8DF81630F7F70CFB06
:109490009DF8163000F07F0203F0010343EA420317
:1094A0008DF816309DF81730C0F3C31023F00F036A
:1094B0000343208B8DF81730F7F7F6FA9DF8173035
:1094C00000F00F0203F00F0343EA02138DF8173088
:1094D0009DF81830C0F3061023F07F030343608B20
:1094E0008DF81830F7F7E0FA9DF8183000F0010217
:1094F00003F07F0343EAC2139DF81A208DF8183059
:10950000C0F347038DF8193022F00302C0F3412362
:109510001343A08B8DF81A30F7F7C6FA9DF81A306E
:1095200000F03F0203F0030343EA82038DF81A3090
:109530009DF81B30C0F3841023F01F030343E08B1E
:109540008DF81B30F7F7B0FA019B0DF1060103F01F
:109550007F420F4B134301939DF81B3000F007022D
:1095600003F01F03C0F3C70043EA42138DF81C0049
:10957000172200208DF81B30F7F702FB2B688DF8BF
:109580001D001A2228461B6801A9984709B030BD62
:10959000C81816002DE9F04700F124071E460446BE
:1095A0003B469DF920A09DF82490904601F12402AD
:1095B00051F8040B914243F8040BF9D1251D3946AB
:1095C0002846F7F723F9E1684B7966B1042B77D881
:1095D000DFE803F07C76345C030000264FF00423C0
:1095E000B046C4E90933E3681D796B1E0B2B07D81D
:1095F0005046F7F722FA0435EDB204EB45056884CE
:10960000E3681D7B6B1E0B2B07D84846F7F730FA33
:109610000435EDB204EB45056884637C002B55D01E
:10962000237C012B46D013F0FD0F4FD13346424629
:1096300039462046BDE8F047FFF7BBBC4FF0780C39
:1096400001F1130304F1220001F11F0513F9012FA9
:10965000C2EB822292FBFCF2AB4202F5806220F860
:10966000022FF3D140F2FF7504F13A02233113F8CF
:10967000010F48B102280CBF28464FF48060994280
:1096800022F8020FF3D1AEE70120F8E74FF4806132
:1096900004F1220304F1460223F8021F9342FBD196
:1096A00002212846F7F7D0F80023103004EB4000E1
:1096B000838098E739462046BDE8F047FFF7F8BDBC
:1096C000042B90D813F0FD0F8DD0E9E7BDE8F087AB
:1096D00030B54B7B0546032B0C4685B042D191F942
:1096E0000000F7F727FA8DF8030094F90100F7F767
:1096F00021FAA3788DF804008DF80530E378207BFB
:109700008DF8063023798DF80730F7F70BFA8DF8CE
:10971000080094F90600F7F7DFF98DF8090094F9CD
:109720000700F7F707FA237A8DF80A008DF80B3057
:10973000637A0DF102018DF80C3040F6C843ADF8A4
:10974000003014230B2200208DF80230F7F718FAAE
:109750002B688DF80D000E22694628461B68984735
:1097600005B030BD022B03D1FF238DF80330BCE7D9
:1097700091F90000F7F7DEF98DF80300FF20B8E754
:10978000837C10B5044633B1F9F740F8E37C1BB194
:109790000023A082E37410BDA28A801A80B2B0F5C3
:1097A0007A6FF8D92046A37404F11601BDE8104081
:1097B000FFF78EBF427C22B1037C012B01D1FFF762
:1097C000DFBF704710B590B01422002108A801F047
:1097D00095FD1422002101A801F090FD02244FF410
:1097E00080330122CDE90D43CDE906234FF48013E8
:1097F00006A80A920F9300F01FFD08B172B6FEE7AB
:109800000F23CDE901344FF480630390CDE9043098
:10981000214601A800F0D8FE08B172B6FEE710B0EC
:1098200010BD000007B500F0A5F8FFF7CBFF0C4B0B
:109830009A6942F020029A619A6902F0200201922C
:10984000019A9A6942F004029A619B6903F0040349
:109850000093009B03B05DF804EBFFF7DDBA00BF97
:10986000001002400E4B82B09A6942F001029A61E8
:109870009A6902F001020092009ADA6942F080527D
:10988000DA61DB69074A03F080530193019B536857
:1098900023F0E06343F00073536002B0704700BFF1
:1098A0000010024000000140FEE7FEE7FEE7FEE791
:1098B000FEE7704770477047F8F796BF70470000A3
:1098C000FFF7FCFF0B480C490C4A002302E0D45878
:1098D000C4500433C4188C42F9D3094A094C0023FC
:1098E00001E013600432A242FBD301F03DFDFFF71B
:1098F00099FF70470000002028000020F4D10008E4
:1099000028000020E82C0020FEE7704710B54FF03B
:10991000FF320024044B1A611C61DA60DC60FFF73F
:10992000F4FF204610BD00BF0010024038B50E4BBA
:1099300005461A784FF47A73B3FBF2F30B4A1068BA
:10994000B0FBF3F000F070F8044658B90F2D09D8B9
:10995000024629464FF0FF3000F036F82046044B0F
:109960001D6038BD0120FCE7200000201C00002005
:1099700024000020074A08B51368032043F01003B1
:10998000136000F00FF80F20FFF7D0FFFFF76AFF1A
:10999000002008BD00200240014B1868704700BF3E
:1099A000A02C002007490302CA6803F4E06322F4F4
:1099B000E0621204120C134343F0BF6343F400331C
:1099C000CB60704700ED00E0154B30B5DC68C4F3A8
:1099D0000224C4F10703251D042B28BF0423062DF0
:1099E0004FF0FF3594BF0024033C05FA03F321EA4E
:1099F0000303A54022EA0502A340002843EA02032C
:109A0000ACBF00F16040074A4FEA0313DBB2ABBFC3
:109A100000F5614000F00F0080F80033135430BDB2
:109A200000ED00E014ED00E00138B0F1807F0BD2D2
:109A30004FF0E023F021054A586182F823100020FE
:109A4000072298611A6170470120704700ED00E01D
:109A5000114AD36813F0100305D01049CB6943F0C5
:109A60000203CB611023D268500706D50B4943F09F
:109A70000403CA6942F00102CA61074AD169C907F1
:109A800008D50648C16941F00401C161D16921F0DE
:109A90000101D161D360704700200240A82C002052
:109AA000064B186910F0800007D0054A5A6002F191
:109AB00088325A601869C0F3C01070470020024015
:109AC00023016745034A0020136943F080031361B3
:109AD000704700BF0020024070B50546FFF75CFFED
:109AE0000646114CE368D80712D4E368990644BFD0
:109AF0002023E360E368DA0606D4E369DB0703D4D6
:109B0000E06810F0040007D0FFF7A2FF012003E097
:109B10006B1CE7D00DB9032070BDFFF73DFF801B24
:109B2000A842DFD9F7E700BF002002400022064B21
:109B3000DA61064B1A6942F002021A6158611A6929
:109B400042F040021A617047A82C00200020024019
:109B50002DE9F041264F05463B7E8846012B44D037
:109B600001243C7603684CF25030022B1AD1FFF7E7
:109B7000B3FF20B1012000233B76BDE8F0811D4CEE
:109B8000F86123694CF2503043F0040323612369E8
:109B900043F040032361FFF79FFF236923F0040391
:109BA0002361E8E7FFF798FF0028E3D14FF0FF3388
:109BB000C8F800302046AE680E4CD5E9023203EBFF
:109BC0008223B342D7D93046FFF7B0FF4CF2503072
:109BD000FFF782FF236923F00203236110B1C8F865
:109BE0000060C8E706F58066E7E70220C5E700BF2A
:109BF000A82C002000200240016800224B6913F4C9
:109C0000806310D06FF480634B612023026380F87F
:109C10003D3080F83E20036C80F83C2043F0040384
:109C2000036401207047184670472DE9F846064640
:109C30000F4691461D464FEA114A3368BAF1010FAB
:109C40000CBF5C699C6927EA0404A4B2B4FA84F4EA
:109C50006409A14501D0002025E06A1CEED0FFF781
:109C60009BFE089BC01AA84201D8002DE5D133689D
:109C7000BAF1010F0CBF5B699B6927EA03039BB232
:109C8000B3FA83F35B099945D7D100232022012041
:109C9000336386F83D2086F83E30326C86F83C30DF
:109CA00042F020023264BDE8F8862DE9F041044616
:109CB0000F46164698462568686927EA000080B274
:109CC000B8B16B695A0516D52B68202243F400738E
:109CD0002B606FF480636B610023236384F83D2065
:109CE00084F83E30226C42F004020120226484F8A1
:109CF0003C30BDE8F081731CDED0FFF74DFEA0EBD9
:109D00000800B04201D8002ED5D123685A6927EA4D
:109D1000020292B2002ACED000232022236384F8CC
:109D20003D2084F83E30226C42F02002DDE770B521
:109D300004460D46164623685B691B0601D50020C4
:109D400070BD2046FFF758FFC8B96A1CF3D0FFF773
:109D500023FE801BA84201D8002DECD123685B694B
:109D600013F08003E7D12022236384F83D2084F898
:109D70003E30226C84F83C3042F020022264012004
:109D8000DEE770B504460D46164623685B695B073F
:109D900001D5002070BD2046FFF72EFFC8B96A1C10
:109DA000F3D0FFF7F9FD801BA84201D8002DECD1BC
:109DB00023685B6913F00403E7D12022236384F84E
:109DC0003D2084F83E30226C84F83C3042F0200282
:109DD00022640120DEE7000070B5044608B90120C6
:109DE00070BD90F83D3003F0FF021BB980F83C20B5
:109DF000F8F750FC242384F83D3023681A6822F0D9
:109E000001021A601A6842F400421A601A6822F4C9
:109E100000421A6000F074FC3F4B65689D4294BF9D
:109E20003E4B3F4B98428CBF00230123002BD6D1E1
:109E3000394E3C4BB542B0FBF3F388BF4FF49676F6
:109E40002268516821F03F0141EA030182BF734358
:109E50004FF47A76B3FBF6F35160116A013321F0C7
:109E60003F010B431362D169431E2B4821F44F413C
:109E7000854221F0FF0132D86D00B3FBF5F340F6C7
:109E8000FC700133034242D0C3F30B031943D16189
:109E90001168D4E9073021F0C00103430B4313607C
:109EA0009168D4E9030321F40341034321F0FF0146
:109EB0000B439360D168D4E9053021F0FF010343DF
:109EC0000B43D3601368002043F001031360202389
:109ED000206484F83D30206384F83E0080E7A06869
:109EE00050B905EB4505B3FBF5F30133C3F30B03A1
:109EF0007BB143F40043C9E719206843B3FBF0F397
:109F00000133C3F30B0323B143F44043BEE70423FF
:109F1000BCE70123BAE700BFA08601007F841E00D2
:109F2000FF083D0040420F002DE9F043044685B094
:109F300098460D4691460C9FFFF72EFD94F83D3054
:109F40000646202B04D00225284605B0BDE8F08344
:109F500000901923012220465B49FFF766FE002886
:109F6000F1D194F83C30012BEDD00123216884F825
:109F70003C300B68DA075EBF0B6843F001030B60EF
:109F80000B6823F400630B60212384F83D30102319
:109F900084F83E3000232364A4F82A80638DC4F83B
:109FA00024902385494BE362E36A082B04D0012BFC
:109FB00002D013F5803F04D10B6843F480730B602B
:109FC00002E0236B122BF7D000223B464FF0011129
:109FD00020460096FFF729FE226838B11368DB059A
:109FE00044BF4FF4007323640125ADE72369B3F543
:109FF000804F21D105F0FE05156133463A462046D3
:10A000003349FFF752FE05460028EDD1236803903F
:10A010005A6903929B690393039B238DF3B92168CB
:10A020000A6842F400720A60202284F83C3084F806
:10A030003D2084F83E3087E7EB1103F0060343F040
:10A04000F0031361204633463A462249FFF72DFEBE
:10A050000028C9D12368EDB21D61CEE732463946EA
:10A060002046FFF764FE40B1236C042BBCD122686C
:10A07000136843F400731360B6E7636A20681A46F6
:10A0800012F8011B01616262628D013A92B262852F
:10A09000228DD0F814C0511E89B21CF0040F218506
:10A0A0000AD049B15978023301616362638D023A83
:10A0B000013B9BB263852285324639462046FFF735
:10A0C00060FE0028A9D0CFE7020010000000FFFFCB
:10A0D00002000100080001002DE9F04F044685B0A0
:10A0E0001F4688469246FFF757FC94F83D300546D8
:10A0F000202B03D0022005B0BDE8F08F009019237B
:10A10000012220464A49FFF790FD0028F2D194F839
:10A110003C30012BEED0012384F83C30236800262C
:10A120001A68DFF80CB1D20758BF1A6808F0FE08A9
:10A130005CBF42F001021A601A6822F400621A60E1
:10A14000242384F83D303B4B2664E36222684FF0C1
:10A1500001111368204643F4807313603B460022CC
:10A160000095FFF762FD236838B11B68DB0502D557
:10A170004FF4007323640320BDE7C3F81080FFF79A
:10A180000BFC4FF0A009054623685A695B69C2F3CE
:10A190004002C3F3802394F83D10A02901D013435B
:10A1A0001DD04FF02009236884F83D905A6912F0C1
:10A1B000020F1A6842F400721A6025D0002203923E
:10A1C0005A69204603929B6901220393039B184915
:10A1D00019230095FFF729FD88B101208BE7FFF7D0
:10A1E000DBFB401BB84200D80FB984F83D902368D0
:10A1F0005A695B69C2F34002C3F38023CBE784F85A
:10A200003D9084F83C0076E76FF4806259465A61CD
:10A210002046192301220095FFF707FD0028DCD115
:10A220000136564592D384F83D9084F83C00D4E73B
:10A23000020010000000FFFF2DE9F341054638B38E
:10A240000368DB0710D42B689F075ED42B681907BF
:10A2500000F195802B685A0700F1C180E869002859
:10A2600040F02C81002029E0904C636803F00C033F
:10A27000042B07D0636803F00C03082B0AD1636832
:10A28000DE0307D523689C03DDD56B68002BDAD18C
:10A29000012013E06B68B3F5803F12D1236843F4CB
:10A2A00080332360FFF778FB064623689803CAD4FF
:10A2B000FFF772FB801B6428F7D9032002B0BDE8CA
:10A2C000F0819BB9236823F480332360236823F44F
:10A2D00080232360FFF760FB064623689903B2D50D
:10A2E000FFF75AFB801B6428F7D9E6E7B3F5A02FE8
:10A2F000236803D143F480232360CFE723F4803322
:10A300002360236823F48023CBE7684C636813F051
:10A310000C0F07D0636803F00C03082B10D163689F
:10A32000DA030DD423689B0702D52B69012BAFD12B
:10A3300023686A6923F0F80343EAC203236085E7D0
:10A340002A695B4B6AB101221A60FFF725FB0646BA
:10A3500023689F07ECD4FFF71FFB801B0228F7D967
:10A36000ABE71A60FFF718FB0646236898077FF5EE
:10A370006DAFFFF711FB801B0228F6D99DE7AA6994
:10A380004A4E4B4BE2B10122C3F88024FFF704FB95
:10A390000446736A9B070DD54FF4FA52454B1B6870
:10A3A000B3FBF2F3019300BF019B5A1E0192002BF5
:10A3B000F9D14FE7FFF7F0FA001B0228E9D97CE753
:10A3C000C3F88024FFF7E8FA0446736A9F077FF515
:10A3D00041AFFFF7E1FA001B0228F6D96DE7334CD5
:10A3E000E369D80024D40127E36943F08053E36193
:10A3F000E36903F080530093009B2F4E3368D90527
:10A4000018D5EB68012B26D1236A43F001032362A0
:10A41000FFF7C2FA41F288380646236A9B073FD508
:10A42000002F3FF41BAFE36923F08053E36115E78E
:10A430000027E2E7336843F480733360FFF7ACFA38
:10A4400080463368DA05DCD4FFF7A6FAA0EB0800F3
:10A450006428F6D931E7ABB9236A41F2883823F092
:10A4600001032362236A23F004032362FFF794FAB3
:10A470000646236A9807D3D5FFF78EFA801B40451E
:10A48000F7D91AE7052B236A03D143F004032362AB
:10A49000BAE723F001032362236A23F00403B6E73B
:10A4A000FFF77AFA801B4045B7D906E70010024053
:10A4B000000042421C000020007000402A4C6368EB
:10A4C00003F00C03082B3ED00022284B02281A660A
:10A4D0002CD1FFF761FA06462368990120D42B6A34
:10A4E000B3F5803F05D16268A96822F400320A43BF
:10A4F0006260696A62680B4322F47412134301229A
:10A5000063601A4B1A66FFF747FA054623689A01FB
:10A510003FF5A8AEFFF740FA401B0228F6D9CCE67B
:10A52000FFF73AFA801B0228D6D9C6E6FFF734FABD
:10A53000054623689B017FF595AEFFF72DFA401B7A
:10A540000228F6D9B9E601283FF4B8AE63682A6A52
:10A5500003F4803191427FF49BAE6A6A03F4701376
:10A5600093423FF47FAE93E6001002400000424267
:10A570000F4A536803F00C01042914D0082914D1A0
:10A580000C48C3F38341DB03405C09D553680A4A96
:10A59000C3F340435043094AD35CB0FBF3F0704728
:10A5A000074B58437047044870470648704700BF40
:10A5B00000100240B8D10008001BB700C8D1000845
:10A5C00000093D0000127A002DE9F0410D460446D5
:10A5D00010B90120BDE8F081444A136803F0070375
:10A5E0008B4228D321688E0730D4CA0743D43F4A10
:10A5F000136803F00703AB4265D822683C4D12F0A4
:10A60000040F6CD1130706D56B68226923F46053DD
:10A6100043EAC2036B60FFF7ABFF6B68354AC3F3D5
:10A620000313D35CD840344B1860344B1868FFF7E1
:10A630007DF90020CEE7136823F007030B43136076
:10A64000136803F007038B42C3D1CBE7284B11F00B
:10A65000040F1EBF5A6842F4E0625A60080742BF06
:10A660005A6842F460525A605A68A06822F0F002B8
:10A6700002435A60B9E762681D4E012A33681AD155
:10A6800013F4003FA5D0736841F2883823F0030328
:10A6900013437360FFF780F907467368626803F03D
:10A6A0000C03B3EB820FA2D0FFF776F9C01B404535
:10A6B000F3D903208EE7022A02D113F0007FE1E7ED
:10A6C00013F0020FDEE7136823F007032B43136038
:10A6D000136803F00703AB427FF47BAF8DE76B6831
:10A6E000E16823F4E0630B436B608BE700200240DA
:10A6F00000100240A0D100081C000020240000200F
:10A70000044B054A5B68C3F30223D35C034A106819
:10A71000D840704700100240B0D100081C00002053
:10A72000224B98420BD103F58433DA6842F00402DD
:10A73000DA60DA6822F004020020DA6070471C4B0D
:10A74000984209D103F58233DA6842F00802DA60F0
:10A75000DA6822F00802EFE7164B984209D103F5B8
:10A760008033DA6842F01002DA60DA6822F0100210
:10A77000E2E7114B984209D103F57C43DA6842F0D5
:10A780002002DA60DA6822F02002D5E70B4B98420B
:10A7900009D103F57843DA6842F04002DA60DA68FA
:10A7A00022F04002C8E70120704700BF00080140C6
:10A7B000000C01400010014000140140001801404D
:10A7C0002DE9F04F0D680446C5F30F2595FAA5F263
:10A7D0004FF00F0AB2FA82F203274FF0040C4FF049
:10A7E000011E40F2011835FA02F001D1BDE8F08FE8
:10A7F000012393402B4265D0072A88BFA2F10803AA
:10A800004E688ABF0EFA03F308FA02F343F080633E
:10A81000082E0ED1E0684FEA132920EA132B99FA8B
:10A82000A9F9B9FA89F9086900FA09F040EA0B00B8
:10A83000E0604FEA136954F8090093FAA3FBBBFAEE
:10A840008BFB4FEA8B0B0AFA0BFB20EA0B0093FA07
:10A85000A3FBBBFA8BFB4FEA8B0B06FA0BF6064306
:10A8600044F80960486820F0080001282AD1886867
:10A8700093FAA3FBBBFA8BFB4FEA8B0B07FA0BFB9C
:10A8800026EA0B0693FAA3FBBBFA8BFB4FEA8B0B72
:10A8900000FA0BF0304344F80900CE6893FAA3FBAA
:10A8A000BBFA8BFB4FEA8B0B0CFA0BFB20EA0B0B72
:10A8B00093FAA3F3B3FA83F39B009E4046EA0B0698
:10A8C00044F8096001328EE7144B1A6842F0010225
:10A8D0001A601A689207FCD55A6822F003025A607F
:10A8E0005A6812F00C0FFBD11A6822F080721A60BD
:10A8F000186810F00070FBD158601A6822F45022DA
:10A900001A601A6822F0F80242F080021A60986019
:10A910005A6A42F080725A62704700BF00100240CB
:10A92000034B044A5B68C3F30313D35CD8407047FE
:10A9300000100240A0D10008034B044A5B68C3F337
:10A940000223D35CD840704700100240B0D1000809
:10A95000034B044A5B68C3F3C223D35CD8407047FF
:10A9600000100240B0D10008094A5368DB0341BF20
:10A9700053680848C3F34043013348BFB0FBF3F0CA
:10A98000536858BF0448C3F38343023358437047A6
:10A9900000100240001BB70000093D00064B5B6839
:10A9A00003F00C03042B03D0082B03D1FFF7DCBF0B
:10A9B000024870470248704700100240001BB70071
:10A9C00000127A0010B50146FFF7E8FF0860FFF7B4
:10A9D000A7FF48600446FFF7AFFF88602046FFF7F7
:10A9E000B7FFC86010BD02460068F0B510F0400027
:10A9F00023D1D1E900373B438F684D693B43CF6892
:10AA000016683B430F690C6A3B438F692B433B43FA
:10AA1000CF6926F47F463B43234326F0BF063343EA
:10AA200013605368B4F5005F23F0040343EA154351
:10AA3000536001D18B8C1361F0BD0120FCE7000055
:10AA40001A4A036890420AD0B0F1804F07D0A2F5AD
:10AA50009432904203D002F58062904215D14A6848
:10AA600023F070031343114A90420AD0B0F1804F93
:10AA700007D0A2F59432904203D002F58062904252
:10AA800003D1CA6823F44073134303608B68C36225
:10AA90000B888362054B984204BF0B6903634369CB
:10AAA00043F0010343610020704700BF002C0140C8
:10AAB000B1F5807F30B500F0908005D801292AD00B
:10AAC000102958D0012030BDB1F5805FFAD1036A5A
:10AAD000156823F480530362036A4468C16923F450
:10AAE000005321F4E64141EA0521156943EA0533A3
:10AAF000556823F4805343EA0533504DA84204BF00
:10AB0000956924F48044D26808BF44EA85144460FF
:10AB1000C16102642CE0036A156823F0010303623B
:10AB2000036A4168846923F0020324F073042C4310
:10AB300015692B43556823F001032B433F4DA84271
:10AB400012D1556923F0080343EA8503956823F081
:10AB5000040343EA8503956921F480712943D5698B
:10AB600021F4007141EA4501D26841608461426389
:10AB700003620020A7E7036A156823F0100303624D
:10AB8000036A4168846923F0200324F4E64444EA1C
:10AB90000524156943EA0513556823F0100343EAB9
:10ABA0000513264DA84213D1556923F0800343EACB
:10ABB0008513956823F0400343EA8513956921F4D2
:10ABC000806141EA8501D56921F4006141EAC5014E
:10ABD000D268416084618263CAE7036A156823F41E
:10ABE00080730362036A4168C46923F4007324F02C
:10ABF00073042C43156943EA0523556823F48073D5
:10AC000043EA05230D4DA84213D1556923F400638F
:10AC100043EA8523956823F4806343EA8523956995
:10AC200021F4805141EA0511D56921F4005141EA2E
:10AC30004511D2684160C461C26399E7002C0140AC
:10AC4000154B98420BD103F55843DA6842F4804221
:10AC5000DA60DA6822F48042DA60002070470F4B35
:10AC600098420AD103F5E6331A6942F400321A61B8
:10AC70001A6922F400321A61EFE7094B984209D1B0
:10AC800003F5E4331A6942F480221A611A6922F446
:10AC90008022F0E701207047003801400044004066
:10ACA0000048004030B5C36804469B040D4685B09B
:10ACB00002D5012005B030BD4B68C968C2680B439E
:10ACC000296922F4B0520B4322F00C021343C360F3
:10ACD0000369AA6823F440531343036143696A6913
:10ACE00023F44073134343616846FFF76BFE134B35
:10ACF0009C4219D1039B002BDBD02A68002AD8D0B4
:10AD000019214B439200B3FBF2F36422B3FBF2F13F
:10AD100002FB11331B013233B3FBF2F303EB0113DC
:10AD20009BB20020A360C5E7054B9C4201D1029B6A
:10AD3000E1E7044B9C42BCD1F9E700BF0038014079
:10AD4000004400400048004030B5302442F20F7506
:10AD5000A84212D80C703021B0F57A7F14D211704D
:10AD60003022632816D81A703023092817D8039A7E
:10AD700030301370049B187030BDA0F51C500134A6
:10AD80001038E4B280B2E3E70131A0F57A70C9B2BD
:10AD900080B2E1E701326438D2B280B2E1E7013338
:10ADA0000A38DBB280B2E0E713B50B1D0193CB1C70
:10ADB00000934A1C8B1C0C46FFF7C6FF00236371EF
:10ADC00002B010BD03099F2894BF303337330B7096
:10ADD000002300F00F00092894BF3030373048704E
:10ADE0008B70704708B50249FFF7ECFF084608BDB5
:10ADF000C82C00202DE9F34105460C4600278E188B
:10AE0000B44202D102B0BDE8F0812B682246D3F8EB
:10AE10000880284601238DF807700DF10701C0470F
:10AE20000134EDE7F7B505460C468E18B44201D162
:10AE300003B0F0BD14F8013B28468DF807302B68AD
:10AE40000DF106029F680DF107010123B847EDE7F8
:10AE500007B503688DF8071001221B690DF1070182
:10AE6000984703B05DF804FB024A02600022C0E983
:10AE700001227047D4D100082DE9F0410D46044667
:10AE800016461F4603681B68984765F07F012046F9
:10AE9000C9B2FFF7DDFF236820463A4631461B69F9
:10AEA000984723682046BDE8F0415B68184707B51E
:10AEB00001238DF807200DF10702FFF7DDFF03B036
:10AEC0005DF804FB2DE9F04104460F4615461E4689
:10AED00003681B689847204607F07F01FFF7B8FF1B
:10AEE0002368204632462946DB6898472368204677
:10AEF000BDE8F0415B68184707B501230DF1070273
:10AF0000FFF7E0FF9DF8070003B05DF804FBF8B51C
:10AF100005460E4614461F46FFF7EEFF20EA0402E0
:10AF2000D2B23C40314628462243FFF7C0FFF8BD6D
:10AF300070B5044615461E460A460D21FFF7B7FFB9
:10AF400033462A462046BDE870400021FFF794BFF3
:10AF500070B5044615461E460A460D21FFF7A7FFA9
:10AF600033462A462046BDE870400021FFF7AABFBD
:10AF700008B500220121FFF79AFF08BD012208B59C
:10AF80001146FFF794FF08BD07B50B0C8DF8043090
:10AF90000B0A8DF805308DF806100323062101AA4F
:10AFA000FFF76AFF03B05DF804FB08B50A430C2104
:10AFB000FFF77DFF08BD902910B5044609D1022294
:10AFC0003621FFF774FF64223A212046FFF76FFF16
:10AFD00010BD03223621F9E7902970B505460C46CD
:10AFE00006D1BDE87040802331211A46FFF78FBF9C
:10AFF000002380223121FFF78AFF302C1ED00AD88F
:10B00000B4B1102C1AD0202C18D0002230212846A0
:10B01000FFF74DFF70BD602C08D003D804F0EF049B
:10B02000402CF1E7702C01D0802CEED1402200E0C2
:10B0300048222F212846FFF73AFFE6E74422F8E7A7
:10B0400038B5044615460A460E21FFF730FF2A465A
:10B050000F212046FFF72BFF38BD602938B5044685
:10B060000D4643EA020316D143F001021D21FFF70A
:10B070001EFF2B46F4221E212046FFF748FF072221
:10B08000052331212046FFF742FF0C2237212046BD
:10B09000FFF70DFF38BDFE221D21FFF738FF2B46BD
:10B0A000F0221E212046FFF732FF07220323312121
:10B0B0002046FFF72CFF0A22E8E72DE9F047044677
:10B0C0000F4616461D46002220219DF820909DF82F
:10B0D0002480FFF7ECFE3A4620462121FFF7E7FEE9
:10B0E0003346204601221D21FFF711FF4B46204623
:10B0F00004221E21FFF70BFF2A4620462221FFF7DC
:10B10000D6FE43462046BDE8F04741223321FFF7F3
:10B11000FEBE70B51646CA431D4604461121D2B282
:10B12000FFF7C5FE204646EA05024021FFF7BFFEB5
:10B130002046BDE870400023F1224121FFF7E7BE21
:10B14000122108B5FFF7D8FE80B208BD08B50A463F
:10B150001221FFF7ACFE08BD70B504460E46FFF79E
:10B16000EFFF0546F1B22046FFF7F0FF2046FFF75C
:10B1700005FF284670BD70B5044603F00F059DF825
:10B1800010602A430A430921FFF791FE3346204607
:10B19000BDE870400F220A21FFF7B9BE08B50322AF
:10B1A0000121FFF784FE08BD08B505220121FFF744
:10B1B0007EFE08BD70B50C461A2115460646FFF7FF
:10B1C0009BFE9D38208019213046FFF795FE40B246
:10B1D00003460028B8BFC31C9B102B700330BEBFB2
:10B1E00022889B18238070BD70B50E46132114462B
:10B1F0000546FFF781FE102130702846FFF77CFEE0
:10B20000207070BD08B54221FFF776FE08BD436887
:10B210008160C91AFFF7B8BE836810B504463BB316
:10B220002821FFF769FE10F0080F636800F007009F
:10B230000BD007280CBF03F1FF33043B6360626847
:10B240000D4B9A4209DA636007E090B901336360FD
:10B2500040F2666362689A42F5DC084B6268272117
:10B260005A43A3682046B2FBF3F2D2B2FFF71FFEA7
:10B2700010BD0433EBE700BF9AF9FFFFF07E0E002C
:10B28000C0F3C7537F3B162B014610B514DC002BCF
:10B2900007DA013300F0004101D141F07E51084648
:10B2A00010BD084A1A411042F9D04FF480011941EB
:10B2B000014421EA0201F2E7802BF0D1F4F760FFAC
:10B2C0000146ECE7FFFF7F00884210B501EB020466
:10B2D00002D98442234607D8431EA14208D011F860
:10B2E000012B03F8012FF8E7014602448A4200D1FE
:10B2F00010BD13F8014D02F8014DF7E70346024473
:10B30000934200D1704703F8011BF9E7024610B5DC
:10B31000147813460132002CFAD1013B11F8012BAD
:10B3200003F8012F002AF9D110BD0346C9B218460F
:10B3300013F8012B12B18A42F9D17047002918BFC6
:10B340000020704710B56AB10139841810F8012B3C
:10B3500011F8013F9A4203D1A04201D0002AF5D151
:10B36000D01A10BD1046FCE770B500260C4D0D4CF0
:10B37000641BA410A64209D100F030F800260A4D43
:10B380000A4C641BA410A64205D170BD55F8043BBD
:10B3900098470136EEE755F8043B98470136F2E747
:10B3A000E8D10008E8D10008E8D10008F0D1000891
:10B3B000034611F8012B03F8012B002AF9D170473D
:10B3C0000A44914200F1FF3300D1704710B511F8E3
:10B3D000014B914203F8014FF9D110BDF8B500BF00
:10B3E000F8BC08BC9E467047F8B500BFF8BC08BC66
:04B3F0009E467047BE
:10B3F40000206C0002206A006D0074000205010246
:10B4040002016D696E2C00206D572C0020572C0012
:10B41400322E3447003931354D003836384D00343A
:10B4240033334D003730636D003836364D003F00FE
:10B434003530487A003331487A003139487A004649
:10B444004C52430046534B003139487A3778000157
:10B454001F136F011300000000D57FAAFE2B815437
:10B4640029FC5683D702A87D52872DF8AC79D306E0
:10B474007BAE04D18550FA2FA471DB0E5A8F25F0D0
:10B484008D58F22773A60CD9F623895C08DD77A2C0
:10B49400DF0AA07521F45E8B9D48E23763B61CC9B0
:10B4A400B461CB1E4A9F35E0CF1AB06531E44E9BA0
:10B4B400E633994C18CD67B239EC4693C712B86D90
:10B4C40010C56FBAEE3B91446BBE14C19540EA3F80
:10B4D40042973DE8BC69C316EF3A904511C46EBB70
:10B4E400C613B96C38ED4792BD68C21743963CE960
:10B4F4009441EB3E6ABF15C04B9E34E1B560CA1F50
:10B5040062B71DC89C49E33619CC66B3E732984D3F
:10B5140030E54F9ACE1BB16472A70DD88C59F3262F
:10B524005B8E24F1A570DA0F20F55F8ADE0BA1741F
:10B5340009DC76A3F722885DD603A97C28FD57820F
:10B54400FF2A805501D47EAB8451FB2E7AAF05D0FF
:10B55400AD78D20753862CF96162636465666768C7
:10B56400696A6B6C6D6E6F707172737475767778CF
:10B57400797A303132333435363738395F232D2EEA
:10B5840000000100010002000200020003000400A8
:10B594000500060008000A000C0010001400190041
:10B5A4002000280032003F00500064007D009E000F
:10B5B400C800FA003C019001F40176022003E8037C
:10B5C400E204DC05D00700000000000000000000D9
:10B5D400051100080000000000000000111100081F
:10B5E4000000000000000000ED1000086D6C727394
:10B5F4002E3000536574757053746172745374788B
:10B6040034527800536574757053746172744D616B
:10B61400726B65720021656E6421004672736B79EA
:10B624002052394D006D4C525301020304006D4CFD
:10B63400525304030201000A0040504152414D2F6D
:10B64400706172616D2E70636B006661696C20615C
:10B654000020005378206E6F74206F6B002E000062
:10B66400000000000000000095270008452700089E
:10B6740000000000000000005D1300087D130008B6
:10B68400A7220008D1220008EF220008A91F000801
:10B6940000000000000000001F1200088F260008B0
:10B6A4006125000825120008AF240008991300083A
:10B6B4000D250008411A0008D9240008A713000822
:10B6C40000000000000000001F1200082112000802
:10B6D4002312000825120008291200082B12000862
:10B6E4002F1200083312000835120008391200081E
:10B6F4000000000000000000234300087D43000810
:10B70400AB130008AF1300080000000000000000A5
:10B714001F120008CD130008231200082512000888
:10B72400BD7A0008357B000875640008ED640008E4
:10B734003512000839120008414E474C4500484F65
:10B7440052495A4F4E004E415620414C54484F4C9A
:10B75400440048454144494E4720484F4C44004822
:10B7640045414446524545004845414441444A0008
:10B7740043414D53544142004E41562052544800D7
:10B784004E415620504F53484F4C44004D414E5566
:10B79400414C00424545504552004C454453204FCE
:10B7A4004646004C4947485453004F5344204F46A3
:10B7B400460054454C454D45545259004155544F4B
:10B7C4002054554E4500424C41434B424F5800468D
:10B7D40041494C53414645004E4156205750004183
:10B7E4004952204D4F444500484F4D452052455342
:10B7F400455400474353204E41560046505620417D
:10B804004E474C45204D49580053555246414345F7
:10B8140000464C415045524F4E005455524E204123
:10B824005353495354004E4156204C41554E4348BE
:10B8340000534552564F204155544F5452494D00E0
:10B8440043414D45524120434F4E54524F4C2031B9
:10B854000043414D45524120434F4E54524F4C20DA
:10B86400320043414D45524120434F4E54524F4CB8
:10B874002033004F534420414C542031004F534453
:10B8840020414C542032004F534420414C54203327
:10B89400004E415620434F5552534520484F4C4487
:10B8A400004D43204252414B494E470055534552A7
:10B8B40031005553455232005553455233005553C8
:10B8C400455234004C4F49544552204348414E4759
:10B8D40045004D5350205243204F5645525249443F
:10B8E400450050524541524D00545552544C450068
:10B8F4004E415620435255495345004155544F201B
:10B904004C4556454C205452494D00575020504CFC
:10B91400414E4E455200534F4152494E47004D4906
:10B924005353494F4E204348414E474500424545F5
:10B93400504552204D555445004D554C54492046D0
:10B94400554E4354494F4E004D495845522050528C
:10B954004F46494C452032004D49584552205452D7
:10B96400414E534954494F4E00414E474C4520489F
:10B974004F4C4400000102050304800CD007B704B7
:10B98400C71B800CB7040410020A0B06972304108B
:10B994000B06000000000000000000000000000092
:10B9A4000000000010CD00082B000000CDCF0008DF
:10B9B40001000000E8CC00080A000000CCCF000819
:10B9C4000100000000000000000000000000000072
:10B9D4000000000000000000000000000000000063
:10B9E4000000000000000000000000000000000053
:10B9F40000000000030002000A000A0014006400B2
:10BA04001800FA001B00F4011E00E803616263647D
:10BA140065666768696A6B6C6D6E6F70717273745A
:10BA240075767778797A3031323334353637383938
:10BA34005F232D2E0000000000070E091C1B1215A9
:10BA4400383F363124232A2D70777E796C6B6265FA
:10BA5400484F464154535A5DE0E7EEE9FCFBF2F5EA
:10BA6400D8DFD6D1C4C3CACD90979E998C8B8285DA
:10BA7400A8AFA6A1B4B3BABDC7C0C9CEDBDCD5D2CA
:10BA8400FFF8F1F6E3E4EDEAB7B0B9BEABACA5A2BA
:10BA94008F88818693949D9A2720292E3B3C3532AA
:10BAA4001F18111603040D0A5750595E4B4C45429A
:10BAB4006F68616673747D7A898E878095929B9C8A
:10BAC400B1B6BFB8ADAAA3A4F9FEF7F0E5E2EBEC7A
:10BAD400C1C6CFC8DDDAD3D4696E676075727B7C6A
:10BAE40051565F584D4A4344191E171005020B0C5A
:10BAF40021262F283D3A33344E49404752555C5B4A
:10BB04007671787F6A6D64633E39303722252C2B39
:10BB14000601080F1A1D1413AEA9A0A7B2B5BCBB29
:10BB24009691989F8A8D8483DED9D0D7C2C5CCCB19
:10BB3400E6E1E8EFFAFDF4F300000000320900004A
:10BB440000000000010000007C2B00000000000049
:10BB540002000000890C0000000000000400000046
:10BB6400ED0E030C0D00000005000000D91C0100BF
:10BB74000000000006000000680300000000000050
:10BB8400070000007720000000000000080000000B
:10BB940075240000000000000B0000005906010499
:10BBA40000000000130000008918030405000000D1
:10BBB40014000000D6140302030000001500000066
:10BBC4009F0203000100000016000000DC190000C1
:10BBD4000000000017000000A8170304050000007F
:10BBE40018000000183400000000000019000000D4
:10BBF40017650000000000001A000000AA180000E9
:10BC0400000000001B000000901D00000000000068
:10BC14001C00000043100000000000001D00000094
:10BC240073100000000000001E000000271C00002C
:10BC3400000000001F000000F630000000000000BB
:10BC440020000000B91C00000000000021000000DA
:10BC5400681C00000000000022000000ED16000037
:10BC64000000000023000000F416000000000000A3
:10BC740024000000DE250000000000002500000074
:10BC8400D40703040500000026000000090703048C
:10BC94000500000027000000FE260320210000000C
:10BCA40028000000E605030203000000290000004C
:10BCB4001C040302030000002A0000001C12000000
:10BCC400000000002B0000008403030001000000BA
:10BCD4002C000000DD090302030000002D00000019
:10BCE400E8030300010000002E0000000B02000026
:10BCF400000000002F00000099080300010000006C
:10BD0400300000002915010C000000003100000083
:10BD14002714000000000000320000004E2503122A
:10BD24001300000033000000C405030203000000F8
:10BD3400350000000305000000000000360000008C
:10BD44000F1B03181900000037000000031900003E
:10BD5400000000003D000000A748000000000000B3
:10BD64003E000000B71A0000000000003F00000081
:10BD740077B500000000000040000000BFE10000B3
:10BD84000000000041000000762A000000000000CE
:10BD94004200000094060302030000004300000078
:10BDA400150400000000000045000000F31E010A15
:10BDB40000000000460000007C2603101100000073
:10BDC4004900000026260320210000004A0000004C
:10BDD40014140000000000004B0000009E23031E0A
:10BDE4001F0000004C0000009821031E1F000000EB
:10BDF4004D0000008F0A03080900000050000000F5
:10BE04000E04030203000000510000006A16000043
:10BE1400000000005200000031330324250000001C
:10BE2400530000001625000000000000540000002C
:10BE34008F35033233000000550000008C330000BE
:10BE440000000000560000000535033233000000F6
:10BE54005700000096330000000000005900000065
:10BE6400E71C0000000000005A000000B738000082
:10BE7400000000005B0000003F2A000000000000FA
:10BE84005C00000036210000000000005D0000009E
:10BE94002F5100000000000064000000AF220000E9
:10BEA400000000006500000066750000000000004E
:10BEB400660000009E75000000000000670000009E
:10BEC400D039000000000000680000003874000051
:10BED40000000000690000005D3F00000000000059
:10BEE4006A0000008A2C0000000000006B000000C3
:10BEF4006C410000000000006C000000205C0000A9
:10BF0400000000006D000000B909000000000000FE
:10BF14006E00000054FE0301020000006F000000E8
:10BF2400221203101100000070000000AE0C00008B
:10BF340000000000710000007C27000000000000E9
:10BF440072000000ED2C00000000000073000000EF
:10BF54000440000000000000740000004C180000C1
:10BF640000000000750000008006030405000000C6
:10BF740076000000380E000000000000770000008A
:10BF8400740C030A0B0000007800000086610000B6
:10BF94000000000079000000ED0203000100000031
:10BFA4007A000000CB020300010000007B000000C7
:10BFB400FA710300010000007C0000005739000002
:10BFC400000000007D000000CB060000000000001F
:10BFD4007E000000DC51034F500000007F00000091
:10BFE400192300000000000080000000E22300008C
:10BFF40000000000810000002E1800000000000076
:10C00400820000001D0D00000000000083000000FD
:10C01400DFFF00000000000084000000552700003E
:10C02400000000008500000006120000000000006F
:10C0340086000000E52B00000000000087000000DF
:10C04400CB0800000000000088000000011600007A
:10C054000000000089000000C31000000000000080
:10C064008A0000006D780000000000008B000000D2
:10C07400A82B03292A0000008C000000B529000029
:10C08400000000008D0000002F20000000000000D0
:10C094008E00000048F30000000000008F00000044
:10C0A4008310000000000000900000007F5D00008D
:10C0B400000000009200000067640000000000001F
:10C0C400930000009A360000000000009400000075
:10C0D400B24E00000000000095000000C83C0000C3
:10C0E4000000000096000000862A00000000000006
:10C0F40097000000DB08030607000000980000001A
:10C10400D00800000000000099000000BC0C0000F2
:10C11400000000009A000000540F0306070000000E
:10C124009B000000160D0304050000009C000000A5
:10C1340013060300010000009D000000150F030C0E
:10C144000D0000009E000000860F030C0D0000008F
:10C15400A00000004E0C030809000000A10000002C
:10C164004403030001000000A2000000BD09000018
:10C1740000000000A30000007F1C0000000000007D
:10C18400A40000009A2C000000000000A50000009C
:10C194001503000000000000A600000015090000BF
:10C1A40000000000A700000090160000000000003E
:10C1B400A8000000010C000000000000A90000001D
:10C1C400EA12000000000000AA000000492200005A
:10C1D40000000000AB000000B542000000000000B9
:10C1E400AC0000001662000000000000AD0000007A
:10C1F4005308000000000000AE000000A73000005B
:10C2040000000000AF0000008A13030E0F000000BE
:10C21400B0000000EA03030001000000B1000000C8
:10C22400F014000000000000B20000002F1800000D
:10C2340000000000B3000000BD1D011A0000000052
:10C24400B4000000342F012A00000000B5000000F3
:10C25400AE04000000000000B6000000E528000065
:10C2640000000000B70000005502030001000000B8
:10C27400B80000009FCE030405000000B9000000D0
:10C28400BA07030405000000BA000000481D0300BB
:10C2940001000000BF0000005C1B00000000000063
:10C2A400C00000002436000000000000C1000000AF
:10C2B400471A000000000000C200000062210000D4
:10C2C40000000000C300000078250000000000000A
:10C2D400C8000000862A032829000000C9000000C5
:10C2E400CD0E030C0D000000D60000004508030627
:10C2F40007000000D70000006503000000000000F4
:10C30400D80000003203030001000000D90000003F
:10C31400CA06000000000000DA0000001107030054
:10C3240001000000DB000000A20200000000000089
:10C33400DC0000002220000000000000DD000000FE
:10C34400472A000000000000DE0000000F03000088
:10C3540000000000DF000000772F032A2B000000FC
:10C36400E0000000662D032A2B000000E10000001D
:10C37400D049000000000000E2000000CF080000E7
:10C3840000000000E6000000A32A000000000000F6
:10C39400E70000006928000000000000E800000039
:10C3A4009741000000000000E900000023B60000EF
:10C3B40000000000EA0000009628000000000000D1
:10C3C400EB000000B32A000000000000F1000000B0
:10C3D4005A20000000000000F2000000683C000049
:10C3E40000000000F3000000553D0134000000008F
:10C3F400F40000005F06000000000000F5000000EB
:10C404008202000000000000F6000000B8260000D0
:10C4140000000000F70000005113000000000000BD
:10C42400F800000008FE030304000000F900000007
:10C43400CC24000000000000FA000000311E0000BF
:10C4440000000000FB000000AA1200000000000031
:10C45400FC0000002C12000000000000FD000000A1
:10C464005336000000000000FE0000002E0900000A
:10C474000000000000010000472A03080900000032
:10C484000101000083090000000000000201000017
:10C49400BBE8030001000000030100005CED0000A4
:10C4A4000000000004010000920E000000000000E3
:10C4B40005010000B33D000000000000060100007B
:10C4C4000C170000000000000701000085FF0000B9
:10C4D40000000000080100003120000000000000FE
:10C4E400090100001A140000000000000A01000005
:10C4F400C1FF0302030000000B01000023FF03023D
:10C50400030000000C0100000E04030203000000FD
:10C514000D0100006DD70000000000000E010000B6
:10C524003B140000000000000F010000163500005D
:10C5340000000000130100007E2000000000000045
:10C544001401000012320000000000001501000078
:10C554003E1E0000000000001801000046210000FB
:10C564000000000019010000300D00000000000070
:10C574001A0100007B230320210000001B0100009E
:10C584004A910000000000001C0100006320031E0B
:10C594001F0000001D010000893103262700000050
:10C5A4001E010000D2390332330000001F010000D5
:10C5B40001170314150000002001000014170314D0
:10C5C4001500000022010000FB2E00000000000006
:10C5D400230100000A3900000000000027010000C8
:10C5E400EA0C0000000000002A010000ED25000014
:10C5F400000000002B010000136200000000000096
:10C604002C010000D9160000000000002D010000DC
:10C61400F33A000000000000360100001C11000085
:10C6240000000000370100005F74000000000000FB
:10C6340040010000F3140302030000004101000064
:10C64400580203000100000042010000F3950000BD
:10C6540000000000430100004E93030001000000AD
:10C664004401000084920000000000004A01000020
:10C6740017A70000000000004B0100005BE9000068
:10C68400000000004C010000ECEF0000000000007E
:10C694004D010000E76D0000000000004E010000A5
:10C6A400480A0000000000004F010000E1180000EB
:10C6B4000000000050010000F554000000000000DC
:10C6C40053010000C70500000000000054010000F1
:10C6D40063460000000000005E010000E8FC00006A
:10C6E4000000000062010000D20E030C0D000000E7
:10C6F40063010000060C0000000000006801000057
:10C704000B19000000000000690100005D21000019
:10C7140000000000710100009718000000000000F4
:10C72400720100001A8C0000000000007301000078
:10C734000A1A00000000000075010000752A0000BC
:10C744000000000077010000FB8C000000000000E6
:10C7540078010000C7080000000000007C01000010
:10C76400E81400000000000081010000938503022A
:10C77400030000008201000084100304050000008F
:10C784008301000004480304050000008401000044
:10C794000825032021000000860100009CEE000013
:10C7A400000000008B01000000D400000000000025
:10C7B4008C01000032A00000000000008D01000088
:10C7C400B66C000000000000900100006EFE03043F
:10C7D4000500000091010000B706030405000000F5
:10C7E4009A010000A0350000000000009B01000039
:10C7F4006A030000000000009C01000021060304FD
:10C80400050000009D0100004D0703040500000021
:10C814009E0100006D100000000000009F01000058
:10C82400A110000000000000A40100001449030648
:10C8340007000000B3010000862E00000000000085
:10C84400B4010000C109000000000000B5010000AF
:10C854001E01000000000000B80100004223000097
:10C8640000000000B9010000A91100000000000050
:10C87400FE010000F56A000000000000FF01000056
:10C884001C47000000000000421F0000DA100000F6
:10C8940000000000431F0000E72900000000000022
:10C8A400441F0000AC62000000000000451F0000AF
:10C8B400FB26000000000000461F0000610E00007F
:10C8C40000000000471F000040200000000000009E
:10C8D400481F0000EA21000000000000491F00007A
:10C8E40090100000000000004A1F00009B29000077
:10C8F400000000004B1F0000146600000000000050
:10C904004C1F000036100000000000004D1F000006
:10C91400DE2E0000000000004E1F0000C80E0000C4
:10C92400000000004F1F0000171800000000000066
:10C93400501F000095120000000000002823000092
:10C9440071890000000000002D2300007522000002
:10C954000000000011270000D114000000000000B6
:10C9640012270000BA29000000000000132700006D
:10C974000401000000000000A7270000C3550000C8
:10C9840000000000F82A00008634030405000000BB
:10C99400F92A00000F88000000000000FA2A0000B5
:10C9A400EAB4030405000000FB2A0000400500006F
:10C9B40000000000FC2A00000BE803080900000046
:10C9C400FD2A00005DE6000000000000022B0000CC
:10C9D4002E31000000000000032B00006A2C000030
:10C9E400000000000C2B0000CD100000000000002F
:10C9F400162B0000902C000000000000172B0000F4
:10CA0400852C000000000000182B0000552C0000AD
:10CA140000000000192B0000C325031011000000C2
:10CA24001A2B00004F050000000000001B2B000023
:10CA340080080304050000001C2B0000B122000044
:10CA4400000000001D2B0000821C000000000000FC
:10CA54001E2B00002F260000000000001F2B0000EA
:10CA64008E09000000000000202B0000842C000030
:10CA740000000000212B0000D02C0000000000006A
:10CA8400222B0000C92C000000000000232B000012
:10CA9400C12C000000000000242B0000BD2C00006D
:10CAA4000000000064320000722C0300010000004A
:10CAB40065320000FE3B031E1F00000066320000CA
:10CAC4008C3503040500000067320000F92E0300D2
:10CAD40001000000683200004D36031C1D000000F8
:10CAE40069320000312B03000100000073320000A2
:10CAF4005EF9030001000000763200008B33000071
:10CB0400000000007732000007120310110000003B
:10CB140078320000140500000000000068420000A4
:10CB240067B3000000000000FE4200001A2100006C
:10CB340000000000FF420000481000000000000058
:10CB44000143000013110000000000000243000034
:10CB54005911000000000000034300001B0A0000FC
:10CB640000000000044300000E5B00000000000011
:10CB740005430000BB540000000000000643000011
:10CB84006A1800000000000010A40000E301000087
:10CB94000000000011A40000EF2E000000000000BF
:10CBA40051C30000F62000000000000052C3000042
:10CBB400B5F600000000000053C300003E1300005F
:10CBC4000000000054C30000F00A0308090000003C
:10CBD40055C30000980603040500000020CB0000A4
:10CBE4000D6400000000000021CB0000EF010000F4
:10CBF4000000000022CB000018010000000000002B
:10CC040023CB0000A61A00000000000024CB000083
:10CC1400270100000000000025CB00009101000066
:10CC24000000000060EA0000041603141500000070
:10CC34006AEA0000D0210000000000006BEA000056
:10CC4400B7070000000000006CEA00006324032022
:10CC5400210000006DEA0000811803141500000093
:10CC64006EEA0000860803040500000074EA000070
:10CC7400CA0400000000000088EA00009CF50000DF
:10CC84000000000089EA0000BFFF0000000000006F
:10CC94008DEA00000E170302030000008EEA000074
:10CCA400AB1C0308090000008FEA000037070000EE
:10CCB4000000000092EA0000DC0E0000000000000A
:10CCC40093EA0000F51800000000000094EA000058
:10CCD400652C00000000000095EA00002D0600000D
:10CCE4000000000099D1D70033F3D700CC14D8004A
:10CCF4006636D8000058D8009979D800339BD800FC
:10CD0400CCBCD80066DED8000000D9009999E100B7
:10CD140000C0E10066E6E100CC0CE2003333E2003F
:10CD24009959E2000080E20066A6E200CCCCE20061
:10CD340033F3E2009919E3000040E3006666E30080
:10CD4400CC8CE30033B3E30099D9E3000000E400A2
:10CD54006626E400CC4CE4003373E4009999E400C3
:10CD640000C0E40066E6E400CC0CE5003333E500E3
:10CD74009959E5000080E50066A6E500CCCCE50005
:10CD840033F3E5009919E6000040E6006666E60024
:10CD9400CC8CE60033B3E60099D9E6000000E70046
:10CDA4006626E700CC4CE7003373E7009999E70067
:10CDB40000C0E70066E6E7000000891112239B32F9
:10CDC4002446AD573665BF74488CC19D5AAFD3BE57
:10CDD4006CCAE5DB7EE9F7F88110080193331A2267
:10CDE400A5562C47B7753E64C99C408DDBBF52AE37
:10CDF400EDDA64CBFFF976E802218B301002991347
:10CE04002667AF763444BD554AADC3BC588ED19F16
:10CE14006EEBE7FA7CC8F5D983310A209112180326
:10CE2400A7772E66B5543C45CBBD42ACD99E508FF6
:10CE3400EFFB66EAFDD874C904428D5316619F70F6
:10CE44002004A9153227BB364CCEC5DF5EEDD7FCD6
:10CE54006888E1997AABF3BA85520C4397711E60E6
:10CE6400A1142805B3373A26CDDE44CFDFFD56ECB6
:10CE7400E9986089FBBB72AA06638F7214409D51C6
:10CE84002225AB343006B9174EEFC7FE5CCCD5DD96
:10CE94006AA9E3B8788AF19B87730E6295501C41A6
:10CEA400A3352A24B1163807CFFF46EEDDDC54CD76
:10CEB400EBB962A8F99A708B088481951AA793B686
:10CEC4002CC2A5D33EE1B7F04008C919522BDB3A76
:10CED400644EED5F766DFF7C899400859BB712A646
:10CEE400ADD224C3BFF136E0C1184809D33B5A2A56
:10CEF400E55E6C4FF77D7E6C0AA583B41886919726
:10CF04002EE3A7F23CC0B5D14229CB38500AD91B35
:10CF1400666FEF7E744CFD5D8BB502A49996108705
:10CF2400AFF326E2BDD034C1C3394A28D11A580B15
:10CF3400E77F6E6EF55C7C4D0CC685D71EE597F4D5
:10CF44002880A1913AA3B3B2444ACD5B5669DF78F5
:10CF5400600CE91D722FFB3E8DD604C79FF516E4C5
:10CF6400A9902081BBB332A2C55A4C4BD7795E68D5
:10CF7400E11C680DF33F7A2E0EE787F61CC495D5A5
:10CF84002AA1A3B03882B193466BCF7A5448DD59B5
:10CF9400622DEB3C700EF91F8FF706E69DD414C585
:10CFA400ABB122A0B9923083C77B4E6AD5585C4995
:10CFB400E33D6A2CF11E780F6090020C015B0001C6
:10CFC4001C57000090FF000000130000E9B800089F
:10CFD400000000003CB700080200000042B700084F
:10CFE400030000004AB700080400000056B7000818
:10CFF4000500000063B70008060000006CB70008D5
:10D00400FF00000074B70008FF0000007CB70008B0
:10D014000700000084B700080800000090B700086B
:10D024000900000097B70008FF0000009EB7000841
:10D03400FF000000A7B70008FF000000AEB700081B
:10D04400FF000000B6B70008FF000000C0B70008EA
:10D054000A000000CAB70008FF000000D3B70008A8
:10D0640001000000DCB700080B000000E3B7000873
:10D074000C000000ECB70008FF000000F7B7000840
:10D08400FF000000FFB70008FF0000000DB8000813
:10D09400FF00000015B800080D0000001EB80008CD
:10D0A4000E0000002AB800080F00000035B8000880
:10D0B400FF00000044B80008FF00000055B8000855
:10D0C400FF00000066B80008FF00000077B8000801
:10D0D400FF00000081B80008FF0000008BB80008C2
:10D0E400FF00000095B8000810000000A5B8000873
:10D0F400FF000000B0B80008FF000000B6B8000848
:10D10400FF000000BCB80008FF000000C2B800081F
:10D11400FF000000C8B80008FF000000D6B80008EF
:10D12400FF000000E6B80008FF000000EDB80008AA
:10D1340011000000F4B8000812000000FFB8000855
:10D14400FF0000000FB90008FF0000001AB9000832
:10D154001300000022B90008FF00000031B90008E4
:10D16400FF0000003DB90008FF0000004CB90008B2
:10D17400FF0000005CB90008FF0000006DB9000862
:10D18400140000000000000000000000D58E00081C
:10D19400D78E0008AB130008AF130008000000008E
:10D1A4000000000001020304060708090000000053
:10D1B4000102030402030405060708090A0B0C0D07
:10D1C4000E0F10100102000000000000000000001B
:10D1D400000000000000000000000000F5AD0008A1
:04D1E40025AE00086C
:08D1E80035010008218E00084A
:04D1F0001101000821
:10D1F40090BADCFE785634120A000000CCB600085F
:10D204009CB60008FF00000014B700080024F400D6
:08D21400010000001000000001
:04000005080098C196
:00000001FF
